
ultrasonic_sensor.elf:     file format elf32-littlearm

Sections:
Idx Name          Size      VMA       LMA       File off  Algn
  0 .isr_vector   000000c0  08000000  08000000  00010000  2**0
                  CONTENTS, ALLOC, LOAD, READONLY, DATA
  1 .text         00009f60  080000c0  080000c0  000100c0  2**2
                  CONTENTS, ALLOC, LOAD, READONLY, CODE
  2 .rodata       000005ac  0800a020  0800a020  0001a020  2**3
                  CONTENTS, ALLOC, LOAD, READONLY, DATA
  3 .ARM.extab    00000000  0800a5cc  0800a5cc  000201e0  2**0
                  CONTENTS
  4 .ARM          00000008  0800a5cc  0800a5cc  0001a5cc  2**2
                  CONTENTS, ALLOC, LOAD, READONLY, DATA
  5 .preinit_array 00000000  0800a5d4  0800a5d4  000201e0  2**0
                  CONTENTS, ALLOC, LOAD, DATA
  6 .init_array   00000004  0800a5d4  0800a5d4  0001a5d4  2**2
                  CONTENTS, ALLOC, LOAD, DATA
  7 .fini_array   00000004  0800a5d8  0800a5d8  0001a5d8  2**2
                  CONTENTS, ALLOC, LOAD, DATA
  8 .data         000001e0  20000000  0800a5dc  00020000  2**2
                  CONTENTS, ALLOC, LOAD, DATA
  9 .bss          00000164  200001e0  0800a7bc  000201e0  2**2
                  ALLOC
 10 ._user_heap_stack 00000604  20000344  0800a7bc  00020344  2**0
                  ALLOC
 11 .ARM.attributes 00000028  00000000  00000000  000201e0  2**0
                  CONTENTS, READONLY
 12 .debug_info   0000c5a6  00000000  00000000  00020208  2**0
                  CONTENTS, READONLY, DEBUGGING, OCTETS
 13 .debug_abbrev 00001ab6  00000000  00000000  0002c7ae  2**0
                  CONTENTS, READONLY, DEBUGGING, OCTETS
 14 .debug_aranges 00000b78  00000000  00000000  0002e268  2**3
                  CONTENTS, READONLY, DEBUGGING, OCTETS
 15 .debug_ranges 00000ac0  00000000  00000000  0002ede0  2**3
                  CONTENTS, READONLY, DEBUGGING, OCTETS
 16 .debug_macro  000158bc  00000000  00000000  0002f8a0  2**0
                  CONTENTS, READONLY, DEBUGGING, OCTETS
 17 .debug_line   0000ce0f  00000000  00000000  0004515c  2**0
                  CONTENTS, READONLY, DEBUGGING, OCTETS
 18 .debug_str    00084976  00000000  00000000  00051f6b  2**0
                  CONTENTS, READONLY, DEBUGGING, OCTETS
 19 .comment      00000050  00000000  00000000  000d68e1  2**0
                  CONTENTS, READONLY
 20 .debug_frame  00003ed8  00000000  00000000  000d6934  2**2
                  CONTENTS, READONLY, DEBUGGING, OCTETS

Disassembly of section .text:

080000c0 <__do_global_dtors_aux>:
 80000c0:	b510      	push	{r4, lr}
 80000c2:	4c06      	ldr	r4, [pc, #24]	; (80000dc <__do_global_dtors_aux+0x1c>)
 80000c4:	7823      	ldrb	r3, [r4, #0]
 80000c6:	2b00      	cmp	r3, #0
 80000c8:	d107      	bne.n	80000da <__do_global_dtors_aux+0x1a>
 80000ca:	4b05      	ldr	r3, [pc, #20]	; (80000e0 <__do_global_dtors_aux+0x20>)
 80000cc:	2b00      	cmp	r3, #0
 80000ce:	d002      	beq.n	80000d6 <__do_global_dtors_aux+0x16>
 80000d0:	4804      	ldr	r0, [pc, #16]	; (80000e4 <__do_global_dtors_aux+0x24>)
 80000d2:	e000      	b.n	80000d6 <__do_global_dtors_aux+0x16>
 80000d4:	bf00      	nop
 80000d6:	2301      	movs	r3, #1
 80000d8:	7023      	strb	r3, [r4, #0]
 80000da:	bd10      	pop	{r4, pc}
 80000dc:	200001e0 	.word	0x200001e0
 80000e0:	00000000 	.word	0x00000000
 80000e4:	0800a008 	.word	0x0800a008

080000e8 <frame_dummy>:
 80000e8:	4b04      	ldr	r3, [pc, #16]	; (80000fc <frame_dummy+0x14>)
 80000ea:	b510      	push	{r4, lr}
 80000ec:	2b00      	cmp	r3, #0
 80000ee:	d003      	beq.n	80000f8 <frame_dummy+0x10>
 80000f0:	4903      	ldr	r1, [pc, #12]	; (8000100 <frame_dummy+0x18>)
 80000f2:	4804      	ldr	r0, [pc, #16]	; (8000104 <frame_dummy+0x1c>)
 80000f4:	e000      	b.n	80000f8 <frame_dummy+0x10>
 80000f6:	bf00      	nop
 80000f8:	bd10      	pop	{r4, pc}
 80000fa:	46c0      	nop			; (mov r8, r8)
 80000fc:	00000000 	.word	0x00000000
 8000100:	200001e4 	.word	0x200001e4
 8000104:	0800a008 	.word	0x0800a008

08000108 <strlen>:
 8000108:	2300      	movs	r3, #0
 800010a:	5cc2      	ldrb	r2, [r0, r3]
 800010c:	3301      	adds	r3, #1
 800010e:	2a00      	cmp	r2, #0
 8000110:	d1fb      	bne.n	800010a <strlen+0x2>
 8000112:	1e58      	subs	r0, r3, #1
 8000114:	4770      	bx	lr
	...

08000118 <__gnu_thumb1_case_uqi>:
 8000118:	b402      	push	{r1}
 800011a:	4671      	mov	r1, lr
 800011c:	0849      	lsrs	r1, r1, #1
 800011e:	0049      	lsls	r1, r1, #1
 8000120:	5c09      	ldrb	r1, [r1, r0]
 8000122:	0049      	lsls	r1, r1, #1
 8000124:	448e      	add	lr, r1
 8000126:	bc02      	pop	{r1}
 8000128:	4770      	bx	lr
 800012a:	46c0      	nop			; (mov r8, r8)

0800012c <__gnu_thumb1_case_shi>:
 800012c:	b403      	push	{r0, r1}
 800012e:	4671      	mov	r1, lr
 8000130:	0849      	lsrs	r1, r1, #1
 8000132:	0040      	lsls	r0, r0, #1
 8000134:	0049      	lsls	r1, r1, #1
 8000136:	5e09      	ldrsh	r1, [r1, r0]
 8000138:	0049      	lsls	r1, r1, #1
 800013a:	448e      	add	lr, r1
 800013c:	bc03      	pop	{r0, r1}
 800013e:	4770      	bx	lr

08000140 <__udivsi3>:
 8000140:	2200      	movs	r2, #0
 8000142:	0843      	lsrs	r3, r0, #1
 8000144:	428b      	cmp	r3, r1
 8000146:	d374      	bcc.n	8000232 <__udivsi3+0xf2>
 8000148:	0903      	lsrs	r3, r0, #4
 800014a:	428b      	cmp	r3, r1
 800014c:	d35f      	bcc.n	800020e <__udivsi3+0xce>
 800014e:	0a03      	lsrs	r3, r0, #8
 8000150:	428b      	cmp	r3, r1
 8000152:	d344      	bcc.n	80001de <__udivsi3+0x9e>
 8000154:	0b03      	lsrs	r3, r0, #12
 8000156:	428b      	cmp	r3, r1
 8000158:	d328      	bcc.n	80001ac <__udivsi3+0x6c>
 800015a:	0c03      	lsrs	r3, r0, #16
 800015c:	428b      	cmp	r3, r1
 800015e:	d30d      	bcc.n	800017c <__udivsi3+0x3c>
 8000160:	22ff      	movs	r2, #255	; 0xff
 8000162:	0209      	lsls	r1, r1, #8
 8000164:	ba12      	rev	r2, r2
 8000166:	0c03      	lsrs	r3, r0, #16
 8000168:	428b      	cmp	r3, r1
 800016a:	d302      	bcc.n	8000172 <__udivsi3+0x32>
 800016c:	1212      	asrs	r2, r2, #8
 800016e:	0209      	lsls	r1, r1, #8
 8000170:	d065      	beq.n	800023e <__udivsi3+0xfe>
 8000172:	0b03      	lsrs	r3, r0, #12
 8000174:	428b      	cmp	r3, r1
 8000176:	d319      	bcc.n	80001ac <__udivsi3+0x6c>
 8000178:	e000      	b.n	800017c <__udivsi3+0x3c>
 800017a:	0a09      	lsrs	r1, r1, #8
 800017c:	0bc3      	lsrs	r3, r0, #15
 800017e:	428b      	cmp	r3, r1
 8000180:	d301      	bcc.n	8000186 <__udivsi3+0x46>
 8000182:	03cb      	lsls	r3, r1, #15
 8000184:	1ac0      	subs	r0, r0, r3
 8000186:	4152      	adcs	r2, r2
 8000188:	0b83      	lsrs	r3, r0, #14
 800018a:	428b      	cmp	r3, r1
 800018c:	d301      	bcc.n	8000192 <__udivsi3+0x52>
 800018e:	038b      	lsls	r3, r1, #14
 8000190:	1ac0      	subs	r0, r0, r3
 8000192:	4152      	adcs	r2, r2
 8000194:	0b43      	lsrs	r3, r0, #13
 8000196:	428b      	cmp	r3, r1
 8000198:	d301      	bcc.n	800019e <__udivsi3+0x5e>
 800019a:	034b      	lsls	r3, r1, #13
 800019c:	1ac0      	subs	r0, r0, r3
 800019e:	4152      	adcs	r2, r2
 80001a0:	0b03      	lsrs	r3, r0, #12
 80001a2:	428b      	cmp	r3, r1
 80001a4:	d301      	bcc.n	80001aa <__udivsi3+0x6a>
 80001a6:	030b      	lsls	r3, r1, #12
 80001a8:	1ac0      	subs	r0, r0, r3
 80001aa:	4152      	adcs	r2, r2
 80001ac:	0ac3      	lsrs	r3, r0, #11
 80001ae:	428b      	cmp	r3, r1
 80001b0:	d301      	bcc.n	80001b6 <__udivsi3+0x76>
 80001b2:	02cb      	lsls	r3, r1, #11
 80001b4:	1ac0      	subs	r0, r0, r3
 80001b6:	4152      	adcs	r2, r2
 80001b8:	0a83      	lsrs	r3, r0, #10
 80001ba:	428b      	cmp	r3, r1
 80001bc:	d301      	bcc.n	80001c2 <__udivsi3+0x82>
 80001be:	028b      	lsls	r3, r1, #10
 80001c0:	1ac0      	subs	r0, r0, r3
 80001c2:	4152      	adcs	r2, r2
 80001c4:	0a43      	lsrs	r3, r0, #9
 80001c6:	428b      	cmp	r3, r1
 80001c8:	d301      	bcc.n	80001ce <__udivsi3+0x8e>
 80001ca:	024b      	lsls	r3, r1, #9
 80001cc:	1ac0      	subs	r0, r0, r3
 80001ce:	4152      	adcs	r2, r2
 80001d0:	0a03      	lsrs	r3, r0, #8
 80001d2:	428b      	cmp	r3, r1
 80001d4:	d301      	bcc.n	80001da <__udivsi3+0x9a>
 80001d6:	020b      	lsls	r3, r1, #8
 80001d8:	1ac0      	subs	r0, r0, r3
 80001da:	4152      	adcs	r2, r2
 80001dc:	d2cd      	bcs.n	800017a <__udivsi3+0x3a>
 80001de:	09c3      	lsrs	r3, r0, #7
 80001e0:	428b      	cmp	r3, r1
 80001e2:	d301      	bcc.n	80001e8 <__udivsi3+0xa8>
 80001e4:	01cb      	lsls	r3, r1, #7
 80001e6:	1ac0      	subs	r0, r0, r3
 80001e8:	4152      	adcs	r2, r2
 80001ea:	0983      	lsrs	r3, r0, #6
 80001ec:	428b      	cmp	r3, r1
 80001ee:	d301      	bcc.n	80001f4 <__udivsi3+0xb4>
 80001f0:	018b      	lsls	r3, r1, #6
 80001f2:	1ac0      	subs	r0, r0, r3
 80001f4:	4152      	adcs	r2, r2
 80001f6:	0943      	lsrs	r3, r0, #5
 80001f8:	428b      	cmp	r3, r1
 80001fa:	d301      	bcc.n	8000200 <__udivsi3+0xc0>
 80001fc:	014b      	lsls	r3, r1, #5
 80001fe:	1ac0      	subs	r0, r0, r3
 8000200:	4152      	adcs	r2, r2
 8000202:	0903      	lsrs	r3, r0, #4
 8000204:	428b      	cmp	r3, r1
 8000206:	d301      	bcc.n	800020c <__udivsi3+0xcc>
 8000208:	010b      	lsls	r3, r1, #4
 800020a:	1ac0      	subs	r0, r0, r3
 800020c:	4152      	adcs	r2, r2
 800020e:	08c3      	lsrs	r3, r0, #3
 8000210:	428b      	cmp	r3, r1
 8000212:	d301      	bcc.n	8000218 <__udivsi3+0xd8>
 8000214:	00cb      	lsls	r3, r1, #3
 8000216:	1ac0      	subs	r0, r0, r3
 8000218:	4152      	adcs	r2, r2
 800021a:	0883      	lsrs	r3, r0, #2
 800021c:	428b      	cmp	r3, r1
 800021e:	d301      	bcc.n	8000224 <__udivsi3+0xe4>
 8000220:	008b      	lsls	r3, r1, #2
 8000222:	1ac0      	subs	r0, r0, r3
 8000224:	4152      	adcs	r2, r2
 8000226:	0843      	lsrs	r3, r0, #1
 8000228:	428b      	cmp	r3, r1
 800022a:	d301      	bcc.n	8000230 <__udivsi3+0xf0>
 800022c:	004b      	lsls	r3, r1, #1
 800022e:	1ac0      	subs	r0, r0, r3
 8000230:	4152      	adcs	r2, r2
 8000232:	1a41      	subs	r1, r0, r1
 8000234:	d200      	bcs.n	8000238 <__udivsi3+0xf8>
 8000236:	4601      	mov	r1, r0
 8000238:	4152      	adcs	r2, r2
 800023a:	4610      	mov	r0, r2
 800023c:	4770      	bx	lr
 800023e:	e7ff      	b.n	8000240 <__udivsi3+0x100>
 8000240:	b501      	push	{r0, lr}
 8000242:	2000      	movs	r0, #0
 8000244:	f000 f8f0 	bl	8000428 <__aeabi_idiv0>
 8000248:	bd02      	pop	{r1, pc}
 800024a:	46c0      	nop			; (mov r8, r8)

0800024c <__aeabi_uidivmod>:
 800024c:	2900      	cmp	r1, #0
 800024e:	d0f7      	beq.n	8000240 <__udivsi3+0x100>
 8000250:	e776      	b.n	8000140 <__udivsi3>
 8000252:	4770      	bx	lr

08000254 <__divsi3>:
 8000254:	4603      	mov	r3, r0
 8000256:	430b      	orrs	r3, r1
 8000258:	d47f      	bmi.n	800035a <__divsi3+0x106>
 800025a:	2200      	movs	r2, #0
 800025c:	0843      	lsrs	r3, r0, #1
 800025e:	428b      	cmp	r3, r1
 8000260:	d374      	bcc.n	800034c <__divsi3+0xf8>
 8000262:	0903      	lsrs	r3, r0, #4
 8000264:	428b      	cmp	r3, r1
 8000266:	d35f      	bcc.n	8000328 <__divsi3+0xd4>
 8000268:	0a03      	lsrs	r3, r0, #8
 800026a:	428b      	cmp	r3, r1
 800026c:	d344      	bcc.n	80002f8 <__divsi3+0xa4>
 800026e:	0b03      	lsrs	r3, r0, #12
 8000270:	428b      	cmp	r3, r1
 8000272:	d328      	bcc.n	80002c6 <__divsi3+0x72>
 8000274:	0c03      	lsrs	r3, r0, #16
 8000276:	428b      	cmp	r3, r1
 8000278:	d30d      	bcc.n	8000296 <__divsi3+0x42>
 800027a:	22ff      	movs	r2, #255	; 0xff
 800027c:	0209      	lsls	r1, r1, #8
 800027e:	ba12      	rev	r2, r2
 8000280:	0c03      	lsrs	r3, r0, #16
 8000282:	428b      	cmp	r3, r1
 8000284:	d302      	bcc.n	800028c <__divsi3+0x38>
 8000286:	1212      	asrs	r2, r2, #8
 8000288:	0209      	lsls	r1, r1, #8
 800028a:	d065      	beq.n	8000358 <__divsi3+0x104>
 800028c:	0b03      	lsrs	r3, r0, #12
 800028e:	428b      	cmp	r3, r1
 8000290:	d319      	bcc.n	80002c6 <__divsi3+0x72>
 8000292:	e000      	b.n	8000296 <__divsi3+0x42>
 8000294:	0a09      	lsrs	r1, r1, #8
 8000296:	0bc3      	lsrs	r3, r0, #15
 8000298:	428b      	cmp	r3, r1
 800029a:	d301      	bcc.n	80002a0 <__divsi3+0x4c>
 800029c:	03cb      	lsls	r3, r1, #15
 800029e:	1ac0      	subs	r0, r0, r3
 80002a0:	4152      	adcs	r2, r2
 80002a2:	0b83      	lsrs	r3, r0, #14
 80002a4:	428b      	cmp	r3, r1
 80002a6:	d301      	bcc.n	80002ac <__divsi3+0x58>
 80002a8:	038b      	lsls	r3, r1, #14
 80002aa:	1ac0      	subs	r0, r0, r3
 80002ac:	4152      	adcs	r2, r2
 80002ae:	0b43      	lsrs	r3, r0, #13
 80002b0:	428b      	cmp	r3, r1
 80002b2:	d301      	bcc.n	80002b8 <__divsi3+0x64>
 80002b4:	034b      	lsls	r3, r1, #13
 80002b6:	1ac0      	subs	r0, r0, r3
 80002b8:	4152      	adcs	r2, r2
 80002ba:	0b03      	lsrs	r3, r0, #12
 80002bc:	428b      	cmp	r3, r1
 80002be:	d301      	bcc.n	80002c4 <__divsi3+0x70>
 80002c0:	030b      	lsls	r3, r1, #12
 80002c2:	1ac0      	subs	r0, r0, r3
 80002c4:	4152      	adcs	r2, r2
 80002c6:	0ac3      	lsrs	r3, r0, #11
 80002c8:	428b      	cmp	r3, r1
 80002ca:	d301      	bcc.n	80002d0 <__divsi3+0x7c>
 80002cc:	02cb      	lsls	r3, r1, #11
 80002ce:	1ac0      	subs	r0, r0, r3
 80002d0:	4152      	adcs	r2, r2
 80002d2:	0a83      	lsrs	r3, r0, #10
 80002d4:	428b      	cmp	r3, r1
 80002d6:	d301      	bcc.n	80002dc <__divsi3+0x88>
 80002d8:	028b      	lsls	r3, r1, #10
 80002da:	1ac0      	subs	r0, r0, r3
 80002dc:	4152      	adcs	r2, r2
 80002de:	0a43      	lsrs	r3, r0, #9
 80002e0:	428b      	cmp	r3, r1
 80002e2:	d301      	bcc.n	80002e8 <__divsi3+0x94>
 80002e4:	024b      	lsls	r3, r1, #9
 80002e6:	1ac0      	subs	r0, r0, r3
 80002e8:	4152      	adcs	r2, r2
 80002ea:	0a03      	lsrs	r3, r0, #8
 80002ec:	428b      	cmp	r3, r1
 80002ee:	d301      	bcc.n	80002f4 <__divsi3+0xa0>
 80002f0:	020b      	lsls	r3, r1, #8
 80002f2:	1ac0      	subs	r0, r0, r3
 80002f4:	4152      	adcs	r2, r2
 80002f6:	d2cd      	bcs.n	8000294 <__divsi3+0x40>
 80002f8:	09c3      	lsrs	r3, r0, #7
 80002fa:	428b      	cmp	r3, r1
 80002fc:	d301      	bcc.n	8000302 <__divsi3+0xae>
 80002fe:	01cb      	lsls	r3, r1, #7
 8000300:	1ac0      	subs	r0, r0, r3
 8000302:	4152      	adcs	r2, r2
 8000304:	0983      	lsrs	r3, r0, #6
 8000306:	428b      	cmp	r3, r1
 8000308:	d301      	bcc.n	800030e <__divsi3+0xba>
 800030a:	018b      	lsls	r3, r1, #6
 800030c:	1ac0      	subs	r0, r0, r3
 800030e:	4152      	adcs	r2, r2
 8000310:	0943      	lsrs	r3, r0, #5
 8000312:	428b      	cmp	r3, r1
 8000314:	d301      	bcc.n	800031a <__divsi3+0xc6>
 8000316:	014b      	lsls	r3, r1, #5
 8000318:	1ac0      	subs	r0, r0, r3
 800031a:	4152      	adcs	r2, r2
 800031c:	0903      	lsrs	r3, r0, #4
 800031e:	428b      	cmp	r3, r1
 8000320:	d301      	bcc.n	8000326 <__divsi3+0xd2>
 8000322:	010b      	lsls	r3, r1, #4
 8000324:	1ac0      	subs	r0, r0, r3
 8000326:	4152      	adcs	r2, r2
 8000328:	08c3      	lsrs	r3, r0, #3
 800032a:	428b      	cmp	r3, r1
 800032c:	d301      	bcc.n	8000332 <__divsi3+0xde>
 800032e:	00cb      	lsls	r3, r1, #3
 8000330:	1ac0      	subs	r0, r0, r3
 8000332:	4152      	adcs	r2, r2
 8000334:	0883      	lsrs	r3, r0, #2
 8000336:	428b      	cmp	r3, r1
 8000338:	d301      	bcc.n	800033e <__divsi3+0xea>
 800033a:	008b      	lsls	r3, r1, #2
 800033c:	1ac0      	subs	r0, r0, r3
 800033e:	4152      	adcs	r2, r2
 8000340:	0843      	lsrs	r3, r0, #1
 8000342:	428b      	cmp	r3, r1
 8000344:	d301      	bcc.n	800034a <__divsi3+0xf6>
 8000346:	004b      	lsls	r3, r1, #1
 8000348:	1ac0      	subs	r0, r0, r3
 800034a:	4152      	adcs	r2, r2
 800034c:	1a41      	subs	r1, r0, r1
 800034e:	d200      	bcs.n	8000352 <__divsi3+0xfe>
 8000350:	4601      	mov	r1, r0
 8000352:	4152      	adcs	r2, r2
 8000354:	4610      	mov	r0, r2
 8000356:	4770      	bx	lr
 8000358:	e05d      	b.n	8000416 <__divsi3+0x1c2>
 800035a:	0fca      	lsrs	r2, r1, #31
 800035c:	d000      	beq.n	8000360 <__divsi3+0x10c>
 800035e:	4249      	negs	r1, r1
 8000360:	1003      	asrs	r3, r0, #32
 8000362:	d300      	bcc.n	8000366 <__divsi3+0x112>
 8000364:	4240      	negs	r0, r0
 8000366:	4053      	eors	r3, r2
 8000368:	2200      	movs	r2, #0
 800036a:	469c      	mov	ip, r3
 800036c:	0903      	lsrs	r3, r0, #4
 800036e:	428b      	cmp	r3, r1
 8000370:	d32d      	bcc.n	80003ce <__divsi3+0x17a>
 8000372:	0a03      	lsrs	r3, r0, #8
 8000374:	428b      	cmp	r3, r1
 8000376:	d312      	bcc.n	800039e <__divsi3+0x14a>
 8000378:	22fc      	movs	r2, #252	; 0xfc
 800037a:	0189      	lsls	r1, r1, #6
 800037c:	ba12      	rev	r2, r2
 800037e:	0a03      	lsrs	r3, r0, #8
 8000380:	428b      	cmp	r3, r1
 8000382:	d30c      	bcc.n	800039e <__divsi3+0x14a>
 8000384:	0189      	lsls	r1, r1, #6
 8000386:	1192      	asrs	r2, r2, #6
 8000388:	428b      	cmp	r3, r1
 800038a:	d308      	bcc.n	800039e <__divsi3+0x14a>
 800038c:	0189      	lsls	r1, r1, #6
 800038e:	1192      	asrs	r2, r2, #6
 8000390:	428b      	cmp	r3, r1
 8000392:	d304      	bcc.n	800039e <__divsi3+0x14a>
 8000394:	0189      	lsls	r1, r1, #6
 8000396:	d03a      	beq.n	800040e <__divsi3+0x1ba>
 8000398:	1192      	asrs	r2, r2, #6
 800039a:	e000      	b.n	800039e <__divsi3+0x14a>
 800039c:	0989      	lsrs	r1, r1, #6
 800039e:	09c3      	lsrs	r3, r0, #7
 80003a0:	428b      	cmp	r3, r1
 80003a2:	d301      	bcc.n	80003a8 <__divsi3+0x154>
 80003a4:	01cb      	lsls	r3, r1, #7
 80003a6:	1ac0      	subs	r0, r0, r3
 80003a8:	4152      	adcs	r2, r2
 80003aa:	0983      	lsrs	r3, r0, #6
 80003ac:	428b      	cmp	r3, r1
 80003ae:	d301      	bcc.n	80003b4 <__divsi3+0x160>
 80003b0:	018b      	lsls	r3, r1, #6
 80003b2:	1ac0      	subs	r0, r0, r3
 80003b4:	4152      	adcs	r2, r2
 80003b6:	0943      	lsrs	r3, r0, #5
 80003b8:	428b      	cmp	r3, r1
 80003ba:	d301      	bcc.n	80003c0 <__divsi3+0x16c>
 80003bc:	014b      	lsls	r3, r1, #5
 80003be:	1ac0      	subs	r0, r0, r3
 80003c0:	4152      	adcs	r2, r2
 80003c2:	0903      	lsrs	r3, r0, #4
 80003c4:	428b      	cmp	r3, r1
 80003c6:	d301      	bcc.n	80003cc <__divsi3+0x178>
 80003c8:	010b      	lsls	r3, r1, #4
 80003ca:	1ac0      	subs	r0, r0, r3
 80003cc:	4152      	adcs	r2, r2
 80003ce:	08c3      	lsrs	r3, r0, #3
 80003d0:	428b      	cmp	r3, r1
 80003d2:	d301      	bcc.n	80003d8 <__divsi3+0x184>
 80003d4:	00cb      	lsls	r3, r1, #3
 80003d6:	1ac0      	subs	r0, r0, r3
 80003d8:	4152      	adcs	r2, r2
 80003da:	0883      	lsrs	r3, r0, #2
 80003dc:	428b      	cmp	r3, r1
 80003de:	d301      	bcc.n	80003e4 <__divsi3+0x190>
 80003e0:	008b      	lsls	r3, r1, #2
 80003e2:	1ac0      	subs	r0, r0, r3
 80003e4:	4152      	adcs	r2, r2
 80003e6:	d2d9      	bcs.n	800039c <__divsi3+0x148>
 80003e8:	0843      	lsrs	r3, r0, #1
 80003ea:	428b      	cmp	r3, r1
 80003ec:	d301      	bcc.n	80003f2 <__divsi3+0x19e>
 80003ee:	004b      	lsls	r3, r1, #1
 80003f0:	1ac0      	subs	r0, r0, r3
 80003f2:	4152      	adcs	r2, r2
 80003f4:	1a41      	subs	r1, r0, r1
 80003f6:	d200      	bcs.n	80003fa <__divsi3+0x1a6>
 80003f8:	4601      	mov	r1, r0
 80003fa:	4663      	mov	r3, ip
 80003fc:	4152      	adcs	r2, r2
 80003fe:	105b      	asrs	r3, r3, #1
 8000400:	4610      	mov	r0, r2
 8000402:	d301      	bcc.n	8000408 <__divsi3+0x1b4>
 8000404:	4240      	negs	r0, r0
 8000406:	2b00      	cmp	r3, #0
 8000408:	d500      	bpl.n	800040c <__divsi3+0x1b8>
 800040a:	4249      	negs	r1, r1
 800040c:	4770      	bx	lr
 800040e:	4663      	mov	r3, ip
 8000410:	105b      	asrs	r3, r3, #1
 8000412:	d300      	bcc.n	8000416 <__divsi3+0x1c2>
 8000414:	4240      	negs	r0, r0
 8000416:	b501      	push	{r0, lr}
 8000418:	2000      	movs	r0, #0
 800041a:	f000 f805 	bl	8000428 <__aeabi_idiv0>
 800041e:	bd02      	pop	{r1, pc}

08000420 <__aeabi_idivmod>:
 8000420:	2900      	cmp	r1, #0
 8000422:	d0f8      	beq.n	8000416 <__divsi3+0x1c2>
 8000424:	e716      	b.n	8000254 <__divsi3>
 8000426:	4770      	bx	lr

08000428 <__aeabi_idiv0>:
 8000428:	4770      	bx	lr
 800042a:	46c0      	nop			; (mov r8, r8)

0800042c <__aeabi_cdrcmple>:
 800042c:	4684      	mov	ip, r0
 800042e:	0010      	movs	r0, r2
 8000430:	4662      	mov	r2, ip
 8000432:	468c      	mov	ip, r1
 8000434:	0019      	movs	r1, r3
 8000436:	4663      	mov	r3, ip
 8000438:	e000      	b.n	800043c <__aeabi_cdcmpeq>
 800043a:	46c0      	nop			; (mov r8, r8)

0800043c <__aeabi_cdcmpeq>:
 800043c:	b51f      	push	{r0, r1, r2, r3, r4, lr}
 800043e:	f001 fa77 	bl	8001930 <__ledf2>
 8000442:	2800      	cmp	r0, #0
 8000444:	d401      	bmi.n	800044a <__aeabi_cdcmpeq+0xe>
 8000446:	2100      	movs	r1, #0
 8000448:	42c8      	cmn	r0, r1
 800044a:	bd1f      	pop	{r0, r1, r2, r3, r4, pc}

0800044c <__aeabi_dcmpeq>:
 800044c:	b510      	push	{r4, lr}
 800044e:	f001 f9c7 	bl	80017e0 <__eqdf2>
 8000452:	4240      	negs	r0, r0
 8000454:	3001      	adds	r0, #1
 8000456:	bd10      	pop	{r4, pc}

08000458 <__aeabi_dcmplt>:
 8000458:	b510      	push	{r4, lr}
 800045a:	f001 fa69 	bl	8001930 <__ledf2>
 800045e:	2800      	cmp	r0, #0
 8000460:	db01      	blt.n	8000466 <__aeabi_dcmplt+0xe>
 8000462:	2000      	movs	r0, #0
 8000464:	bd10      	pop	{r4, pc}
 8000466:	2001      	movs	r0, #1
 8000468:	bd10      	pop	{r4, pc}
 800046a:	46c0      	nop			; (mov r8, r8)

0800046c <__aeabi_dcmple>:
 800046c:	b510      	push	{r4, lr}
 800046e:	f001 fa5f 	bl	8001930 <__ledf2>
 8000472:	2800      	cmp	r0, #0
 8000474:	dd01      	ble.n	800047a <__aeabi_dcmple+0xe>
 8000476:	2000      	movs	r0, #0
 8000478:	bd10      	pop	{r4, pc}
 800047a:	2001      	movs	r0, #1
 800047c:	bd10      	pop	{r4, pc}
 800047e:	46c0      	nop			; (mov r8, r8)

08000480 <__aeabi_dcmpgt>:
 8000480:	b510      	push	{r4, lr}
 8000482:	f001 f9ef 	bl	8001864 <__gedf2>
 8000486:	2800      	cmp	r0, #0
 8000488:	dc01      	bgt.n	800048e <__aeabi_dcmpgt+0xe>
 800048a:	2000      	movs	r0, #0
 800048c:	bd10      	pop	{r4, pc}
 800048e:	2001      	movs	r0, #1
 8000490:	bd10      	pop	{r4, pc}
 8000492:	46c0      	nop			; (mov r8, r8)

08000494 <__aeabi_dcmpge>:
 8000494:	b510      	push	{r4, lr}
 8000496:	f001 f9e5 	bl	8001864 <__gedf2>
 800049a:	2800      	cmp	r0, #0
 800049c:	da01      	bge.n	80004a2 <__aeabi_dcmpge+0xe>
 800049e:	2000      	movs	r0, #0
 80004a0:	bd10      	pop	{r4, pc}
 80004a2:	2001      	movs	r0, #1
 80004a4:	bd10      	pop	{r4, pc}
 80004a6:	46c0      	nop			; (mov r8, r8)

080004a8 <__aeabi_uldivmod>:
 80004a8:	2b00      	cmp	r3, #0
 80004aa:	d111      	bne.n	80004d0 <__aeabi_uldivmod+0x28>
 80004ac:	2a00      	cmp	r2, #0
 80004ae:	d10f      	bne.n	80004d0 <__aeabi_uldivmod+0x28>
 80004b0:	2900      	cmp	r1, #0
 80004b2:	d100      	bne.n	80004b6 <__aeabi_uldivmod+0xe>
 80004b4:	2800      	cmp	r0, #0
 80004b6:	d002      	beq.n	80004be <__aeabi_uldivmod+0x16>
 80004b8:	2100      	movs	r1, #0
 80004ba:	43c9      	mvns	r1, r1
 80004bc:	0008      	movs	r0, r1
 80004be:	b407      	push	{r0, r1, r2}
 80004c0:	4802      	ldr	r0, [pc, #8]	; (80004cc <__aeabi_uldivmod+0x24>)
 80004c2:	a102      	add	r1, pc, #8	; (adr r1, 80004cc <__aeabi_uldivmod+0x24>)
 80004c4:	1840      	adds	r0, r0, r1
 80004c6:	9002      	str	r0, [sp, #8]
 80004c8:	bd03      	pop	{r0, r1, pc}
 80004ca:	46c0      	nop			; (mov r8, r8)
 80004cc:	ffffff5d 	.word	0xffffff5d
 80004d0:	b403      	push	{r0, r1}
 80004d2:	4668      	mov	r0, sp
 80004d4:	b501      	push	{r0, lr}
 80004d6:	9802      	ldr	r0, [sp, #8]
 80004d8:	f000 f8a4 	bl	8000624 <__udivmoddi4>
 80004dc:	9b01      	ldr	r3, [sp, #4]
 80004de:	469e      	mov	lr, r3
 80004e0:	b002      	add	sp, #8
 80004e2:	bc0c      	pop	{r2, r3}
 80004e4:	4770      	bx	lr
 80004e6:	46c0      	nop			; (mov r8, r8)

080004e8 <__aeabi_lmul>:
 80004e8:	b5f0      	push	{r4, r5, r6, r7, lr}
 80004ea:	46ce      	mov	lr, r9
 80004ec:	4647      	mov	r7, r8
 80004ee:	b580      	push	{r7, lr}
 80004f0:	0007      	movs	r7, r0
 80004f2:	4699      	mov	r9, r3
 80004f4:	0c3b      	lsrs	r3, r7, #16
 80004f6:	469c      	mov	ip, r3
 80004f8:	0413      	lsls	r3, r2, #16
 80004fa:	0c1b      	lsrs	r3, r3, #16
 80004fc:	001d      	movs	r5, r3
 80004fe:	000e      	movs	r6, r1
 8000500:	4661      	mov	r1, ip
 8000502:	0400      	lsls	r0, r0, #16
 8000504:	0c14      	lsrs	r4, r2, #16
 8000506:	0c00      	lsrs	r0, r0, #16
 8000508:	4345      	muls	r5, r0
 800050a:	434b      	muls	r3, r1
 800050c:	4360      	muls	r0, r4
 800050e:	4361      	muls	r1, r4
 8000510:	18c0      	adds	r0, r0, r3
 8000512:	0c2c      	lsrs	r4, r5, #16
 8000514:	1820      	adds	r0, r4, r0
 8000516:	468c      	mov	ip, r1
 8000518:	4283      	cmp	r3, r0
 800051a:	d903      	bls.n	8000524 <__aeabi_lmul+0x3c>
 800051c:	2380      	movs	r3, #128	; 0x80
 800051e:	025b      	lsls	r3, r3, #9
 8000520:	4698      	mov	r8, r3
 8000522:	44c4      	add	ip, r8
 8000524:	4649      	mov	r1, r9
 8000526:	4379      	muls	r1, r7
 8000528:	4372      	muls	r2, r6
 800052a:	0c03      	lsrs	r3, r0, #16
 800052c:	4463      	add	r3, ip
 800052e:	042d      	lsls	r5, r5, #16
 8000530:	0c2d      	lsrs	r5, r5, #16
 8000532:	18c9      	adds	r1, r1, r3
 8000534:	0400      	lsls	r0, r0, #16
 8000536:	1940      	adds	r0, r0, r5
 8000538:	1889      	adds	r1, r1, r2
 800053a:	bcc0      	pop	{r6, r7}
 800053c:	46b9      	mov	r9, r7
 800053e:	46b0      	mov	r8, r6
 8000540:	bdf0      	pop	{r4, r5, r6, r7, pc}
 8000542:	46c0      	nop			; (mov r8, r8)

08000544 <__aeabi_d2uiz>:
 8000544:	b570      	push	{r4, r5, r6, lr}
 8000546:	2200      	movs	r2, #0
 8000548:	4b0c      	ldr	r3, [pc, #48]	; (800057c <__aeabi_d2uiz+0x38>)
 800054a:	0004      	movs	r4, r0
 800054c:	000d      	movs	r5, r1
 800054e:	f7ff ffa1 	bl	8000494 <__aeabi_dcmpge>
 8000552:	2800      	cmp	r0, #0
 8000554:	d104      	bne.n	8000560 <__aeabi_d2uiz+0x1c>
 8000556:	0020      	movs	r0, r4
 8000558:	0029      	movs	r1, r5
 800055a:	f002 f869 	bl	8002630 <__aeabi_d2iz>
 800055e:	bd70      	pop	{r4, r5, r6, pc}
 8000560:	4b06      	ldr	r3, [pc, #24]	; (800057c <__aeabi_d2uiz+0x38>)
 8000562:	2200      	movs	r2, #0
 8000564:	0020      	movs	r0, r4
 8000566:	0029      	movs	r1, r5
 8000568:	f001 fcb2 	bl	8001ed0 <__aeabi_dsub>
 800056c:	f002 f860 	bl	8002630 <__aeabi_d2iz>
 8000570:	2380      	movs	r3, #128	; 0x80
 8000572:	061b      	lsls	r3, r3, #24
 8000574:	469c      	mov	ip, r3
 8000576:	4460      	add	r0, ip
 8000578:	e7f1      	b.n	800055e <__aeabi_d2uiz+0x1a>
 800057a:	46c0      	nop			; (mov r8, r8)
 800057c:	41e00000 	.word	0x41e00000

08000580 <__aeabi_d2lz>:
 8000580:	b570      	push	{r4, r5, r6, lr}
 8000582:	0005      	movs	r5, r0
 8000584:	000c      	movs	r4, r1
 8000586:	2200      	movs	r2, #0
 8000588:	2300      	movs	r3, #0
 800058a:	0028      	movs	r0, r5
 800058c:	0021      	movs	r1, r4
 800058e:	f7ff ff63 	bl	8000458 <__aeabi_dcmplt>
 8000592:	2800      	cmp	r0, #0
 8000594:	d108      	bne.n	80005a8 <__aeabi_d2lz+0x28>
 8000596:	0028      	movs	r0, r5
 8000598:	0021      	movs	r1, r4
 800059a:	f000 f80f 	bl	80005bc <__aeabi_d2ulz>
 800059e:	0002      	movs	r2, r0
 80005a0:	000b      	movs	r3, r1
 80005a2:	0010      	movs	r0, r2
 80005a4:	0019      	movs	r1, r3
 80005a6:	bd70      	pop	{r4, r5, r6, pc}
 80005a8:	2380      	movs	r3, #128	; 0x80
 80005aa:	061b      	lsls	r3, r3, #24
 80005ac:	18e1      	adds	r1, r4, r3
 80005ae:	0028      	movs	r0, r5
 80005b0:	f000 f804 	bl	80005bc <__aeabi_d2ulz>
 80005b4:	2300      	movs	r3, #0
 80005b6:	4242      	negs	r2, r0
 80005b8:	418b      	sbcs	r3, r1
 80005ba:	e7f2      	b.n	80005a2 <__aeabi_d2lz+0x22>

080005bc <__aeabi_d2ulz>:
 80005bc:	b570      	push	{r4, r5, r6, lr}
 80005be:	2200      	movs	r2, #0
 80005c0:	4b0b      	ldr	r3, [pc, #44]	; (80005f0 <__aeabi_d2ulz+0x34>)
 80005c2:	000d      	movs	r5, r1
 80005c4:	0004      	movs	r4, r0
 80005c6:	f001 fa17 	bl	80019f8 <__aeabi_dmul>
 80005ca:	f7ff ffbb 	bl	8000544 <__aeabi_d2uiz>
 80005ce:	0006      	movs	r6, r0
 80005d0:	f002 f894 	bl	80026fc <__aeabi_ui2d>
 80005d4:	2200      	movs	r2, #0
 80005d6:	4b07      	ldr	r3, [pc, #28]	; (80005f4 <__aeabi_d2ulz+0x38>)
 80005d8:	f001 fa0e 	bl	80019f8 <__aeabi_dmul>
 80005dc:	0002      	movs	r2, r0
 80005de:	000b      	movs	r3, r1
 80005e0:	0020      	movs	r0, r4
 80005e2:	0029      	movs	r1, r5
 80005e4:	f001 fc74 	bl	8001ed0 <__aeabi_dsub>
 80005e8:	f7ff ffac 	bl	8000544 <__aeabi_d2uiz>
 80005ec:	0031      	movs	r1, r6
 80005ee:	bd70      	pop	{r4, r5, r6, pc}
 80005f0:	3df00000 	.word	0x3df00000
 80005f4:	41f00000 	.word	0x41f00000

080005f8 <__aeabi_l2d>:
 80005f8:	b570      	push	{r4, r5, r6, lr}
 80005fa:	0006      	movs	r6, r0
 80005fc:	0008      	movs	r0, r1
 80005fe:	f002 f84d 	bl	800269c <__aeabi_i2d>
 8000602:	2200      	movs	r2, #0
 8000604:	4b06      	ldr	r3, [pc, #24]	; (8000620 <__aeabi_l2d+0x28>)
 8000606:	f001 f9f7 	bl	80019f8 <__aeabi_dmul>
 800060a:	000d      	movs	r5, r1
 800060c:	0004      	movs	r4, r0
 800060e:	0030      	movs	r0, r6
 8000610:	f002 f874 	bl	80026fc <__aeabi_ui2d>
 8000614:	002b      	movs	r3, r5
 8000616:	0022      	movs	r2, r4
 8000618:	f000 fab0 	bl	8000b7c <__aeabi_dadd>
 800061c:	bd70      	pop	{r4, r5, r6, pc}
 800061e:	46c0      	nop			; (mov r8, r8)
 8000620:	41f00000 	.word	0x41f00000

08000624 <__udivmoddi4>:
 8000624:	b5f0      	push	{r4, r5, r6, r7, lr}
 8000626:	4657      	mov	r7, sl
 8000628:	464e      	mov	r6, r9
 800062a:	4645      	mov	r5, r8
 800062c:	46de      	mov	lr, fp
 800062e:	b5e0      	push	{r5, r6, r7, lr}
 8000630:	0004      	movs	r4, r0
 8000632:	000d      	movs	r5, r1
 8000634:	4692      	mov	sl, r2
 8000636:	4699      	mov	r9, r3
 8000638:	b083      	sub	sp, #12
 800063a:	428b      	cmp	r3, r1
 800063c:	d830      	bhi.n	80006a0 <__udivmoddi4+0x7c>
 800063e:	d02d      	beq.n	800069c <__udivmoddi4+0x78>
 8000640:	4649      	mov	r1, r9
 8000642:	4650      	mov	r0, sl
 8000644:	f002 f96e 	bl	8002924 <__clzdi2>
 8000648:	0029      	movs	r1, r5
 800064a:	0006      	movs	r6, r0
 800064c:	0020      	movs	r0, r4
 800064e:	f002 f969 	bl	8002924 <__clzdi2>
 8000652:	1a33      	subs	r3, r6, r0
 8000654:	4698      	mov	r8, r3
 8000656:	3b20      	subs	r3, #32
 8000658:	469b      	mov	fp, r3
 800065a:	d433      	bmi.n	80006c4 <__udivmoddi4+0xa0>
 800065c:	465a      	mov	r2, fp
 800065e:	4653      	mov	r3, sl
 8000660:	4093      	lsls	r3, r2
 8000662:	4642      	mov	r2, r8
 8000664:	001f      	movs	r7, r3
 8000666:	4653      	mov	r3, sl
 8000668:	4093      	lsls	r3, r2
 800066a:	001e      	movs	r6, r3
 800066c:	42af      	cmp	r7, r5
 800066e:	d83a      	bhi.n	80006e6 <__udivmoddi4+0xc2>
 8000670:	42af      	cmp	r7, r5
 8000672:	d100      	bne.n	8000676 <__udivmoddi4+0x52>
 8000674:	e078      	b.n	8000768 <__udivmoddi4+0x144>
 8000676:	465b      	mov	r3, fp
 8000678:	1ba4      	subs	r4, r4, r6
 800067a:	41bd      	sbcs	r5, r7
 800067c:	2b00      	cmp	r3, #0
 800067e:	da00      	bge.n	8000682 <__udivmoddi4+0x5e>
 8000680:	e075      	b.n	800076e <__udivmoddi4+0x14a>
 8000682:	2200      	movs	r2, #0
 8000684:	2300      	movs	r3, #0
 8000686:	9200      	str	r2, [sp, #0]
 8000688:	9301      	str	r3, [sp, #4]
 800068a:	2301      	movs	r3, #1
 800068c:	465a      	mov	r2, fp
 800068e:	4093      	lsls	r3, r2
 8000690:	9301      	str	r3, [sp, #4]
 8000692:	2301      	movs	r3, #1
 8000694:	4642      	mov	r2, r8
 8000696:	4093      	lsls	r3, r2
 8000698:	9300      	str	r3, [sp, #0]
 800069a:	e028      	b.n	80006ee <__udivmoddi4+0xca>
 800069c:	4282      	cmp	r2, r0
 800069e:	d9cf      	bls.n	8000640 <__udivmoddi4+0x1c>
 80006a0:	2200      	movs	r2, #0
 80006a2:	2300      	movs	r3, #0
 80006a4:	9200      	str	r2, [sp, #0]
 80006a6:	9301      	str	r3, [sp, #4]
 80006a8:	9b0c      	ldr	r3, [sp, #48]	; 0x30
 80006aa:	2b00      	cmp	r3, #0
 80006ac:	d001      	beq.n	80006b2 <__udivmoddi4+0x8e>
 80006ae:	601c      	str	r4, [r3, #0]
 80006b0:	605d      	str	r5, [r3, #4]
 80006b2:	9800      	ldr	r0, [sp, #0]
 80006b4:	9901      	ldr	r1, [sp, #4]
 80006b6:	b003      	add	sp, #12
 80006b8:	bcf0      	pop	{r4, r5, r6, r7}
 80006ba:	46bb      	mov	fp, r7
 80006bc:	46b2      	mov	sl, r6
 80006be:	46a9      	mov	r9, r5
 80006c0:	46a0      	mov	r8, r4
 80006c2:	bdf0      	pop	{r4, r5, r6, r7, pc}
 80006c4:	4642      	mov	r2, r8
 80006c6:	2320      	movs	r3, #32
 80006c8:	1a9b      	subs	r3, r3, r2
 80006ca:	4652      	mov	r2, sl
 80006cc:	40da      	lsrs	r2, r3
 80006ce:	4641      	mov	r1, r8
 80006d0:	0013      	movs	r3, r2
 80006d2:	464a      	mov	r2, r9
 80006d4:	408a      	lsls	r2, r1
 80006d6:	0017      	movs	r7, r2
 80006d8:	4642      	mov	r2, r8
 80006da:	431f      	orrs	r7, r3
 80006dc:	4653      	mov	r3, sl
 80006de:	4093      	lsls	r3, r2
 80006e0:	001e      	movs	r6, r3
 80006e2:	42af      	cmp	r7, r5
 80006e4:	d9c4      	bls.n	8000670 <__udivmoddi4+0x4c>
 80006e6:	2200      	movs	r2, #0
 80006e8:	2300      	movs	r3, #0
 80006ea:	9200      	str	r2, [sp, #0]
 80006ec:	9301      	str	r3, [sp, #4]
 80006ee:	4643      	mov	r3, r8
 80006f0:	2b00      	cmp	r3, #0
 80006f2:	d0d9      	beq.n	80006a8 <__udivmoddi4+0x84>
 80006f4:	07fb      	lsls	r3, r7, #31
 80006f6:	0872      	lsrs	r2, r6, #1
 80006f8:	431a      	orrs	r2, r3
 80006fa:	4646      	mov	r6, r8
 80006fc:	087b      	lsrs	r3, r7, #1
 80006fe:	e00e      	b.n	800071e <__udivmoddi4+0xfa>
 8000700:	42ab      	cmp	r3, r5
 8000702:	d101      	bne.n	8000708 <__udivmoddi4+0xe4>
 8000704:	42a2      	cmp	r2, r4
 8000706:	d80c      	bhi.n	8000722 <__udivmoddi4+0xfe>
 8000708:	1aa4      	subs	r4, r4, r2
 800070a:	419d      	sbcs	r5, r3
 800070c:	2001      	movs	r0, #1
 800070e:	1924      	adds	r4, r4, r4
 8000710:	416d      	adcs	r5, r5
 8000712:	2100      	movs	r1, #0
 8000714:	3e01      	subs	r6, #1
 8000716:	1824      	adds	r4, r4, r0
 8000718:	414d      	adcs	r5, r1
 800071a:	2e00      	cmp	r6, #0
 800071c:	d006      	beq.n	800072c <__udivmoddi4+0x108>
 800071e:	42ab      	cmp	r3, r5
 8000720:	d9ee      	bls.n	8000700 <__udivmoddi4+0xdc>
 8000722:	3e01      	subs	r6, #1
 8000724:	1924      	adds	r4, r4, r4
 8000726:	416d      	adcs	r5, r5
 8000728:	2e00      	cmp	r6, #0
 800072a:	d1f8      	bne.n	800071e <__udivmoddi4+0xfa>
 800072c:	9800      	ldr	r0, [sp, #0]
 800072e:	9901      	ldr	r1, [sp, #4]
 8000730:	465b      	mov	r3, fp
 8000732:	1900      	adds	r0, r0, r4
 8000734:	4169      	adcs	r1, r5
 8000736:	2b00      	cmp	r3, #0
 8000738:	db24      	blt.n	8000784 <__udivmoddi4+0x160>
 800073a:	002b      	movs	r3, r5
 800073c:	465a      	mov	r2, fp
 800073e:	4644      	mov	r4, r8
 8000740:	40d3      	lsrs	r3, r2
 8000742:	002a      	movs	r2, r5
 8000744:	40e2      	lsrs	r2, r4
 8000746:	001c      	movs	r4, r3
 8000748:	465b      	mov	r3, fp
 800074a:	0015      	movs	r5, r2
 800074c:	2b00      	cmp	r3, #0
 800074e:	db2a      	blt.n	80007a6 <__udivmoddi4+0x182>
 8000750:	0026      	movs	r6, r4
 8000752:	409e      	lsls	r6, r3
 8000754:	0033      	movs	r3, r6
 8000756:	0026      	movs	r6, r4
 8000758:	4647      	mov	r7, r8
 800075a:	40be      	lsls	r6, r7
 800075c:	0032      	movs	r2, r6
 800075e:	1a80      	subs	r0, r0, r2
 8000760:	4199      	sbcs	r1, r3
 8000762:	9000      	str	r0, [sp, #0]
 8000764:	9101      	str	r1, [sp, #4]
 8000766:	e79f      	b.n	80006a8 <__udivmoddi4+0x84>
 8000768:	42a3      	cmp	r3, r4
 800076a:	d8bc      	bhi.n	80006e6 <__udivmoddi4+0xc2>
 800076c:	e783      	b.n	8000676 <__udivmoddi4+0x52>
 800076e:	4642      	mov	r2, r8
 8000770:	2320      	movs	r3, #32
 8000772:	2100      	movs	r1, #0
 8000774:	1a9b      	subs	r3, r3, r2
 8000776:	2200      	movs	r2, #0
 8000778:	9100      	str	r1, [sp, #0]
 800077a:	9201      	str	r2, [sp, #4]
 800077c:	2201      	movs	r2, #1
 800077e:	40da      	lsrs	r2, r3
 8000780:	9201      	str	r2, [sp, #4]
 8000782:	e786      	b.n	8000692 <__udivmoddi4+0x6e>
 8000784:	4642      	mov	r2, r8
 8000786:	2320      	movs	r3, #32
 8000788:	1a9b      	subs	r3, r3, r2
 800078a:	002a      	movs	r2, r5
 800078c:	4646      	mov	r6, r8
 800078e:	409a      	lsls	r2, r3
 8000790:	0023      	movs	r3, r4
 8000792:	40f3      	lsrs	r3, r6
 8000794:	4644      	mov	r4, r8
 8000796:	4313      	orrs	r3, r2
 8000798:	002a      	movs	r2, r5
 800079a:	40e2      	lsrs	r2, r4
 800079c:	001c      	movs	r4, r3
 800079e:	465b      	mov	r3, fp
 80007a0:	0015      	movs	r5, r2
 80007a2:	2b00      	cmp	r3, #0
 80007a4:	dad4      	bge.n	8000750 <__udivmoddi4+0x12c>
 80007a6:	4642      	mov	r2, r8
 80007a8:	002f      	movs	r7, r5
 80007aa:	2320      	movs	r3, #32
 80007ac:	0026      	movs	r6, r4
 80007ae:	4097      	lsls	r7, r2
 80007b0:	1a9b      	subs	r3, r3, r2
 80007b2:	40de      	lsrs	r6, r3
 80007b4:	003b      	movs	r3, r7
 80007b6:	4333      	orrs	r3, r6
 80007b8:	e7cd      	b.n	8000756 <__udivmoddi4+0x132>
 80007ba:	46c0      	nop			; (mov r8, r8)

080007bc <__aeabi_fadd>:
 80007bc:	b5f0      	push	{r4, r5, r6, r7, lr}
 80007be:	46c6      	mov	lr, r8
 80007c0:	0243      	lsls	r3, r0, #9
 80007c2:	0a5b      	lsrs	r3, r3, #9
 80007c4:	024e      	lsls	r6, r1, #9
 80007c6:	0045      	lsls	r5, r0, #1
 80007c8:	004f      	lsls	r7, r1, #1
 80007ca:	00da      	lsls	r2, r3, #3
 80007cc:	0fc4      	lsrs	r4, r0, #31
 80007ce:	469c      	mov	ip, r3
 80007d0:	0a70      	lsrs	r0, r6, #9
 80007d2:	4690      	mov	r8, r2
 80007d4:	b500      	push	{lr}
 80007d6:	0e2d      	lsrs	r5, r5, #24
 80007d8:	0e3f      	lsrs	r7, r7, #24
 80007da:	0fc9      	lsrs	r1, r1, #31
 80007dc:	09b6      	lsrs	r6, r6, #6
 80007de:	428c      	cmp	r4, r1
 80007e0:	d04b      	beq.n	800087a <__aeabi_fadd+0xbe>
 80007e2:	1bea      	subs	r2, r5, r7
 80007e4:	2a00      	cmp	r2, #0
 80007e6:	dd36      	ble.n	8000856 <__aeabi_fadd+0x9a>
 80007e8:	2f00      	cmp	r7, #0
 80007ea:	d061      	beq.n	80008b0 <__aeabi_fadd+0xf4>
 80007ec:	2dff      	cmp	r5, #255	; 0xff
 80007ee:	d100      	bne.n	80007f2 <__aeabi_fadd+0x36>
 80007f0:	e0ad      	b.n	800094e <__aeabi_fadd+0x192>
 80007f2:	2380      	movs	r3, #128	; 0x80
 80007f4:	04db      	lsls	r3, r3, #19
 80007f6:	431e      	orrs	r6, r3
 80007f8:	2a1b      	cmp	r2, #27
 80007fa:	dc00      	bgt.n	80007fe <__aeabi_fadd+0x42>
 80007fc:	e0d3      	b.n	80009a6 <__aeabi_fadd+0x1ea>
 80007fe:	2001      	movs	r0, #1
 8000800:	4643      	mov	r3, r8
 8000802:	1a18      	subs	r0, r3, r0
 8000804:	0143      	lsls	r3, r0, #5
 8000806:	d400      	bmi.n	800080a <__aeabi_fadd+0x4e>
 8000808:	e08c      	b.n	8000924 <__aeabi_fadd+0x168>
 800080a:	0180      	lsls	r0, r0, #6
 800080c:	0987      	lsrs	r7, r0, #6
 800080e:	0038      	movs	r0, r7
 8000810:	f002 f86a 	bl	80028e8 <__clzsi2>
 8000814:	3805      	subs	r0, #5
 8000816:	4087      	lsls	r7, r0
 8000818:	4285      	cmp	r5, r0
 800081a:	dc00      	bgt.n	800081e <__aeabi_fadd+0x62>
 800081c:	e0b6      	b.n	800098c <__aeabi_fadd+0x1d0>
 800081e:	1a2d      	subs	r5, r5, r0
 8000820:	48b3      	ldr	r0, [pc, #716]	; (8000af0 <__aeabi_fadd+0x334>)
 8000822:	4038      	ands	r0, r7
 8000824:	0743      	lsls	r3, r0, #29
 8000826:	d004      	beq.n	8000832 <__aeabi_fadd+0x76>
 8000828:	230f      	movs	r3, #15
 800082a:	4003      	ands	r3, r0
 800082c:	2b04      	cmp	r3, #4
 800082e:	d000      	beq.n	8000832 <__aeabi_fadd+0x76>
 8000830:	3004      	adds	r0, #4
 8000832:	0143      	lsls	r3, r0, #5
 8000834:	d400      	bmi.n	8000838 <__aeabi_fadd+0x7c>
 8000836:	e078      	b.n	800092a <__aeabi_fadd+0x16e>
 8000838:	1c6a      	adds	r2, r5, #1
 800083a:	2dfe      	cmp	r5, #254	; 0xfe
 800083c:	d065      	beq.n	800090a <__aeabi_fadd+0x14e>
 800083e:	0180      	lsls	r0, r0, #6
 8000840:	0a43      	lsrs	r3, r0, #9
 8000842:	469c      	mov	ip, r3
 8000844:	b2d2      	uxtb	r2, r2
 8000846:	4663      	mov	r3, ip
 8000848:	05d0      	lsls	r0, r2, #23
 800084a:	4318      	orrs	r0, r3
 800084c:	07e4      	lsls	r4, r4, #31
 800084e:	4320      	orrs	r0, r4
 8000850:	bc80      	pop	{r7}
 8000852:	46b8      	mov	r8, r7
 8000854:	bdf0      	pop	{r4, r5, r6, r7, pc}
 8000856:	2a00      	cmp	r2, #0
 8000858:	d035      	beq.n	80008c6 <__aeabi_fadd+0x10a>
 800085a:	1b7a      	subs	r2, r7, r5
 800085c:	2d00      	cmp	r5, #0
 800085e:	d000      	beq.n	8000862 <__aeabi_fadd+0xa6>
 8000860:	e0af      	b.n	80009c2 <__aeabi_fadd+0x206>
 8000862:	4643      	mov	r3, r8
 8000864:	2b00      	cmp	r3, #0
 8000866:	d100      	bne.n	800086a <__aeabi_fadd+0xae>
 8000868:	e0a7      	b.n	80009ba <__aeabi_fadd+0x1fe>
 800086a:	1e53      	subs	r3, r2, #1
 800086c:	2a01      	cmp	r2, #1
 800086e:	d100      	bne.n	8000872 <__aeabi_fadd+0xb6>
 8000870:	e12f      	b.n	8000ad2 <__aeabi_fadd+0x316>
 8000872:	2aff      	cmp	r2, #255	; 0xff
 8000874:	d069      	beq.n	800094a <__aeabi_fadd+0x18e>
 8000876:	001a      	movs	r2, r3
 8000878:	e0aa      	b.n	80009d0 <__aeabi_fadd+0x214>
 800087a:	1be9      	subs	r1, r5, r7
 800087c:	2900      	cmp	r1, #0
 800087e:	dd70      	ble.n	8000962 <__aeabi_fadd+0x1a6>
 8000880:	2f00      	cmp	r7, #0
 8000882:	d037      	beq.n	80008f4 <__aeabi_fadd+0x138>
 8000884:	2dff      	cmp	r5, #255	; 0xff
 8000886:	d062      	beq.n	800094e <__aeabi_fadd+0x192>
 8000888:	2380      	movs	r3, #128	; 0x80
 800088a:	04db      	lsls	r3, r3, #19
 800088c:	431e      	orrs	r6, r3
 800088e:	291b      	cmp	r1, #27
 8000890:	dc00      	bgt.n	8000894 <__aeabi_fadd+0xd8>
 8000892:	e0b0      	b.n	80009f6 <__aeabi_fadd+0x23a>
 8000894:	2001      	movs	r0, #1
 8000896:	4440      	add	r0, r8
 8000898:	0143      	lsls	r3, r0, #5
 800089a:	d543      	bpl.n	8000924 <__aeabi_fadd+0x168>
 800089c:	3501      	adds	r5, #1
 800089e:	2dff      	cmp	r5, #255	; 0xff
 80008a0:	d033      	beq.n	800090a <__aeabi_fadd+0x14e>
 80008a2:	2301      	movs	r3, #1
 80008a4:	4a93      	ldr	r2, [pc, #588]	; (8000af4 <__aeabi_fadd+0x338>)
 80008a6:	4003      	ands	r3, r0
 80008a8:	0840      	lsrs	r0, r0, #1
 80008aa:	4010      	ands	r0, r2
 80008ac:	4318      	orrs	r0, r3
 80008ae:	e7b9      	b.n	8000824 <__aeabi_fadd+0x68>
 80008b0:	2e00      	cmp	r6, #0
 80008b2:	d100      	bne.n	80008b6 <__aeabi_fadd+0xfa>
 80008b4:	e083      	b.n	80009be <__aeabi_fadd+0x202>
 80008b6:	1e51      	subs	r1, r2, #1
 80008b8:	2a01      	cmp	r2, #1
 80008ba:	d100      	bne.n	80008be <__aeabi_fadd+0x102>
 80008bc:	e0d8      	b.n	8000a70 <__aeabi_fadd+0x2b4>
 80008be:	2aff      	cmp	r2, #255	; 0xff
 80008c0:	d045      	beq.n	800094e <__aeabi_fadd+0x192>
 80008c2:	000a      	movs	r2, r1
 80008c4:	e798      	b.n	80007f8 <__aeabi_fadd+0x3c>
 80008c6:	27fe      	movs	r7, #254	; 0xfe
 80008c8:	1c6a      	adds	r2, r5, #1
 80008ca:	4217      	tst	r7, r2
 80008cc:	d000      	beq.n	80008d0 <__aeabi_fadd+0x114>
 80008ce:	e086      	b.n	80009de <__aeabi_fadd+0x222>
 80008d0:	2d00      	cmp	r5, #0
 80008d2:	d000      	beq.n	80008d6 <__aeabi_fadd+0x11a>
 80008d4:	e0b7      	b.n	8000a46 <__aeabi_fadd+0x28a>
 80008d6:	4643      	mov	r3, r8
 80008d8:	2b00      	cmp	r3, #0
 80008da:	d100      	bne.n	80008de <__aeabi_fadd+0x122>
 80008dc:	e0f3      	b.n	8000ac6 <__aeabi_fadd+0x30a>
 80008de:	2200      	movs	r2, #0
 80008e0:	2e00      	cmp	r6, #0
 80008e2:	d0b0      	beq.n	8000846 <__aeabi_fadd+0x8a>
 80008e4:	1b98      	subs	r0, r3, r6
 80008e6:	0143      	lsls	r3, r0, #5
 80008e8:	d400      	bmi.n	80008ec <__aeabi_fadd+0x130>
 80008ea:	e0fa      	b.n	8000ae2 <__aeabi_fadd+0x326>
 80008ec:	4643      	mov	r3, r8
 80008ee:	000c      	movs	r4, r1
 80008f0:	1af0      	subs	r0, r6, r3
 80008f2:	e797      	b.n	8000824 <__aeabi_fadd+0x68>
 80008f4:	2e00      	cmp	r6, #0
 80008f6:	d100      	bne.n	80008fa <__aeabi_fadd+0x13e>
 80008f8:	e0c8      	b.n	8000a8c <__aeabi_fadd+0x2d0>
 80008fa:	1e4a      	subs	r2, r1, #1
 80008fc:	2901      	cmp	r1, #1
 80008fe:	d100      	bne.n	8000902 <__aeabi_fadd+0x146>
 8000900:	e0ae      	b.n	8000a60 <__aeabi_fadd+0x2a4>
 8000902:	29ff      	cmp	r1, #255	; 0xff
 8000904:	d023      	beq.n	800094e <__aeabi_fadd+0x192>
 8000906:	0011      	movs	r1, r2
 8000908:	e7c1      	b.n	800088e <__aeabi_fadd+0xd2>
 800090a:	2300      	movs	r3, #0
 800090c:	22ff      	movs	r2, #255	; 0xff
 800090e:	469c      	mov	ip, r3
 8000910:	e799      	b.n	8000846 <__aeabi_fadd+0x8a>
 8000912:	21fe      	movs	r1, #254	; 0xfe
 8000914:	1c6a      	adds	r2, r5, #1
 8000916:	4211      	tst	r1, r2
 8000918:	d077      	beq.n	8000a0a <__aeabi_fadd+0x24e>
 800091a:	2aff      	cmp	r2, #255	; 0xff
 800091c:	d0f5      	beq.n	800090a <__aeabi_fadd+0x14e>
 800091e:	0015      	movs	r5, r2
 8000920:	4446      	add	r6, r8
 8000922:	0870      	lsrs	r0, r6, #1
 8000924:	0743      	lsls	r3, r0, #29
 8000926:	d000      	beq.n	800092a <__aeabi_fadd+0x16e>
 8000928:	e77e      	b.n	8000828 <__aeabi_fadd+0x6c>
 800092a:	08c3      	lsrs	r3, r0, #3
 800092c:	2dff      	cmp	r5, #255	; 0xff
 800092e:	d00e      	beq.n	800094e <__aeabi_fadd+0x192>
 8000930:	025b      	lsls	r3, r3, #9
 8000932:	0a5b      	lsrs	r3, r3, #9
 8000934:	469c      	mov	ip, r3
 8000936:	b2ea      	uxtb	r2, r5
 8000938:	e785      	b.n	8000846 <__aeabi_fadd+0x8a>
 800093a:	2e00      	cmp	r6, #0
 800093c:	d007      	beq.n	800094e <__aeabi_fadd+0x192>
 800093e:	2280      	movs	r2, #128	; 0x80
 8000940:	03d2      	lsls	r2, r2, #15
 8000942:	4213      	tst	r3, r2
 8000944:	d003      	beq.n	800094e <__aeabi_fadd+0x192>
 8000946:	4210      	tst	r0, r2
 8000948:	d101      	bne.n	800094e <__aeabi_fadd+0x192>
 800094a:	000c      	movs	r4, r1
 800094c:	0003      	movs	r3, r0
 800094e:	2b00      	cmp	r3, #0
 8000950:	d0db      	beq.n	800090a <__aeabi_fadd+0x14e>
 8000952:	2080      	movs	r0, #128	; 0x80
 8000954:	03c0      	lsls	r0, r0, #15
 8000956:	4318      	orrs	r0, r3
 8000958:	0240      	lsls	r0, r0, #9
 800095a:	0a43      	lsrs	r3, r0, #9
 800095c:	469c      	mov	ip, r3
 800095e:	22ff      	movs	r2, #255	; 0xff
 8000960:	e771      	b.n	8000846 <__aeabi_fadd+0x8a>
 8000962:	2900      	cmp	r1, #0
 8000964:	d0d5      	beq.n	8000912 <__aeabi_fadd+0x156>
 8000966:	1b7a      	subs	r2, r7, r5
 8000968:	2d00      	cmp	r5, #0
 800096a:	d160      	bne.n	8000a2e <__aeabi_fadd+0x272>
 800096c:	4643      	mov	r3, r8
 800096e:	2b00      	cmp	r3, #0
 8000970:	d024      	beq.n	80009bc <__aeabi_fadd+0x200>
 8000972:	1e53      	subs	r3, r2, #1
 8000974:	2a01      	cmp	r2, #1
 8000976:	d073      	beq.n	8000a60 <__aeabi_fadd+0x2a4>
 8000978:	2aff      	cmp	r2, #255	; 0xff
 800097a:	d0e7      	beq.n	800094c <__aeabi_fadd+0x190>
 800097c:	001a      	movs	r2, r3
 800097e:	2a1b      	cmp	r2, #27
 8000980:	dc00      	bgt.n	8000984 <__aeabi_fadd+0x1c8>
 8000982:	e085      	b.n	8000a90 <__aeabi_fadd+0x2d4>
 8000984:	2001      	movs	r0, #1
 8000986:	003d      	movs	r5, r7
 8000988:	1980      	adds	r0, r0, r6
 800098a:	e785      	b.n	8000898 <__aeabi_fadd+0xdc>
 800098c:	2320      	movs	r3, #32
 800098e:	003a      	movs	r2, r7
 8000990:	1b45      	subs	r5, r0, r5
 8000992:	0038      	movs	r0, r7
 8000994:	3501      	adds	r5, #1
 8000996:	40ea      	lsrs	r2, r5
 8000998:	1b5d      	subs	r5, r3, r5
 800099a:	40a8      	lsls	r0, r5
 800099c:	1e43      	subs	r3, r0, #1
 800099e:	4198      	sbcs	r0, r3
 80009a0:	2500      	movs	r5, #0
 80009a2:	4310      	orrs	r0, r2
 80009a4:	e73e      	b.n	8000824 <__aeabi_fadd+0x68>
 80009a6:	2320      	movs	r3, #32
 80009a8:	0030      	movs	r0, r6
 80009aa:	1a9b      	subs	r3, r3, r2
 80009ac:	0031      	movs	r1, r6
 80009ae:	4098      	lsls	r0, r3
 80009b0:	40d1      	lsrs	r1, r2
 80009b2:	1e43      	subs	r3, r0, #1
 80009b4:	4198      	sbcs	r0, r3
 80009b6:	4308      	orrs	r0, r1
 80009b8:	e722      	b.n	8000800 <__aeabi_fadd+0x44>
 80009ba:	000c      	movs	r4, r1
 80009bc:	0003      	movs	r3, r0
 80009be:	0015      	movs	r5, r2
 80009c0:	e7b4      	b.n	800092c <__aeabi_fadd+0x170>
 80009c2:	2fff      	cmp	r7, #255	; 0xff
 80009c4:	d0c1      	beq.n	800094a <__aeabi_fadd+0x18e>
 80009c6:	2380      	movs	r3, #128	; 0x80
 80009c8:	4640      	mov	r0, r8
 80009ca:	04db      	lsls	r3, r3, #19
 80009cc:	4318      	orrs	r0, r3
 80009ce:	4680      	mov	r8, r0
 80009d0:	2a1b      	cmp	r2, #27
 80009d2:	dd51      	ble.n	8000a78 <__aeabi_fadd+0x2bc>
 80009d4:	2001      	movs	r0, #1
 80009d6:	000c      	movs	r4, r1
 80009d8:	003d      	movs	r5, r7
 80009da:	1a30      	subs	r0, r6, r0
 80009dc:	e712      	b.n	8000804 <__aeabi_fadd+0x48>
 80009de:	4643      	mov	r3, r8
 80009e0:	1b9f      	subs	r7, r3, r6
 80009e2:	017b      	lsls	r3, r7, #5
 80009e4:	d42b      	bmi.n	8000a3e <__aeabi_fadd+0x282>
 80009e6:	2f00      	cmp	r7, #0
 80009e8:	d000      	beq.n	80009ec <__aeabi_fadd+0x230>
 80009ea:	e710      	b.n	800080e <__aeabi_fadd+0x52>
 80009ec:	2300      	movs	r3, #0
 80009ee:	2400      	movs	r4, #0
 80009f0:	2200      	movs	r2, #0
 80009f2:	469c      	mov	ip, r3
 80009f4:	e727      	b.n	8000846 <__aeabi_fadd+0x8a>
 80009f6:	2320      	movs	r3, #32
 80009f8:	0032      	movs	r2, r6
 80009fa:	0030      	movs	r0, r6
 80009fc:	40ca      	lsrs	r2, r1
 80009fe:	1a59      	subs	r1, r3, r1
 8000a00:	4088      	lsls	r0, r1
 8000a02:	1e43      	subs	r3, r0, #1
 8000a04:	4198      	sbcs	r0, r3
 8000a06:	4310      	orrs	r0, r2
 8000a08:	e745      	b.n	8000896 <__aeabi_fadd+0xda>
 8000a0a:	2d00      	cmp	r5, #0
 8000a0c:	d14a      	bne.n	8000aa4 <__aeabi_fadd+0x2e8>
 8000a0e:	4643      	mov	r3, r8
 8000a10:	2b00      	cmp	r3, #0
 8000a12:	d063      	beq.n	8000adc <__aeabi_fadd+0x320>
 8000a14:	2200      	movs	r2, #0
 8000a16:	2e00      	cmp	r6, #0
 8000a18:	d100      	bne.n	8000a1c <__aeabi_fadd+0x260>
 8000a1a:	e714      	b.n	8000846 <__aeabi_fadd+0x8a>
 8000a1c:	0030      	movs	r0, r6
 8000a1e:	4440      	add	r0, r8
 8000a20:	0143      	lsls	r3, r0, #5
 8000a22:	d400      	bmi.n	8000a26 <__aeabi_fadd+0x26a>
 8000a24:	e77e      	b.n	8000924 <__aeabi_fadd+0x168>
 8000a26:	4b32      	ldr	r3, [pc, #200]	; (8000af0 <__aeabi_fadd+0x334>)
 8000a28:	3501      	adds	r5, #1
 8000a2a:	4018      	ands	r0, r3
 8000a2c:	e77a      	b.n	8000924 <__aeabi_fadd+0x168>
 8000a2e:	2fff      	cmp	r7, #255	; 0xff
 8000a30:	d08c      	beq.n	800094c <__aeabi_fadd+0x190>
 8000a32:	2380      	movs	r3, #128	; 0x80
 8000a34:	4641      	mov	r1, r8
 8000a36:	04db      	lsls	r3, r3, #19
 8000a38:	4319      	orrs	r1, r3
 8000a3a:	4688      	mov	r8, r1
 8000a3c:	e79f      	b.n	800097e <__aeabi_fadd+0x1c2>
 8000a3e:	4643      	mov	r3, r8
 8000a40:	000c      	movs	r4, r1
 8000a42:	1af7      	subs	r7, r6, r3
 8000a44:	e6e3      	b.n	800080e <__aeabi_fadd+0x52>
 8000a46:	4642      	mov	r2, r8
 8000a48:	2a00      	cmp	r2, #0
 8000a4a:	d000      	beq.n	8000a4e <__aeabi_fadd+0x292>
 8000a4c:	e775      	b.n	800093a <__aeabi_fadd+0x17e>
 8000a4e:	2e00      	cmp	r6, #0
 8000a50:	d000      	beq.n	8000a54 <__aeabi_fadd+0x298>
 8000a52:	e77a      	b.n	800094a <__aeabi_fadd+0x18e>
 8000a54:	2380      	movs	r3, #128	; 0x80
 8000a56:	03db      	lsls	r3, r3, #15
 8000a58:	2400      	movs	r4, #0
 8000a5a:	469c      	mov	ip, r3
 8000a5c:	22ff      	movs	r2, #255	; 0xff
 8000a5e:	e6f2      	b.n	8000846 <__aeabi_fadd+0x8a>
 8000a60:	0030      	movs	r0, r6
 8000a62:	4440      	add	r0, r8
 8000a64:	2501      	movs	r5, #1
 8000a66:	0143      	lsls	r3, r0, #5
 8000a68:	d400      	bmi.n	8000a6c <__aeabi_fadd+0x2b0>
 8000a6a:	e75b      	b.n	8000924 <__aeabi_fadd+0x168>
 8000a6c:	2502      	movs	r5, #2
 8000a6e:	e718      	b.n	80008a2 <__aeabi_fadd+0xe6>
 8000a70:	4643      	mov	r3, r8
 8000a72:	2501      	movs	r5, #1
 8000a74:	1b98      	subs	r0, r3, r6
 8000a76:	e6c5      	b.n	8000804 <__aeabi_fadd+0x48>
 8000a78:	2320      	movs	r3, #32
 8000a7a:	4644      	mov	r4, r8
 8000a7c:	4640      	mov	r0, r8
 8000a7e:	40d4      	lsrs	r4, r2
 8000a80:	1a9a      	subs	r2, r3, r2
 8000a82:	4090      	lsls	r0, r2
 8000a84:	1e43      	subs	r3, r0, #1
 8000a86:	4198      	sbcs	r0, r3
 8000a88:	4320      	orrs	r0, r4
 8000a8a:	e7a4      	b.n	80009d6 <__aeabi_fadd+0x21a>
 8000a8c:	000d      	movs	r5, r1
 8000a8e:	e74d      	b.n	800092c <__aeabi_fadd+0x170>
 8000a90:	2320      	movs	r3, #32
 8000a92:	4641      	mov	r1, r8
 8000a94:	4640      	mov	r0, r8
 8000a96:	40d1      	lsrs	r1, r2
 8000a98:	1a9a      	subs	r2, r3, r2
 8000a9a:	4090      	lsls	r0, r2
 8000a9c:	1e43      	subs	r3, r0, #1
 8000a9e:	4198      	sbcs	r0, r3
 8000aa0:	4308      	orrs	r0, r1
 8000aa2:	e770      	b.n	8000986 <__aeabi_fadd+0x1ca>
 8000aa4:	4642      	mov	r2, r8
 8000aa6:	2a00      	cmp	r2, #0
 8000aa8:	d100      	bne.n	8000aac <__aeabi_fadd+0x2f0>
 8000aaa:	e74f      	b.n	800094c <__aeabi_fadd+0x190>
 8000aac:	2e00      	cmp	r6, #0
 8000aae:	d100      	bne.n	8000ab2 <__aeabi_fadd+0x2f6>
 8000ab0:	e74d      	b.n	800094e <__aeabi_fadd+0x192>
 8000ab2:	2280      	movs	r2, #128	; 0x80
 8000ab4:	03d2      	lsls	r2, r2, #15
 8000ab6:	4213      	tst	r3, r2
 8000ab8:	d100      	bne.n	8000abc <__aeabi_fadd+0x300>
 8000aba:	e748      	b.n	800094e <__aeabi_fadd+0x192>
 8000abc:	4210      	tst	r0, r2
 8000abe:	d000      	beq.n	8000ac2 <__aeabi_fadd+0x306>
 8000ac0:	e745      	b.n	800094e <__aeabi_fadd+0x192>
 8000ac2:	0003      	movs	r3, r0
 8000ac4:	e743      	b.n	800094e <__aeabi_fadd+0x192>
 8000ac6:	2e00      	cmp	r6, #0
 8000ac8:	d090      	beq.n	80009ec <__aeabi_fadd+0x230>
 8000aca:	000c      	movs	r4, r1
 8000acc:	4684      	mov	ip, r0
 8000ace:	2200      	movs	r2, #0
 8000ad0:	e6b9      	b.n	8000846 <__aeabi_fadd+0x8a>
 8000ad2:	4643      	mov	r3, r8
 8000ad4:	000c      	movs	r4, r1
 8000ad6:	1af0      	subs	r0, r6, r3
 8000ad8:	3501      	adds	r5, #1
 8000ada:	e693      	b.n	8000804 <__aeabi_fadd+0x48>
 8000adc:	4684      	mov	ip, r0
 8000ade:	2200      	movs	r2, #0
 8000ae0:	e6b1      	b.n	8000846 <__aeabi_fadd+0x8a>
 8000ae2:	2800      	cmp	r0, #0
 8000ae4:	d000      	beq.n	8000ae8 <__aeabi_fadd+0x32c>
 8000ae6:	e71d      	b.n	8000924 <__aeabi_fadd+0x168>
 8000ae8:	2300      	movs	r3, #0
 8000aea:	2400      	movs	r4, #0
 8000aec:	469c      	mov	ip, r3
 8000aee:	e6aa      	b.n	8000846 <__aeabi_fadd+0x8a>
 8000af0:	fbffffff 	.word	0xfbffffff
 8000af4:	7dffffff 	.word	0x7dffffff

08000af8 <__aeabi_ui2f>:
 8000af8:	b570      	push	{r4, r5, r6, lr}
 8000afa:	1e05      	subs	r5, r0, #0
 8000afc:	d00e      	beq.n	8000b1c <__aeabi_ui2f+0x24>
 8000afe:	f001 fef3 	bl	80028e8 <__clzsi2>
 8000b02:	239e      	movs	r3, #158	; 0x9e
 8000b04:	0004      	movs	r4, r0
 8000b06:	1a1b      	subs	r3, r3, r0
 8000b08:	2b96      	cmp	r3, #150	; 0x96
 8000b0a:	dc0c      	bgt.n	8000b26 <__aeabi_ui2f+0x2e>
 8000b0c:	2808      	cmp	r0, #8
 8000b0e:	dd01      	ble.n	8000b14 <__aeabi_ui2f+0x1c>
 8000b10:	3c08      	subs	r4, #8
 8000b12:	40a5      	lsls	r5, r4
 8000b14:	026d      	lsls	r5, r5, #9
 8000b16:	0a6d      	lsrs	r5, r5, #9
 8000b18:	b2d8      	uxtb	r0, r3
 8000b1a:	e001      	b.n	8000b20 <__aeabi_ui2f+0x28>
 8000b1c:	2000      	movs	r0, #0
 8000b1e:	2500      	movs	r5, #0
 8000b20:	05c0      	lsls	r0, r0, #23
 8000b22:	4328      	orrs	r0, r5
 8000b24:	bd70      	pop	{r4, r5, r6, pc}
 8000b26:	2b99      	cmp	r3, #153	; 0x99
 8000b28:	dd09      	ble.n	8000b3e <__aeabi_ui2f+0x46>
 8000b2a:	0002      	movs	r2, r0
 8000b2c:	0029      	movs	r1, r5
 8000b2e:	321b      	adds	r2, #27
 8000b30:	4091      	lsls	r1, r2
 8000b32:	1e4a      	subs	r2, r1, #1
 8000b34:	4191      	sbcs	r1, r2
 8000b36:	2205      	movs	r2, #5
 8000b38:	1a12      	subs	r2, r2, r0
 8000b3a:	40d5      	lsrs	r5, r2
 8000b3c:	430d      	orrs	r5, r1
 8000b3e:	2c05      	cmp	r4, #5
 8000b40:	dc12      	bgt.n	8000b68 <__aeabi_ui2f+0x70>
 8000b42:	0029      	movs	r1, r5
 8000b44:	4e0c      	ldr	r6, [pc, #48]	; (8000b78 <__aeabi_ui2f+0x80>)
 8000b46:	4031      	ands	r1, r6
 8000b48:	076a      	lsls	r2, r5, #29
 8000b4a:	d009      	beq.n	8000b60 <__aeabi_ui2f+0x68>
 8000b4c:	200f      	movs	r0, #15
 8000b4e:	4028      	ands	r0, r5
 8000b50:	2804      	cmp	r0, #4
 8000b52:	d005      	beq.n	8000b60 <__aeabi_ui2f+0x68>
 8000b54:	3104      	adds	r1, #4
 8000b56:	014a      	lsls	r2, r1, #5
 8000b58:	d502      	bpl.n	8000b60 <__aeabi_ui2f+0x68>
 8000b5a:	239f      	movs	r3, #159	; 0x9f
 8000b5c:	4031      	ands	r1, r6
 8000b5e:	1b1b      	subs	r3, r3, r4
 8000b60:	0189      	lsls	r1, r1, #6
 8000b62:	0a4d      	lsrs	r5, r1, #9
 8000b64:	b2d8      	uxtb	r0, r3
 8000b66:	e7db      	b.n	8000b20 <__aeabi_ui2f+0x28>
 8000b68:	1f62      	subs	r2, r4, #5
 8000b6a:	4095      	lsls	r5, r2
 8000b6c:	0029      	movs	r1, r5
 8000b6e:	4e02      	ldr	r6, [pc, #8]	; (8000b78 <__aeabi_ui2f+0x80>)
 8000b70:	4031      	ands	r1, r6
 8000b72:	076a      	lsls	r2, r5, #29
 8000b74:	d0f4      	beq.n	8000b60 <__aeabi_ui2f+0x68>
 8000b76:	e7e9      	b.n	8000b4c <__aeabi_ui2f+0x54>
 8000b78:	fbffffff 	.word	0xfbffffff

08000b7c <__aeabi_dadd>:
 8000b7c:	b5f0      	push	{r4, r5, r6, r7, lr}
 8000b7e:	464f      	mov	r7, r9
 8000b80:	4646      	mov	r6, r8
 8000b82:	46d6      	mov	lr, sl
 8000b84:	000d      	movs	r5, r1
 8000b86:	0004      	movs	r4, r0
 8000b88:	b5c0      	push	{r6, r7, lr}
 8000b8a:	001f      	movs	r7, r3
 8000b8c:	0011      	movs	r1, r2
 8000b8e:	0328      	lsls	r0, r5, #12
 8000b90:	0f62      	lsrs	r2, r4, #29
 8000b92:	0a40      	lsrs	r0, r0, #9
 8000b94:	4310      	orrs	r0, r2
 8000b96:	007a      	lsls	r2, r7, #1
 8000b98:	0d52      	lsrs	r2, r2, #21
 8000b9a:	00e3      	lsls	r3, r4, #3
 8000b9c:	033c      	lsls	r4, r7, #12
 8000b9e:	4691      	mov	r9, r2
 8000ba0:	0a64      	lsrs	r4, r4, #9
 8000ba2:	0ffa      	lsrs	r2, r7, #31
 8000ba4:	0f4f      	lsrs	r7, r1, #29
 8000ba6:	006e      	lsls	r6, r5, #1
 8000ba8:	4327      	orrs	r7, r4
 8000baa:	4692      	mov	sl, r2
 8000bac:	46b8      	mov	r8, r7
 8000bae:	0d76      	lsrs	r6, r6, #21
 8000bb0:	0fed      	lsrs	r5, r5, #31
 8000bb2:	00c9      	lsls	r1, r1, #3
 8000bb4:	4295      	cmp	r5, r2
 8000bb6:	d100      	bne.n	8000bba <__aeabi_dadd+0x3e>
 8000bb8:	e099      	b.n	8000cee <__aeabi_dadd+0x172>
 8000bba:	464c      	mov	r4, r9
 8000bbc:	1b34      	subs	r4, r6, r4
 8000bbe:	46a4      	mov	ip, r4
 8000bc0:	2c00      	cmp	r4, #0
 8000bc2:	dc00      	bgt.n	8000bc6 <__aeabi_dadd+0x4a>
 8000bc4:	e07c      	b.n	8000cc0 <__aeabi_dadd+0x144>
 8000bc6:	464a      	mov	r2, r9
 8000bc8:	2a00      	cmp	r2, #0
 8000bca:	d100      	bne.n	8000bce <__aeabi_dadd+0x52>
 8000bcc:	e0b8      	b.n	8000d40 <__aeabi_dadd+0x1c4>
 8000bce:	4ac5      	ldr	r2, [pc, #788]	; (8000ee4 <__aeabi_dadd+0x368>)
 8000bd0:	4296      	cmp	r6, r2
 8000bd2:	d100      	bne.n	8000bd6 <__aeabi_dadd+0x5a>
 8000bd4:	e11c      	b.n	8000e10 <__aeabi_dadd+0x294>
 8000bd6:	2280      	movs	r2, #128	; 0x80
 8000bd8:	003c      	movs	r4, r7
 8000bda:	0412      	lsls	r2, r2, #16
 8000bdc:	4314      	orrs	r4, r2
 8000bde:	46a0      	mov	r8, r4
 8000be0:	4662      	mov	r2, ip
 8000be2:	2a38      	cmp	r2, #56	; 0x38
 8000be4:	dd00      	ble.n	8000be8 <__aeabi_dadd+0x6c>
 8000be6:	e161      	b.n	8000eac <__aeabi_dadd+0x330>
 8000be8:	2a1f      	cmp	r2, #31
 8000bea:	dd00      	ble.n	8000bee <__aeabi_dadd+0x72>
 8000bec:	e1cc      	b.n	8000f88 <__aeabi_dadd+0x40c>
 8000bee:	4664      	mov	r4, ip
 8000bf0:	2220      	movs	r2, #32
 8000bf2:	1b12      	subs	r2, r2, r4
 8000bf4:	4644      	mov	r4, r8
 8000bf6:	4094      	lsls	r4, r2
 8000bf8:	000f      	movs	r7, r1
 8000bfa:	46a1      	mov	r9, r4
 8000bfc:	4664      	mov	r4, ip
 8000bfe:	4091      	lsls	r1, r2
 8000c00:	40e7      	lsrs	r7, r4
 8000c02:	464c      	mov	r4, r9
 8000c04:	1e4a      	subs	r2, r1, #1
 8000c06:	4191      	sbcs	r1, r2
 8000c08:	433c      	orrs	r4, r7
 8000c0a:	4642      	mov	r2, r8
 8000c0c:	4321      	orrs	r1, r4
 8000c0e:	4664      	mov	r4, ip
 8000c10:	40e2      	lsrs	r2, r4
 8000c12:	1a80      	subs	r0, r0, r2
 8000c14:	1a5c      	subs	r4, r3, r1
 8000c16:	42a3      	cmp	r3, r4
 8000c18:	419b      	sbcs	r3, r3
 8000c1a:	425f      	negs	r7, r3
 8000c1c:	1bc7      	subs	r7, r0, r7
 8000c1e:	023b      	lsls	r3, r7, #8
 8000c20:	d400      	bmi.n	8000c24 <__aeabi_dadd+0xa8>
 8000c22:	e0d0      	b.n	8000dc6 <__aeabi_dadd+0x24a>
 8000c24:	027f      	lsls	r7, r7, #9
 8000c26:	0a7f      	lsrs	r7, r7, #9
 8000c28:	2f00      	cmp	r7, #0
 8000c2a:	d100      	bne.n	8000c2e <__aeabi_dadd+0xb2>
 8000c2c:	e0ff      	b.n	8000e2e <__aeabi_dadd+0x2b2>
 8000c2e:	0038      	movs	r0, r7
 8000c30:	f001 fe5a 	bl	80028e8 <__clzsi2>
 8000c34:	0001      	movs	r1, r0
 8000c36:	3908      	subs	r1, #8
 8000c38:	2320      	movs	r3, #32
 8000c3a:	0022      	movs	r2, r4
 8000c3c:	1a5b      	subs	r3, r3, r1
 8000c3e:	408f      	lsls	r7, r1
 8000c40:	40da      	lsrs	r2, r3
 8000c42:	408c      	lsls	r4, r1
 8000c44:	4317      	orrs	r7, r2
 8000c46:	42b1      	cmp	r1, r6
 8000c48:	da00      	bge.n	8000c4c <__aeabi_dadd+0xd0>
 8000c4a:	e0ff      	b.n	8000e4c <__aeabi_dadd+0x2d0>
 8000c4c:	1b89      	subs	r1, r1, r6
 8000c4e:	1c4b      	adds	r3, r1, #1
 8000c50:	2b1f      	cmp	r3, #31
 8000c52:	dd00      	ble.n	8000c56 <__aeabi_dadd+0xda>
 8000c54:	e0a8      	b.n	8000da8 <__aeabi_dadd+0x22c>
 8000c56:	2220      	movs	r2, #32
 8000c58:	0039      	movs	r1, r7
 8000c5a:	1ad2      	subs	r2, r2, r3
 8000c5c:	0020      	movs	r0, r4
 8000c5e:	4094      	lsls	r4, r2
 8000c60:	4091      	lsls	r1, r2
 8000c62:	40d8      	lsrs	r0, r3
 8000c64:	1e62      	subs	r2, r4, #1
 8000c66:	4194      	sbcs	r4, r2
 8000c68:	40df      	lsrs	r7, r3
 8000c6a:	2600      	movs	r6, #0
 8000c6c:	4301      	orrs	r1, r0
 8000c6e:	430c      	orrs	r4, r1
 8000c70:	0763      	lsls	r3, r4, #29
 8000c72:	d009      	beq.n	8000c88 <__aeabi_dadd+0x10c>
 8000c74:	230f      	movs	r3, #15
 8000c76:	4023      	ands	r3, r4
 8000c78:	2b04      	cmp	r3, #4
 8000c7a:	d005      	beq.n	8000c88 <__aeabi_dadd+0x10c>
 8000c7c:	1d23      	adds	r3, r4, #4
 8000c7e:	42a3      	cmp	r3, r4
 8000c80:	41a4      	sbcs	r4, r4
 8000c82:	4264      	negs	r4, r4
 8000c84:	193f      	adds	r7, r7, r4
 8000c86:	001c      	movs	r4, r3
 8000c88:	023b      	lsls	r3, r7, #8
 8000c8a:	d400      	bmi.n	8000c8e <__aeabi_dadd+0x112>
 8000c8c:	e09e      	b.n	8000dcc <__aeabi_dadd+0x250>
 8000c8e:	4b95      	ldr	r3, [pc, #596]	; (8000ee4 <__aeabi_dadd+0x368>)
 8000c90:	3601      	adds	r6, #1
 8000c92:	429e      	cmp	r6, r3
 8000c94:	d100      	bne.n	8000c98 <__aeabi_dadd+0x11c>
 8000c96:	e0b7      	b.n	8000e08 <__aeabi_dadd+0x28c>
 8000c98:	4a93      	ldr	r2, [pc, #588]	; (8000ee8 <__aeabi_dadd+0x36c>)
 8000c9a:	08e4      	lsrs	r4, r4, #3
 8000c9c:	4017      	ands	r7, r2
 8000c9e:	077b      	lsls	r3, r7, #29
 8000ca0:	0571      	lsls	r1, r6, #21
 8000ca2:	027f      	lsls	r7, r7, #9
 8000ca4:	4323      	orrs	r3, r4
 8000ca6:	0b3f      	lsrs	r7, r7, #12
 8000ca8:	0d4a      	lsrs	r2, r1, #21
 8000caa:	0512      	lsls	r2, r2, #20
 8000cac:	433a      	orrs	r2, r7
 8000cae:	07ed      	lsls	r5, r5, #31
 8000cb0:	432a      	orrs	r2, r5
 8000cb2:	0018      	movs	r0, r3
 8000cb4:	0011      	movs	r1, r2
 8000cb6:	bce0      	pop	{r5, r6, r7}
 8000cb8:	46ba      	mov	sl, r7
 8000cba:	46b1      	mov	r9, r6
 8000cbc:	46a8      	mov	r8, r5
 8000cbe:	bdf0      	pop	{r4, r5, r6, r7, pc}
 8000cc0:	2c00      	cmp	r4, #0
 8000cc2:	d04b      	beq.n	8000d5c <__aeabi_dadd+0x1e0>
 8000cc4:	464c      	mov	r4, r9
 8000cc6:	1ba4      	subs	r4, r4, r6
 8000cc8:	46a4      	mov	ip, r4
 8000cca:	2e00      	cmp	r6, #0
 8000ccc:	d000      	beq.n	8000cd0 <__aeabi_dadd+0x154>
 8000cce:	e123      	b.n	8000f18 <__aeabi_dadd+0x39c>
 8000cd0:	0004      	movs	r4, r0
 8000cd2:	431c      	orrs	r4, r3
 8000cd4:	d100      	bne.n	8000cd8 <__aeabi_dadd+0x15c>
 8000cd6:	e1af      	b.n	8001038 <__aeabi_dadd+0x4bc>
 8000cd8:	4662      	mov	r2, ip
 8000cda:	1e54      	subs	r4, r2, #1
 8000cdc:	2a01      	cmp	r2, #1
 8000cde:	d100      	bne.n	8000ce2 <__aeabi_dadd+0x166>
 8000ce0:	e215      	b.n	800110e <__aeabi_dadd+0x592>
 8000ce2:	4d80      	ldr	r5, [pc, #512]	; (8000ee4 <__aeabi_dadd+0x368>)
 8000ce4:	45ac      	cmp	ip, r5
 8000ce6:	d100      	bne.n	8000cea <__aeabi_dadd+0x16e>
 8000ce8:	e1c8      	b.n	800107c <__aeabi_dadd+0x500>
 8000cea:	46a4      	mov	ip, r4
 8000cec:	e11b      	b.n	8000f26 <__aeabi_dadd+0x3aa>
 8000cee:	464a      	mov	r2, r9
 8000cf0:	1ab2      	subs	r2, r6, r2
 8000cf2:	4694      	mov	ip, r2
 8000cf4:	2a00      	cmp	r2, #0
 8000cf6:	dc00      	bgt.n	8000cfa <__aeabi_dadd+0x17e>
 8000cf8:	e0ac      	b.n	8000e54 <__aeabi_dadd+0x2d8>
 8000cfa:	464a      	mov	r2, r9
 8000cfc:	2a00      	cmp	r2, #0
 8000cfe:	d043      	beq.n	8000d88 <__aeabi_dadd+0x20c>
 8000d00:	4a78      	ldr	r2, [pc, #480]	; (8000ee4 <__aeabi_dadd+0x368>)
 8000d02:	4296      	cmp	r6, r2
 8000d04:	d100      	bne.n	8000d08 <__aeabi_dadd+0x18c>
 8000d06:	e1af      	b.n	8001068 <__aeabi_dadd+0x4ec>
 8000d08:	2280      	movs	r2, #128	; 0x80
 8000d0a:	003c      	movs	r4, r7
 8000d0c:	0412      	lsls	r2, r2, #16
 8000d0e:	4314      	orrs	r4, r2
 8000d10:	46a0      	mov	r8, r4
 8000d12:	4662      	mov	r2, ip
 8000d14:	2a38      	cmp	r2, #56	; 0x38
 8000d16:	dc67      	bgt.n	8000de8 <__aeabi_dadd+0x26c>
 8000d18:	2a1f      	cmp	r2, #31
 8000d1a:	dc00      	bgt.n	8000d1e <__aeabi_dadd+0x1a2>
 8000d1c:	e15f      	b.n	8000fde <__aeabi_dadd+0x462>
 8000d1e:	4647      	mov	r7, r8
 8000d20:	3a20      	subs	r2, #32
 8000d22:	40d7      	lsrs	r7, r2
 8000d24:	4662      	mov	r2, ip
 8000d26:	2a20      	cmp	r2, #32
 8000d28:	d005      	beq.n	8000d36 <__aeabi_dadd+0x1ba>
 8000d2a:	4664      	mov	r4, ip
 8000d2c:	2240      	movs	r2, #64	; 0x40
 8000d2e:	1b12      	subs	r2, r2, r4
 8000d30:	4644      	mov	r4, r8
 8000d32:	4094      	lsls	r4, r2
 8000d34:	4321      	orrs	r1, r4
 8000d36:	1e4a      	subs	r2, r1, #1
 8000d38:	4191      	sbcs	r1, r2
 8000d3a:	000c      	movs	r4, r1
 8000d3c:	433c      	orrs	r4, r7
 8000d3e:	e057      	b.n	8000df0 <__aeabi_dadd+0x274>
 8000d40:	003a      	movs	r2, r7
 8000d42:	430a      	orrs	r2, r1
 8000d44:	d100      	bne.n	8000d48 <__aeabi_dadd+0x1cc>
 8000d46:	e105      	b.n	8000f54 <__aeabi_dadd+0x3d8>
 8000d48:	0022      	movs	r2, r4
 8000d4a:	3a01      	subs	r2, #1
 8000d4c:	2c01      	cmp	r4, #1
 8000d4e:	d100      	bne.n	8000d52 <__aeabi_dadd+0x1d6>
 8000d50:	e182      	b.n	8001058 <__aeabi_dadd+0x4dc>
 8000d52:	4c64      	ldr	r4, [pc, #400]	; (8000ee4 <__aeabi_dadd+0x368>)
 8000d54:	45a4      	cmp	ip, r4
 8000d56:	d05b      	beq.n	8000e10 <__aeabi_dadd+0x294>
 8000d58:	4694      	mov	ip, r2
 8000d5a:	e741      	b.n	8000be0 <__aeabi_dadd+0x64>
 8000d5c:	4c63      	ldr	r4, [pc, #396]	; (8000eec <__aeabi_dadd+0x370>)
 8000d5e:	1c77      	adds	r7, r6, #1
 8000d60:	4227      	tst	r7, r4
 8000d62:	d000      	beq.n	8000d66 <__aeabi_dadd+0x1ea>
 8000d64:	e0c4      	b.n	8000ef0 <__aeabi_dadd+0x374>
 8000d66:	0004      	movs	r4, r0
 8000d68:	431c      	orrs	r4, r3
 8000d6a:	2e00      	cmp	r6, #0
 8000d6c:	d000      	beq.n	8000d70 <__aeabi_dadd+0x1f4>
 8000d6e:	e169      	b.n	8001044 <__aeabi_dadd+0x4c8>
 8000d70:	2c00      	cmp	r4, #0
 8000d72:	d100      	bne.n	8000d76 <__aeabi_dadd+0x1fa>
 8000d74:	e1bf      	b.n	80010f6 <__aeabi_dadd+0x57a>
 8000d76:	4644      	mov	r4, r8
 8000d78:	430c      	orrs	r4, r1
 8000d7a:	d000      	beq.n	8000d7e <__aeabi_dadd+0x202>
 8000d7c:	e1d0      	b.n	8001120 <__aeabi_dadd+0x5a4>
 8000d7e:	0742      	lsls	r2, r0, #29
 8000d80:	08db      	lsrs	r3, r3, #3
 8000d82:	4313      	orrs	r3, r2
 8000d84:	08c0      	lsrs	r0, r0, #3
 8000d86:	e029      	b.n	8000ddc <__aeabi_dadd+0x260>
 8000d88:	003a      	movs	r2, r7
 8000d8a:	430a      	orrs	r2, r1
 8000d8c:	d100      	bne.n	8000d90 <__aeabi_dadd+0x214>
 8000d8e:	e170      	b.n	8001072 <__aeabi_dadd+0x4f6>
 8000d90:	4662      	mov	r2, ip
 8000d92:	4664      	mov	r4, ip
 8000d94:	3a01      	subs	r2, #1
 8000d96:	2c01      	cmp	r4, #1
 8000d98:	d100      	bne.n	8000d9c <__aeabi_dadd+0x220>
 8000d9a:	e0e0      	b.n	8000f5e <__aeabi_dadd+0x3e2>
 8000d9c:	4c51      	ldr	r4, [pc, #324]	; (8000ee4 <__aeabi_dadd+0x368>)
 8000d9e:	45a4      	cmp	ip, r4
 8000da0:	d100      	bne.n	8000da4 <__aeabi_dadd+0x228>
 8000da2:	e161      	b.n	8001068 <__aeabi_dadd+0x4ec>
 8000da4:	4694      	mov	ip, r2
 8000da6:	e7b4      	b.n	8000d12 <__aeabi_dadd+0x196>
 8000da8:	003a      	movs	r2, r7
 8000daa:	391f      	subs	r1, #31
 8000dac:	40ca      	lsrs	r2, r1
 8000dae:	0011      	movs	r1, r2
 8000db0:	2b20      	cmp	r3, #32
 8000db2:	d003      	beq.n	8000dbc <__aeabi_dadd+0x240>
 8000db4:	2240      	movs	r2, #64	; 0x40
 8000db6:	1ad3      	subs	r3, r2, r3
 8000db8:	409f      	lsls	r7, r3
 8000dba:	433c      	orrs	r4, r7
 8000dbc:	1e63      	subs	r3, r4, #1
 8000dbe:	419c      	sbcs	r4, r3
 8000dc0:	2700      	movs	r7, #0
 8000dc2:	2600      	movs	r6, #0
 8000dc4:	430c      	orrs	r4, r1
 8000dc6:	0763      	lsls	r3, r4, #29
 8000dc8:	d000      	beq.n	8000dcc <__aeabi_dadd+0x250>
 8000dca:	e753      	b.n	8000c74 <__aeabi_dadd+0xf8>
 8000dcc:	46b4      	mov	ip, r6
 8000dce:	08e4      	lsrs	r4, r4, #3
 8000dd0:	077b      	lsls	r3, r7, #29
 8000dd2:	4323      	orrs	r3, r4
 8000dd4:	08f8      	lsrs	r0, r7, #3
 8000dd6:	4a43      	ldr	r2, [pc, #268]	; (8000ee4 <__aeabi_dadd+0x368>)
 8000dd8:	4594      	cmp	ip, r2
 8000dda:	d01d      	beq.n	8000e18 <__aeabi_dadd+0x29c>
 8000ddc:	4662      	mov	r2, ip
 8000dde:	0307      	lsls	r7, r0, #12
 8000de0:	0552      	lsls	r2, r2, #21
 8000de2:	0b3f      	lsrs	r7, r7, #12
 8000de4:	0d52      	lsrs	r2, r2, #21
 8000de6:	e760      	b.n	8000caa <__aeabi_dadd+0x12e>
 8000de8:	4644      	mov	r4, r8
 8000dea:	430c      	orrs	r4, r1
 8000dec:	1e62      	subs	r2, r4, #1
 8000dee:	4194      	sbcs	r4, r2
 8000df0:	18e4      	adds	r4, r4, r3
 8000df2:	429c      	cmp	r4, r3
 8000df4:	419b      	sbcs	r3, r3
 8000df6:	425f      	negs	r7, r3
 8000df8:	183f      	adds	r7, r7, r0
 8000dfa:	023b      	lsls	r3, r7, #8
 8000dfc:	d5e3      	bpl.n	8000dc6 <__aeabi_dadd+0x24a>
 8000dfe:	4b39      	ldr	r3, [pc, #228]	; (8000ee4 <__aeabi_dadd+0x368>)
 8000e00:	3601      	adds	r6, #1
 8000e02:	429e      	cmp	r6, r3
 8000e04:	d000      	beq.n	8000e08 <__aeabi_dadd+0x28c>
 8000e06:	e0b5      	b.n	8000f74 <__aeabi_dadd+0x3f8>
 8000e08:	0032      	movs	r2, r6
 8000e0a:	2700      	movs	r7, #0
 8000e0c:	2300      	movs	r3, #0
 8000e0e:	e74c      	b.n	8000caa <__aeabi_dadd+0x12e>
 8000e10:	0742      	lsls	r2, r0, #29
 8000e12:	08db      	lsrs	r3, r3, #3
 8000e14:	4313      	orrs	r3, r2
 8000e16:	08c0      	lsrs	r0, r0, #3
 8000e18:	001a      	movs	r2, r3
 8000e1a:	4302      	orrs	r2, r0
 8000e1c:	d100      	bne.n	8000e20 <__aeabi_dadd+0x2a4>
 8000e1e:	e1e1      	b.n	80011e4 <__aeabi_dadd+0x668>
 8000e20:	2780      	movs	r7, #128	; 0x80
 8000e22:	033f      	lsls	r7, r7, #12
 8000e24:	4307      	orrs	r7, r0
 8000e26:	033f      	lsls	r7, r7, #12
 8000e28:	4a2e      	ldr	r2, [pc, #184]	; (8000ee4 <__aeabi_dadd+0x368>)
 8000e2a:	0b3f      	lsrs	r7, r7, #12
 8000e2c:	e73d      	b.n	8000caa <__aeabi_dadd+0x12e>
 8000e2e:	0020      	movs	r0, r4
 8000e30:	f001 fd5a 	bl	80028e8 <__clzsi2>
 8000e34:	0001      	movs	r1, r0
 8000e36:	3118      	adds	r1, #24
 8000e38:	291f      	cmp	r1, #31
 8000e3a:	dc00      	bgt.n	8000e3e <__aeabi_dadd+0x2c2>
 8000e3c:	e6fc      	b.n	8000c38 <__aeabi_dadd+0xbc>
 8000e3e:	3808      	subs	r0, #8
 8000e40:	4084      	lsls	r4, r0
 8000e42:	0027      	movs	r7, r4
 8000e44:	2400      	movs	r4, #0
 8000e46:	42b1      	cmp	r1, r6
 8000e48:	db00      	blt.n	8000e4c <__aeabi_dadd+0x2d0>
 8000e4a:	e6ff      	b.n	8000c4c <__aeabi_dadd+0xd0>
 8000e4c:	4a26      	ldr	r2, [pc, #152]	; (8000ee8 <__aeabi_dadd+0x36c>)
 8000e4e:	1a76      	subs	r6, r6, r1
 8000e50:	4017      	ands	r7, r2
 8000e52:	e70d      	b.n	8000c70 <__aeabi_dadd+0xf4>
 8000e54:	2a00      	cmp	r2, #0
 8000e56:	d02f      	beq.n	8000eb8 <__aeabi_dadd+0x33c>
 8000e58:	464a      	mov	r2, r9
 8000e5a:	1b92      	subs	r2, r2, r6
 8000e5c:	4694      	mov	ip, r2
 8000e5e:	2e00      	cmp	r6, #0
 8000e60:	d100      	bne.n	8000e64 <__aeabi_dadd+0x2e8>
 8000e62:	e0ad      	b.n	8000fc0 <__aeabi_dadd+0x444>
 8000e64:	4a1f      	ldr	r2, [pc, #124]	; (8000ee4 <__aeabi_dadd+0x368>)
 8000e66:	4591      	cmp	r9, r2
 8000e68:	d100      	bne.n	8000e6c <__aeabi_dadd+0x2f0>
 8000e6a:	e10f      	b.n	800108c <__aeabi_dadd+0x510>
 8000e6c:	2280      	movs	r2, #128	; 0x80
 8000e6e:	0412      	lsls	r2, r2, #16
 8000e70:	4310      	orrs	r0, r2
 8000e72:	4662      	mov	r2, ip
 8000e74:	2a38      	cmp	r2, #56	; 0x38
 8000e76:	dd00      	ble.n	8000e7a <__aeabi_dadd+0x2fe>
 8000e78:	e10f      	b.n	800109a <__aeabi_dadd+0x51e>
 8000e7a:	2a1f      	cmp	r2, #31
 8000e7c:	dd00      	ble.n	8000e80 <__aeabi_dadd+0x304>
 8000e7e:	e180      	b.n	8001182 <__aeabi_dadd+0x606>
 8000e80:	4664      	mov	r4, ip
 8000e82:	2220      	movs	r2, #32
 8000e84:	001e      	movs	r6, r3
 8000e86:	1b12      	subs	r2, r2, r4
 8000e88:	4667      	mov	r7, ip
 8000e8a:	0004      	movs	r4, r0
 8000e8c:	4093      	lsls	r3, r2
 8000e8e:	4094      	lsls	r4, r2
 8000e90:	40fe      	lsrs	r6, r7
 8000e92:	1e5a      	subs	r2, r3, #1
 8000e94:	4193      	sbcs	r3, r2
 8000e96:	40f8      	lsrs	r0, r7
 8000e98:	4334      	orrs	r4, r6
 8000e9a:	431c      	orrs	r4, r3
 8000e9c:	4480      	add	r8, r0
 8000e9e:	1864      	adds	r4, r4, r1
 8000ea0:	428c      	cmp	r4, r1
 8000ea2:	41bf      	sbcs	r7, r7
 8000ea4:	427f      	negs	r7, r7
 8000ea6:	464e      	mov	r6, r9
 8000ea8:	4447      	add	r7, r8
 8000eaa:	e7a6      	b.n	8000dfa <__aeabi_dadd+0x27e>
 8000eac:	4642      	mov	r2, r8
 8000eae:	430a      	orrs	r2, r1
 8000eb0:	0011      	movs	r1, r2
 8000eb2:	1e4a      	subs	r2, r1, #1
 8000eb4:	4191      	sbcs	r1, r2
 8000eb6:	e6ad      	b.n	8000c14 <__aeabi_dadd+0x98>
 8000eb8:	4c0c      	ldr	r4, [pc, #48]	; (8000eec <__aeabi_dadd+0x370>)
 8000eba:	1c72      	adds	r2, r6, #1
 8000ebc:	4222      	tst	r2, r4
 8000ebe:	d000      	beq.n	8000ec2 <__aeabi_dadd+0x346>
 8000ec0:	e0a1      	b.n	8001006 <__aeabi_dadd+0x48a>
 8000ec2:	0002      	movs	r2, r0
 8000ec4:	431a      	orrs	r2, r3
 8000ec6:	2e00      	cmp	r6, #0
 8000ec8:	d000      	beq.n	8000ecc <__aeabi_dadd+0x350>
 8000eca:	e0fa      	b.n	80010c2 <__aeabi_dadd+0x546>
 8000ecc:	2a00      	cmp	r2, #0
 8000ece:	d100      	bne.n	8000ed2 <__aeabi_dadd+0x356>
 8000ed0:	e145      	b.n	800115e <__aeabi_dadd+0x5e2>
 8000ed2:	003a      	movs	r2, r7
 8000ed4:	430a      	orrs	r2, r1
 8000ed6:	d000      	beq.n	8000eda <__aeabi_dadd+0x35e>
 8000ed8:	e146      	b.n	8001168 <__aeabi_dadd+0x5ec>
 8000eda:	0742      	lsls	r2, r0, #29
 8000edc:	08db      	lsrs	r3, r3, #3
 8000ede:	4313      	orrs	r3, r2
 8000ee0:	08c0      	lsrs	r0, r0, #3
 8000ee2:	e77b      	b.n	8000ddc <__aeabi_dadd+0x260>
 8000ee4:	000007ff 	.word	0x000007ff
 8000ee8:	ff7fffff 	.word	0xff7fffff
 8000eec:	000007fe 	.word	0x000007fe
 8000ef0:	4647      	mov	r7, r8
 8000ef2:	1a5c      	subs	r4, r3, r1
 8000ef4:	1bc2      	subs	r2, r0, r7
 8000ef6:	42a3      	cmp	r3, r4
 8000ef8:	41bf      	sbcs	r7, r7
 8000efa:	427f      	negs	r7, r7
 8000efc:	46b9      	mov	r9, r7
 8000efe:	0017      	movs	r7, r2
 8000f00:	464a      	mov	r2, r9
 8000f02:	1abf      	subs	r7, r7, r2
 8000f04:	023a      	lsls	r2, r7, #8
 8000f06:	d500      	bpl.n	8000f0a <__aeabi_dadd+0x38e>
 8000f08:	e08d      	b.n	8001026 <__aeabi_dadd+0x4aa>
 8000f0a:	0023      	movs	r3, r4
 8000f0c:	433b      	orrs	r3, r7
 8000f0e:	d000      	beq.n	8000f12 <__aeabi_dadd+0x396>
 8000f10:	e68a      	b.n	8000c28 <__aeabi_dadd+0xac>
 8000f12:	2000      	movs	r0, #0
 8000f14:	2500      	movs	r5, #0
 8000f16:	e761      	b.n	8000ddc <__aeabi_dadd+0x260>
 8000f18:	4cb4      	ldr	r4, [pc, #720]	; (80011ec <__aeabi_dadd+0x670>)
 8000f1a:	45a1      	cmp	r9, r4
 8000f1c:	d100      	bne.n	8000f20 <__aeabi_dadd+0x3a4>
 8000f1e:	e0ad      	b.n	800107c <__aeabi_dadd+0x500>
 8000f20:	2480      	movs	r4, #128	; 0x80
 8000f22:	0424      	lsls	r4, r4, #16
 8000f24:	4320      	orrs	r0, r4
 8000f26:	4664      	mov	r4, ip
 8000f28:	2c38      	cmp	r4, #56	; 0x38
 8000f2a:	dc3d      	bgt.n	8000fa8 <__aeabi_dadd+0x42c>
 8000f2c:	4662      	mov	r2, ip
 8000f2e:	2c1f      	cmp	r4, #31
 8000f30:	dd00      	ble.n	8000f34 <__aeabi_dadd+0x3b8>
 8000f32:	e0b7      	b.n	80010a4 <__aeabi_dadd+0x528>
 8000f34:	2520      	movs	r5, #32
 8000f36:	001e      	movs	r6, r3
 8000f38:	1b2d      	subs	r5, r5, r4
 8000f3a:	0004      	movs	r4, r0
 8000f3c:	40ab      	lsls	r3, r5
 8000f3e:	40ac      	lsls	r4, r5
 8000f40:	40d6      	lsrs	r6, r2
 8000f42:	40d0      	lsrs	r0, r2
 8000f44:	4642      	mov	r2, r8
 8000f46:	1e5d      	subs	r5, r3, #1
 8000f48:	41ab      	sbcs	r3, r5
 8000f4a:	4334      	orrs	r4, r6
 8000f4c:	1a12      	subs	r2, r2, r0
 8000f4e:	4690      	mov	r8, r2
 8000f50:	4323      	orrs	r3, r4
 8000f52:	e02c      	b.n	8000fae <__aeabi_dadd+0x432>
 8000f54:	0742      	lsls	r2, r0, #29
 8000f56:	08db      	lsrs	r3, r3, #3
 8000f58:	4313      	orrs	r3, r2
 8000f5a:	08c0      	lsrs	r0, r0, #3
 8000f5c:	e73b      	b.n	8000dd6 <__aeabi_dadd+0x25a>
 8000f5e:	185c      	adds	r4, r3, r1
 8000f60:	429c      	cmp	r4, r3
 8000f62:	419b      	sbcs	r3, r3
 8000f64:	4440      	add	r0, r8
 8000f66:	425b      	negs	r3, r3
 8000f68:	18c7      	adds	r7, r0, r3
 8000f6a:	2601      	movs	r6, #1
 8000f6c:	023b      	lsls	r3, r7, #8
 8000f6e:	d400      	bmi.n	8000f72 <__aeabi_dadd+0x3f6>
 8000f70:	e729      	b.n	8000dc6 <__aeabi_dadd+0x24a>
 8000f72:	2602      	movs	r6, #2
 8000f74:	4a9e      	ldr	r2, [pc, #632]	; (80011f0 <__aeabi_dadd+0x674>)
 8000f76:	0863      	lsrs	r3, r4, #1
 8000f78:	4017      	ands	r7, r2
 8000f7a:	2201      	movs	r2, #1
 8000f7c:	4014      	ands	r4, r2
 8000f7e:	431c      	orrs	r4, r3
 8000f80:	07fb      	lsls	r3, r7, #31
 8000f82:	431c      	orrs	r4, r3
 8000f84:	087f      	lsrs	r7, r7, #1
 8000f86:	e673      	b.n	8000c70 <__aeabi_dadd+0xf4>
 8000f88:	4644      	mov	r4, r8
 8000f8a:	3a20      	subs	r2, #32
 8000f8c:	40d4      	lsrs	r4, r2
 8000f8e:	4662      	mov	r2, ip
 8000f90:	2a20      	cmp	r2, #32
 8000f92:	d005      	beq.n	8000fa0 <__aeabi_dadd+0x424>
 8000f94:	4667      	mov	r7, ip
 8000f96:	2240      	movs	r2, #64	; 0x40
 8000f98:	1bd2      	subs	r2, r2, r7
 8000f9a:	4647      	mov	r7, r8
 8000f9c:	4097      	lsls	r7, r2
 8000f9e:	4339      	orrs	r1, r7
 8000fa0:	1e4a      	subs	r2, r1, #1
 8000fa2:	4191      	sbcs	r1, r2
 8000fa4:	4321      	orrs	r1, r4
 8000fa6:	e635      	b.n	8000c14 <__aeabi_dadd+0x98>
 8000fa8:	4303      	orrs	r3, r0
 8000faa:	1e58      	subs	r0, r3, #1
 8000fac:	4183      	sbcs	r3, r0
 8000fae:	1acc      	subs	r4, r1, r3
 8000fb0:	42a1      	cmp	r1, r4
 8000fb2:	41bf      	sbcs	r7, r7
 8000fb4:	4643      	mov	r3, r8
 8000fb6:	427f      	negs	r7, r7
 8000fb8:	4655      	mov	r5, sl
 8000fba:	464e      	mov	r6, r9
 8000fbc:	1bdf      	subs	r7, r3, r7
 8000fbe:	e62e      	b.n	8000c1e <__aeabi_dadd+0xa2>
 8000fc0:	0002      	movs	r2, r0
 8000fc2:	431a      	orrs	r2, r3
 8000fc4:	d100      	bne.n	8000fc8 <__aeabi_dadd+0x44c>
 8000fc6:	e0bd      	b.n	8001144 <__aeabi_dadd+0x5c8>
 8000fc8:	4662      	mov	r2, ip
 8000fca:	4664      	mov	r4, ip
 8000fcc:	3a01      	subs	r2, #1
 8000fce:	2c01      	cmp	r4, #1
 8000fd0:	d100      	bne.n	8000fd4 <__aeabi_dadd+0x458>
 8000fd2:	e0e5      	b.n	80011a0 <__aeabi_dadd+0x624>
 8000fd4:	4c85      	ldr	r4, [pc, #532]	; (80011ec <__aeabi_dadd+0x670>)
 8000fd6:	45a4      	cmp	ip, r4
 8000fd8:	d058      	beq.n	800108c <__aeabi_dadd+0x510>
 8000fda:	4694      	mov	ip, r2
 8000fdc:	e749      	b.n	8000e72 <__aeabi_dadd+0x2f6>
 8000fde:	4664      	mov	r4, ip
 8000fe0:	2220      	movs	r2, #32
 8000fe2:	1b12      	subs	r2, r2, r4
 8000fe4:	4644      	mov	r4, r8
 8000fe6:	4094      	lsls	r4, r2
 8000fe8:	000f      	movs	r7, r1
 8000fea:	46a1      	mov	r9, r4
 8000fec:	4664      	mov	r4, ip
 8000fee:	4091      	lsls	r1, r2
 8000ff0:	40e7      	lsrs	r7, r4
 8000ff2:	464c      	mov	r4, r9
 8000ff4:	1e4a      	subs	r2, r1, #1
 8000ff6:	4191      	sbcs	r1, r2
 8000ff8:	433c      	orrs	r4, r7
 8000ffa:	4642      	mov	r2, r8
 8000ffc:	430c      	orrs	r4, r1
 8000ffe:	4661      	mov	r1, ip
 8001000:	40ca      	lsrs	r2, r1
 8001002:	1880      	adds	r0, r0, r2
 8001004:	e6f4      	b.n	8000df0 <__aeabi_dadd+0x274>
 8001006:	4c79      	ldr	r4, [pc, #484]	; (80011ec <__aeabi_dadd+0x670>)
 8001008:	42a2      	cmp	r2, r4
 800100a:	d100      	bne.n	800100e <__aeabi_dadd+0x492>
 800100c:	e6fd      	b.n	8000e0a <__aeabi_dadd+0x28e>
 800100e:	1859      	adds	r1, r3, r1
 8001010:	4299      	cmp	r1, r3
 8001012:	419b      	sbcs	r3, r3
 8001014:	4440      	add	r0, r8
 8001016:	425f      	negs	r7, r3
 8001018:	19c7      	adds	r7, r0, r7
 800101a:	07fc      	lsls	r4, r7, #31
 800101c:	0849      	lsrs	r1, r1, #1
 800101e:	0016      	movs	r6, r2
 8001020:	430c      	orrs	r4, r1
 8001022:	087f      	lsrs	r7, r7, #1
 8001024:	e6cf      	b.n	8000dc6 <__aeabi_dadd+0x24a>
 8001026:	1acc      	subs	r4, r1, r3
 8001028:	42a1      	cmp	r1, r4
 800102a:	41bf      	sbcs	r7, r7
 800102c:	4643      	mov	r3, r8
 800102e:	427f      	negs	r7, r7
 8001030:	1a18      	subs	r0, r3, r0
 8001032:	4655      	mov	r5, sl
 8001034:	1bc7      	subs	r7, r0, r7
 8001036:	e5f7      	b.n	8000c28 <__aeabi_dadd+0xac>
 8001038:	08c9      	lsrs	r1, r1, #3
 800103a:	077b      	lsls	r3, r7, #29
 800103c:	4655      	mov	r5, sl
 800103e:	430b      	orrs	r3, r1
 8001040:	08f8      	lsrs	r0, r7, #3
 8001042:	e6c8      	b.n	8000dd6 <__aeabi_dadd+0x25a>
 8001044:	2c00      	cmp	r4, #0
 8001046:	d000      	beq.n	800104a <__aeabi_dadd+0x4ce>
 8001048:	e081      	b.n	800114e <__aeabi_dadd+0x5d2>
 800104a:	4643      	mov	r3, r8
 800104c:	430b      	orrs	r3, r1
 800104e:	d115      	bne.n	800107c <__aeabi_dadd+0x500>
 8001050:	2080      	movs	r0, #128	; 0x80
 8001052:	2500      	movs	r5, #0
 8001054:	0300      	lsls	r0, r0, #12
 8001056:	e6e3      	b.n	8000e20 <__aeabi_dadd+0x2a4>
 8001058:	1a5c      	subs	r4, r3, r1
 800105a:	42a3      	cmp	r3, r4
 800105c:	419b      	sbcs	r3, r3
 800105e:	1bc7      	subs	r7, r0, r7
 8001060:	425b      	negs	r3, r3
 8001062:	2601      	movs	r6, #1
 8001064:	1aff      	subs	r7, r7, r3
 8001066:	e5da      	b.n	8000c1e <__aeabi_dadd+0xa2>
 8001068:	0742      	lsls	r2, r0, #29
 800106a:	08db      	lsrs	r3, r3, #3
 800106c:	4313      	orrs	r3, r2
 800106e:	08c0      	lsrs	r0, r0, #3
 8001070:	e6d2      	b.n	8000e18 <__aeabi_dadd+0x29c>
 8001072:	0742      	lsls	r2, r0, #29
 8001074:	08db      	lsrs	r3, r3, #3
 8001076:	4313      	orrs	r3, r2
 8001078:	08c0      	lsrs	r0, r0, #3
 800107a:	e6ac      	b.n	8000dd6 <__aeabi_dadd+0x25a>
 800107c:	4643      	mov	r3, r8
 800107e:	4642      	mov	r2, r8
 8001080:	08c9      	lsrs	r1, r1, #3
 8001082:	075b      	lsls	r3, r3, #29
 8001084:	4655      	mov	r5, sl
 8001086:	430b      	orrs	r3, r1
 8001088:	08d0      	lsrs	r0, r2, #3
 800108a:	e6c5      	b.n	8000e18 <__aeabi_dadd+0x29c>
 800108c:	4643      	mov	r3, r8
 800108e:	4642      	mov	r2, r8
 8001090:	075b      	lsls	r3, r3, #29
 8001092:	08c9      	lsrs	r1, r1, #3
 8001094:	430b      	orrs	r3, r1
 8001096:	08d0      	lsrs	r0, r2, #3
 8001098:	e6be      	b.n	8000e18 <__aeabi_dadd+0x29c>
 800109a:	4303      	orrs	r3, r0
 800109c:	001c      	movs	r4, r3
 800109e:	1e63      	subs	r3, r4, #1
 80010a0:	419c      	sbcs	r4, r3
 80010a2:	e6fc      	b.n	8000e9e <__aeabi_dadd+0x322>
 80010a4:	0002      	movs	r2, r0
 80010a6:	3c20      	subs	r4, #32
 80010a8:	40e2      	lsrs	r2, r4
 80010aa:	0014      	movs	r4, r2
 80010ac:	4662      	mov	r2, ip
 80010ae:	2a20      	cmp	r2, #32
 80010b0:	d003      	beq.n	80010ba <__aeabi_dadd+0x53e>
 80010b2:	2540      	movs	r5, #64	; 0x40
 80010b4:	1aad      	subs	r5, r5, r2
 80010b6:	40a8      	lsls	r0, r5
 80010b8:	4303      	orrs	r3, r0
 80010ba:	1e58      	subs	r0, r3, #1
 80010bc:	4183      	sbcs	r3, r0
 80010be:	4323      	orrs	r3, r4
 80010c0:	e775      	b.n	8000fae <__aeabi_dadd+0x432>
 80010c2:	2a00      	cmp	r2, #0
 80010c4:	d0e2      	beq.n	800108c <__aeabi_dadd+0x510>
 80010c6:	003a      	movs	r2, r7
 80010c8:	430a      	orrs	r2, r1
 80010ca:	d0cd      	beq.n	8001068 <__aeabi_dadd+0x4ec>
 80010cc:	0742      	lsls	r2, r0, #29
 80010ce:	08db      	lsrs	r3, r3, #3
 80010d0:	4313      	orrs	r3, r2
 80010d2:	2280      	movs	r2, #128	; 0x80
 80010d4:	08c0      	lsrs	r0, r0, #3
 80010d6:	0312      	lsls	r2, r2, #12
 80010d8:	4210      	tst	r0, r2
 80010da:	d006      	beq.n	80010ea <__aeabi_dadd+0x56e>
 80010dc:	08fc      	lsrs	r4, r7, #3
 80010de:	4214      	tst	r4, r2
 80010e0:	d103      	bne.n	80010ea <__aeabi_dadd+0x56e>
 80010e2:	0020      	movs	r0, r4
 80010e4:	08cb      	lsrs	r3, r1, #3
 80010e6:	077a      	lsls	r2, r7, #29
 80010e8:	4313      	orrs	r3, r2
 80010ea:	0f5a      	lsrs	r2, r3, #29
 80010ec:	00db      	lsls	r3, r3, #3
 80010ee:	0752      	lsls	r2, r2, #29
 80010f0:	08db      	lsrs	r3, r3, #3
 80010f2:	4313      	orrs	r3, r2
 80010f4:	e690      	b.n	8000e18 <__aeabi_dadd+0x29c>
 80010f6:	4643      	mov	r3, r8
 80010f8:	430b      	orrs	r3, r1
 80010fa:	d100      	bne.n	80010fe <__aeabi_dadd+0x582>
 80010fc:	e709      	b.n	8000f12 <__aeabi_dadd+0x396>
 80010fe:	4643      	mov	r3, r8
 8001100:	4642      	mov	r2, r8
 8001102:	08c9      	lsrs	r1, r1, #3
 8001104:	075b      	lsls	r3, r3, #29
 8001106:	4655      	mov	r5, sl
 8001108:	430b      	orrs	r3, r1
 800110a:	08d0      	lsrs	r0, r2, #3
 800110c:	e666      	b.n	8000ddc <__aeabi_dadd+0x260>
 800110e:	1acc      	subs	r4, r1, r3
 8001110:	42a1      	cmp	r1, r4
 8001112:	4189      	sbcs	r1, r1
 8001114:	1a3f      	subs	r7, r7, r0
 8001116:	4249      	negs	r1, r1
 8001118:	4655      	mov	r5, sl
 800111a:	2601      	movs	r6, #1
 800111c:	1a7f      	subs	r7, r7, r1
 800111e:	e57e      	b.n	8000c1e <__aeabi_dadd+0xa2>
 8001120:	4642      	mov	r2, r8
 8001122:	1a5c      	subs	r4, r3, r1
 8001124:	1a87      	subs	r7, r0, r2
 8001126:	42a3      	cmp	r3, r4
 8001128:	4192      	sbcs	r2, r2
 800112a:	4252      	negs	r2, r2
 800112c:	1abf      	subs	r7, r7, r2
 800112e:	023a      	lsls	r2, r7, #8
 8001130:	d53d      	bpl.n	80011ae <__aeabi_dadd+0x632>
 8001132:	1acc      	subs	r4, r1, r3
 8001134:	42a1      	cmp	r1, r4
 8001136:	4189      	sbcs	r1, r1
 8001138:	4643      	mov	r3, r8
 800113a:	4249      	negs	r1, r1
 800113c:	1a1f      	subs	r7, r3, r0
 800113e:	4655      	mov	r5, sl
 8001140:	1a7f      	subs	r7, r7, r1
 8001142:	e595      	b.n	8000c70 <__aeabi_dadd+0xf4>
 8001144:	077b      	lsls	r3, r7, #29
 8001146:	08c9      	lsrs	r1, r1, #3
 8001148:	430b      	orrs	r3, r1
 800114a:	08f8      	lsrs	r0, r7, #3
 800114c:	e643      	b.n	8000dd6 <__aeabi_dadd+0x25a>
 800114e:	4644      	mov	r4, r8
 8001150:	08db      	lsrs	r3, r3, #3
 8001152:	430c      	orrs	r4, r1
 8001154:	d130      	bne.n	80011b8 <__aeabi_dadd+0x63c>
 8001156:	0742      	lsls	r2, r0, #29
 8001158:	4313      	orrs	r3, r2
 800115a:	08c0      	lsrs	r0, r0, #3
 800115c:	e65c      	b.n	8000e18 <__aeabi_dadd+0x29c>
 800115e:	077b      	lsls	r3, r7, #29
 8001160:	08c9      	lsrs	r1, r1, #3
 8001162:	430b      	orrs	r3, r1
 8001164:	08f8      	lsrs	r0, r7, #3
 8001166:	e639      	b.n	8000ddc <__aeabi_dadd+0x260>
 8001168:	185c      	adds	r4, r3, r1
 800116a:	429c      	cmp	r4, r3
 800116c:	419b      	sbcs	r3, r3
 800116e:	4440      	add	r0, r8
 8001170:	425b      	negs	r3, r3
 8001172:	18c7      	adds	r7, r0, r3
 8001174:	023b      	lsls	r3, r7, #8
 8001176:	d400      	bmi.n	800117a <__aeabi_dadd+0x5fe>
 8001178:	e625      	b.n	8000dc6 <__aeabi_dadd+0x24a>
 800117a:	4b1d      	ldr	r3, [pc, #116]	; (80011f0 <__aeabi_dadd+0x674>)
 800117c:	2601      	movs	r6, #1
 800117e:	401f      	ands	r7, r3
 8001180:	e621      	b.n	8000dc6 <__aeabi_dadd+0x24a>
 8001182:	0004      	movs	r4, r0
 8001184:	3a20      	subs	r2, #32
 8001186:	40d4      	lsrs	r4, r2
 8001188:	4662      	mov	r2, ip
 800118a:	2a20      	cmp	r2, #32
 800118c:	d004      	beq.n	8001198 <__aeabi_dadd+0x61c>
 800118e:	2240      	movs	r2, #64	; 0x40
 8001190:	4666      	mov	r6, ip
 8001192:	1b92      	subs	r2, r2, r6
 8001194:	4090      	lsls	r0, r2
 8001196:	4303      	orrs	r3, r0
 8001198:	1e5a      	subs	r2, r3, #1
 800119a:	4193      	sbcs	r3, r2
 800119c:	431c      	orrs	r4, r3
 800119e:	e67e      	b.n	8000e9e <__aeabi_dadd+0x322>
 80011a0:	185c      	adds	r4, r3, r1
 80011a2:	428c      	cmp	r4, r1
 80011a4:	4189      	sbcs	r1, r1
 80011a6:	4440      	add	r0, r8
 80011a8:	4249      	negs	r1, r1
 80011aa:	1847      	adds	r7, r0, r1
 80011ac:	e6dd      	b.n	8000f6a <__aeabi_dadd+0x3ee>
 80011ae:	0023      	movs	r3, r4
 80011b0:	433b      	orrs	r3, r7
 80011b2:	d100      	bne.n	80011b6 <__aeabi_dadd+0x63a>
 80011b4:	e6ad      	b.n	8000f12 <__aeabi_dadd+0x396>
 80011b6:	e606      	b.n	8000dc6 <__aeabi_dadd+0x24a>
 80011b8:	0744      	lsls	r4, r0, #29
 80011ba:	4323      	orrs	r3, r4
 80011bc:	2480      	movs	r4, #128	; 0x80
 80011be:	08c0      	lsrs	r0, r0, #3
 80011c0:	0324      	lsls	r4, r4, #12
 80011c2:	4220      	tst	r0, r4
 80011c4:	d008      	beq.n	80011d8 <__aeabi_dadd+0x65c>
 80011c6:	4642      	mov	r2, r8
 80011c8:	08d6      	lsrs	r6, r2, #3
 80011ca:	4226      	tst	r6, r4
 80011cc:	d104      	bne.n	80011d8 <__aeabi_dadd+0x65c>
 80011ce:	4655      	mov	r5, sl
 80011d0:	0030      	movs	r0, r6
 80011d2:	08cb      	lsrs	r3, r1, #3
 80011d4:	0751      	lsls	r1, r2, #29
 80011d6:	430b      	orrs	r3, r1
 80011d8:	0f5a      	lsrs	r2, r3, #29
 80011da:	00db      	lsls	r3, r3, #3
 80011dc:	08db      	lsrs	r3, r3, #3
 80011de:	0752      	lsls	r2, r2, #29
 80011e0:	4313      	orrs	r3, r2
 80011e2:	e619      	b.n	8000e18 <__aeabi_dadd+0x29c>
 80011e4:	2300      	movs	r3, #0
 80011e6:	4a01      	ldr	r2, [pc, #4]	; (80011ec <__aeabi_dadd+0x670>)
 80011e8:	001f      	movs	r7, r3
 80011ea:	e55e      	b.n	8000caa <__aeabi_dadd+0x12e>
 80011ec:	000007ff 	.word	0x000007ff
 80011f0:	ff7fffff 	.word	0xff7fffff

080011f4 <__aeabi_ddiv>:
 80011f4:	b5f0      	push	{r4, r5, r6, r7, lr}
 80011f6:	4657      	mov	r7, sl
 80011f8:	464e      	mov	r6, r9
 80011fa:	4645      	mov	r5, r8
 80011fc:	46de      	mov	lr, fp
 80011fe:	b5e0      	push	{r5, r6, r7, lr}
 8001200:	4681      	mov	r9, r0
 8001202:	0005      	movs	r5, r0
 8001204:	030c      	lsls	r4, r1, #12
 8001206:	0048      	lsls	r0, r1, #1
 8001208:	4692      	mov	sl, r2
 800120a:	001f      	movs	r7, r3
 800120c:	b085      	sub	sp, #20
 800120e:	0b24      	lsrs	r4, r4, #12
 8001210:	0d40      	lsrs	r0, r0, #21
 8001212:	0fce      	lsrs	r6, r1, #31
 8001214:	2800      	cmp	r0, #0
 8001216:	d100      	bne.n	800121a <__aeabi_ddiv+0x26>
 8001218:	e156      	b.n	80014c8 <__aeabi_ddiv+0x2d4>
 800121a:	4bd4      	ldr	r3, [pc, #848]	; (800156c <__aeabi_ddiv+0x378>)
 800121c:	4298      	cmp	r0, r3
 800121e:	d100      	bne.n	8001222 <__aeabi_ddiv+0x2e>
 8001220:	e172      	b.n	8001508 <__aeabi_ddiv+0x314>
 8001222:	0f6b      	lsrs	r3, r5, #29
 8001224:	00e4      	lsls	r4, r4, #3
 8001226:	431c      	orrs	r4, r3
 8001228:	2380      	movs	r3, #128	; 0x80
 800122a:	041b      	lsls	r3, r3, #16
 800122c:	4323      	orrs	r3, r4
 800122e:	4698      	mov	r8, r3
 8001230:	4bcf      	ldr	r3, [pc, #828]	; (8001570 <__aeabi_ddiv+0x37c>)
 8001232:	00ed      	lsls	r5, r5, #3
 8001234:	469b      	mov	fp, r3
 8001236:	2300      	movs	r3, #0
 8001238:	4699      	mov	r9, r3
 800123a:	4483      	add	fp, r0
 800123c:	9300      	str	r3, [sp, #0]
 800123e:	033c      	lsls	r4, r7, #12
 8001240:	007b      	lsls	r3, r7, #1
 8001242:	4650      	mov	r0, sl
 8001244:	0b24      	lsrs	r4, r4, #12
 8001246:	0d5b      	lsrs	r3, r3, #21
 8001248:	0fff      	lsrs	r7, r7, #31
 800124a:	2b00      	cmp	r3, #0
 800124c:	d100      	bne.n	8001250 <__aeabi_ddiv+0x5c>
 800124e:	e11f      	b.n	8001490 <__aeabi_ddiv+0x29c>
 8001250:	4ac6      	ldr	r2, [pc, #792]	; (800156c <__aeabi_ddiv+0x378>)
 8001252:	4293      	cmp	r3, r2
 8001254:	d100      	bne.n	8001258 <__aeabi_ddiv+0x64>
 8001256:	e162      	b.n	800151e <__aeabi_ddiv+0x32a>
 8001258:	49c5      	ldr	r1, [pc, #788]	; (8001570 <__aeabi_ddiv+0x37c>)
 800125a:	0f42      	lsrs	r2, r0, #29
 800125c:	468c      	mov	ip, r1
 800125e:	00e4      	lsls	r4, r4, #3
 8001260:	4659      	mov	r1, fp
 8001262:	4314      	orrs	r4, r2
 8001264:	2280      	movs	r2, #128	; 0x80
 8001266:	4463      	add	r3, ip
 8001268:	0412      	lsls	r2, r2, #16
 800126a:	1acb      	subs	r3, r1, r3
 800126c:	4314      	orrs	r4, r2
 800126e:	469b      	mov	fp, r3
 8001270:	00c2      	lsls	r2, r0, #3
 8001272:	2000      	movs	r0, #0
 8001274:	0033      	movs	r3, r6
 8001276:	407b      	eors	r3, r7
 8001278:	469a      	mov	sl, r3
 800127a:	464b      	mov	r3, r9
 800127c:	2b0f      	cmp	r3, #15
 800127e:	d827      	bhi.n	80012d0 <__aeabi_ddiv+0xdc>
 8001280:	49bc      	ldr	r1, [pc, #752]	; (8001574 <__aeabi_ddiv+0x380>)
 8001282:	009b      	lsls	r3, r3, #2
 8001284:	58cb      	ldr	r3, [r1, r3]
 8001286:	469f      	mov	pc, r3
 8001288:	46b2      	mov	sl, r6
 800128a:	9b00      	ldr	r3, [sp, #0]
 800128c:	2b02      	cmp	r3, #2
 800128e:	d016      	beq.n	80012be <__aeabi_ddiv+0xca>
 8001290:	2b03      	cmp	r3, #3
 8001292:	d100      	bne.n	8001296 <__aeabi_ddiv+0xa2>
 8001294:	e28e      	b.n	80017b4 <__aeabi_ddiv+0x5c0>
 8001296:	2b01      	cmp	r3, #1
 8001298:	d000      	beq.n	800129c <__aeabi_ddiv+0xa8>
 800129a:	e0d9      	b.n	8001450 <__aeabi_ddiv+0x25c>
 800129c:	2300      	movs	r3, #0
 800129e:	2400      	movs	r4, #0
 80012a0:	2500      	movs	r5, #0
 80012a2:	4652      	mov	r2, sl
 80012a4:	051b      	lsls	r3, r3, #20
 80012a6:	4323      	orrs	r3, r4
 80012a8:	07d2      	lsls	r2, r2, #31
 80012aa:	4313      	orrs	r3, r2
 80012ac:	0028      	movs	r0, r5
 80012ae:	0019      	movs	r1, r3
 80012b0:	b005      	add	sp, #20
 80012b2:	bcf0      	pop	{r4, r5, r6, r7}
 80012b4:	46bb      	mov	fp, r7
 80012b6:	46b2      	mov	sl, r6
 80012b8:	46a9      	mov	r9, r5
 80012ba:	46a0      	mov	r8, r4
 80012bc:	bdf0      	pop	{r4, r5, r6, r7, pc}
 80012be:	2400      	movs	r4, #0
 80012c0:	2500      	movs	r5, #0
 80012c2:	4baa      	ldr	r3, [pc, #680]	; (800156c <__aeabi_ddiv+0x378>)
 80012c4:	e7ed      	b.n	80012a2 <__aeabi_ddiv+0xae>
 80012c6:	46ba      	mov	sl, r7
 80012c8:	46a0      	mov	r8, r4
 80012ca:	0015      	movs	r5, r2
 80012cc:	9000      	str	r0, [sp, #0]
 80012ce:	e7dc      	b.n	800128a <__aeabi_ddiv+0x96>
 80012d0:	4544      	cmp	r4, r8
 80012d2:	d200      	bcs.n	80012d6 <__aeabi_ddiv+0xe2>
 80012d4:	e1c7      	b.n	8001666 <__aeabi_ddiv+0x472>
 80012d6:	d100      	bne.n	80012da <__aeabi_ddiv+0xe6>
 80012d8:	e1c2      	b.n	8001660 <__aeabi_ddiv+0x46c>
 80012da:	2301      	movs	r3, #1
 80012dc:	425b      	negs	r3, r3
 80012de:	469c      	mov	ip, r3
 80012e0:	002e      	movs	r6, r5
 80012e2:	4640      	mov	r0, r8
 80012e4:	2500      	movs	r5, #0
 80012e6:	44e3      	add	fp, ip
 80012e8:	0223      	lsls	r3, r4, #8
 80012ea:	0e14      	lsrs	r4, r2, #24
 80012ec:	431c      	orrs	r4, r3
 80012ee:	0c1b      	lsrs	r3, r3, #16
 80012f0:	4699      	mov	r9, r3
 80012f2:	0423      	lsls	r3, r4, #16
 80012f4:	0c1f      	lsrs	r7, r3, #16
 80012f6:	0212      	lsls	r2, r2, #8
 80012f8:	4649      	mov	r1, r9
 80012fa:	9200      	str	r2, [sp, #0]
 80012fc:	9701      	str	r7, [sp, #4]
 80012fe:	f7fe ffa5 	bl	800024c <__aeabi_uidivmod>
 8001302:	0002      	movs	r2, r0
 8001304:	437a      	muls	r2, r7
 8001306:	040b      	lsls	r3, r1, #16
 8001308:	0c31      	lsrs	r1, r6, #16
 800130a:	4680      	mov	r8, r0
 800130c:	4319      	orrs	r1, r3
 800130e:	428a      	cmp	r2, r1
 8001310:	d907      	bls.n	8001322 <__aeabi_ddiv+0x12e>
 8001312:	2301      	movs	r3, #1
 8001314:	425b      	negs	r3, r3
 8001316:	469c      	mov	ip, r3
 8001318:	1909      	adds	r1, r1, r4
 800131a:	44e0      	add	r8, ip
 800131c:	428c      	cmp	r4, r1
 800131e:	d800      	bhi.n	8001322 <__aeabi_ddiv+0x12e>
 8001320:	e207      	b.n	8001732 <__aeabi_ddiv+0x53e>
 8001322:	1a88      	subs	r0, r1, r2
 8001324:	4649      	mov	r1, r9
 8001326:	f7fe ff91 	bl	800024c <__aeabi_uidivmod>
 800132a:	0409      	lsls	r1, r1, #16
 800132c:	468c      	mov	ip, r1
 800132e:	0431      	lsls	r1, r6, #16
 8001330:	4666      	mov	r6, ip
 8001332:	9a01      	ldr	r2, [sp, #4]
 8001334:	0c09      	lsrs	r1, r1, #16
 8001336:	4342      	muls	r2, r0
 8001338:	0003      	movs	r3, r0
 800133a:	4331      	orrs	r1, r6
 800133c:	428a      	cmp	r2, r1
 800133e:	d904      	bls.n	800134a <__aeabi_ddiv+0x156>
 8001340:	1909      	adds	r1, r1, r4
 8001342:	3b01      	subs	r3, #1
 8001344:	428c      	cmp	r4, r1
 8001346:	d800      	bhi.n	800134a <__aeabi_ddiv+0x156>
 8001348:	e1ed      	b.n	8001726 <__aeabi_ddiv+0x532>
 800134a:	1a88      	subs	r0, r1, r2
 800134c:	4642      	mov	r2, r8
 800134e:	0412      	lsls	r2, r2, #16
 8001350:	431a      	orrs	r2, r3
 8001352:	4690      	mov	r8, r2
 8001354:	4641      	mov	r1, r8
 8001356:	9b00      	ldr	r3, [sp, #0]
 8001358:	040e      	lsls	r6, r1, #16
 800135a:	0c1b      	lsrs	r3, r3, #16
 800135c:	001f      	movs	r7, r3
 800135e:	9302      	str	r3, [sp, #8]
 8001360:	9b00      	ldr	r3, [sp, #0]
 8001362:	0c36      	lsrs	r6, r6, #16
 8001364:	041b      	lsls	r3, r3, #16
 8001366:	0c19      	lsrs	r1, r3, #16
 8001368:	000b      	movs	r3, r1
 800136a:	4373      	muls	r3, r6
 800136c:	0c12      	lsrs	r2, r2, #16
 800136e:	437e      	muls	r6, r7
 8001370:	9103      	str	r1, [sp, #12]
 8001372:	4351      	muls	r1, r2
 8001374:	437a      	muls	r2, r7
 8001376:	0c1f      	lsrs	r7, r3, #16
 8001378:	46bc      	mov	ip, r7
 800137a:	1876      	adds	r6, r6, r1
 800137c:	4466      	add	r6, ip
 800137e:	42b1      	cmp	r1, r6
 8001380:	d903      	bls.n	800138a <__aeabi_ddiv+0x196>
 8001382:	2180      	movs	r1, #128	; 0x80
 8001384:	0249      	lsls	r1, r1, #9
 8001386:	468c      	mov	ip, r1
 8001388:	4462      	add	r2, ip
 800138a:	0c31      	lsrs	r1, r6, #16
 800138c:	188a      	adds	r2, r1, r2
 800138e:	0431      	lsls	r1, r6, #16
 8001390:	041e      	lsls	r6, r3, #16
 8001392:	0c36      	lsrs	r6, r6, #16
 8001394:	198e      	adds	r6, r1, r6
 8001396:	4290      	cmp	r0, r2
 8001398:	d302      	bcc.n	80013a0 <__aeabi_ddiv+0x1ac>
 800139a:	d112      	bne.n	80013c2 <__aeabi_ddiv+0x1ce>
 800139c:	42b5      	cmp	r5, r6
 800139e:	d210      	bcs.n	80013c2 <__aeabi_ddiv+0x1ce>
 80013a0:	4643      	mov	r3, r8
 80013a2:	1e59      	subs	r1, r3, #1
 80013a4:	9b00      	ldr	r3, [sp, #0]
 80013a6:	469c      	mov	ip, r3
 80013a8:	4465      	add	r5, ip
 80013aa:	001f      	movs	r7, r3
 80013ac:	429d      	cmp	r5, r3
 80013ae:	419b      	sbcs	r3, r3
 80013b0:	425b      	negs	r3, r3
 80013b2:	191b      	adds	r3, r3, r4
 80013b4:	18c0      	adds	r0, r0, r3
 80013b6:	4284      	cmp	r4, r0
 80013b8:	d200      	bcs.n	80013bc <__aeabi_ddiv+0x1c8>
 80013ba:	e1a0      	b.n	80016fe <__aeabi_ddiv+0x50a>
 80013bc:	d100      	bne.n	80013c0 <__aeabi_ddiv+0x1cc>
 80013be:	e19b      	b.n	80016f8 <__aeabi_ddiv+0x504>
 80013c0:	4688      	mov	r8, r1
 80013c2:	1bae      	subs	r6, r5, r6
 80013c4:	42b5      	cmp	r5, r6
 80013c6:	41ad      	sbcs	r5, r5
 80013c8:	1a80      	subs	r0, r0, r2
 80013ca:	426d      	negs	r5, r5
 80013cc:	1b40      	subs	r0, r0, r5
 80013ce:	4284      	cmp	r4, r0
 80013d0:	d100      	bne.n	80013d4 <__aeabi_ddiv+0x1e0>
 80013d2:	e1d5      	b.n	8001780 <__aeabi_ddiv+0x58c>
 80013d4:	4649      	mov	r1, r9
 80013d6:	f7fe ff39 	bl	800024c <__aeabi_uidivmod>
 80013da:	9a01      	ldr	r2, [sp, #4]
 80013dc:	040b      	lsls	r3, r1, #16
 80013de:	4342      	muls	r2, r0
 80013e0:	0c31      	lsrs	r1, r6, #16
 80013e2:	0005      	movs	r5, r0
 80013e4:	4319      	orrs	r1, r3
 80013e6:	428a      	cmp	r2, r1
 80013e8:	d900      	bls.n	80013ec <__aeabi_ddiv+0x1f8>
 80013ea:	e16c      	b.n	80016c6 <__aeabi_ddiv+0x4d2>
 80013ec:	1a88      	subs	r0, r1, r2
 80013ee:	4649      	mov	r1, r9
 80013f0:	f7fe ff2c 	bl	800024c <__aeabi_uidivmod>
 80013f4:	9a01      	ldr	r2, [sp, #4]
 80013f6:	0436      	lsls	r6, r6, #16
 80013f8:	4342      	muls	r2, r0
 80013fa:	0409      	lsls	r1, r1, #16
 80013fc:	0c36      	lsrs	r6, r6, #16
 80013fe:	0003      	movs	r3, r0
 8001400:	430e      	orrs	r6, r1
 8001402:	42b2      	cmp	r2, r6
 8001404:	d900      	bls.n	8001408 <__aeabi_ddiv+0x214>
 8001406:	e153      	b.n	80016b0 <__aeabi_ddiv+0x4bc>
 8001408:	9803      	ldr	r0, [sp, #12]
 800140a:	1ab6      	subs	r6, r6, r2
 800140c:	0002      	movs	r2, r0
 800140e:	042d      	lsls	r5, r5, #16
 8001410:	431d      	orrs	r5, r3
 8001412:	9f02      	ldr	r7, [sp, #8]
 8001414:	042b      	lsls	r3, r5, #16
 8001416:	0c1b      	lsrs	r3, r3, #16
 8001418:	435a      	muls	r2, r3
 800141a:	437b      	muls	r3, r7
 800141c:	469c      	mov	ip, r3
 800141e:	0c29      	lsrs	r1, r5, #16
 8001420:	4348      	muls	r0, r1
 8001422:	0c13      	lsrs	r3, r2, #16
 8001424:	4484      	add	ip, r0
 8001426:	4463      	add	r3, ip
 8001428:	4379      	muls	r1, r7
 800142a:	4298      	cmp	r0, r3
 800142c:	d903      	bls.n	8001436 <__aeabi_ddiv+0x242>
 800142e:	2080      	movs	r0, #128	; 0x80
 8001430:	0240      	lsls	r0, r0, #9
 8001432:	4684      	mov	ip, r0
 8001434:	4461      	add	r1, ip
 8001436:	0c18      	lsrs	r0, r3, #16
 8001438:	0412      	lsls	r2, r2, #16
 800143a:	041b      	lsls	r3, r3, #16
 800143c:	0c12      	lsrs	r2, r2, #16
 800143e:	1841      	adds	r1, r0, r1
 8001440:	189b      	adds	r3, r3, r2
 8001442:	428e      	cmp	r6, r1
 8001444:	d200      	bcs.n	8001448 <__aeabi_ddiv+0x254>
 8001446:	e0ff      	b.n	8001648 <__aeabi_ddiv+0x454>
 8001448:	d100      	bne.n	800144c <__aeabi_ddiv+0x258>
 800144a:	e0fa      	b.n	8001642 <__aeabi_ddiv+0x44e>
 800144c:	2301      	movs	r3, #1
 800144e:	431d      	orrs	r5, r3
 8001450:	4a49      	ldr	r2, [pc, #292]	; (8001578 <__aeabi_ddiv+0x384>)
 8001452:	445a      	add	r2, fp
 8001454:	2a00      	cmp	r2, #0
 8001456:	dc00      	bgt.n	800145a <__aeabi_ddiv+0x266>
 8001458:	e0aa      	b.n	80015b0 <__aeabi_ddiv+0x3bc>
 800145a:	076b      	lsls	r3, r5, #29
 800145c:	d000      	beq.n	8001460 <__aeabi_ddiv+0x26c>
 800145e:	e13d      	b.n	80016dc <__aeabi_ddiv+0x4e8>
 8001460:	08ed      	lsrs	r5, r5, #3
 8001462:	4643      	mov	r3, r8
 8001464:	01db      	lsls	r3, r3, #7
 8001466:	d506      	bpl.n	8001476 <__aeabi_ddiv+0x282>
 8001468:	4642      	mov	r2, r8
 800146a:	4b44      	ldr	r3, [pc, #272]	; (800157c <__aeabi_ddiv+0x388>)
 800146c:	401a      	ands	r2, r3
 800146e:	4690      	mov	r8, r2
 8001470:	2280      	movs	r2, #128	; 0x80
 8001472:	00d2      	lsls	r2, r2, #3
 8001474:	445a      	add	r2, fp
 8001476:	4b42      	ldr	r3, [pc, #264]	; (8001580 <__aeabi_ddiv+0x38c>)
 8001478:	429a      	cmp	r2, r3
 800147a:	dd00      	ble.n	800147e <__aeabi_ddiv+0x28a>
 800147c:	e71f      	b.n	80012be <__aeabi_ddiv+0xca>
 800147e:	4643      	mov	r3, r8
 8001480:	075b      	lsls	r3, r3, #29
 8001482:	431d      	orrs	r5, r3
 8001484:	4643      	mov	r3, r8
 8001486:	0552      	lsls	r2, r2, #21
 8001488:	025c      	lsls	r4, r3, #9
 800148a:	0b24      	lsrs	r4, r4, #12
 800148c:	0d53      	lsrs	r3, r2, #21
 800148e:	e708      	b.n	80012a2 <__aeabi_ddiv+0xae>
 8001490:	4652      	mov	r2, sl
 8001492:	4322      	orrs	r2, r4
 8001494:	d100      	bne.n	8001498 <__aeabi_ddiv+0x2a4>
 8001496:	e07b      	b.n	8001590 <__aeabi_ddiv+0x39c>
 8001498:	2c00      	cmp	r4, #0
 800149a:	d100      	bne.n	800149e <__aeabi_ddiv+0x2aa>
 800149c:	e0fa      	b.n	8001694 <__aeabi_ddiv+0x4a0>
 800149e:	0020      	movs	r0, r4
 80014a0:	f001 fa22 	bl	80028e8 <__clzsi2>
 80014a4:	0002      	movs	r2, r0
 80014a6:	3a0b      	subs	r2, #11
 80014a8:	231d      	movs	r3, #29
 80014aa:	0001      	movs	r1, r0
 80014ac:	1a9b      	subs	r3, r3, r2
 80014ae:	4652      	mov	r2, sl
 80014b0:	3908      	subs	r1, #8
 80014b2:	40da      	lsrs	r2, r3
 80014b4:	408c      	lsls	r4, r1
 80014b6:	4314      	orrs	r4, r2
 80014b8:	4652      	mov	r2, sl
 80014ba:	408a      	lsls	r2, r1
 80014bc:	4b31      	ldr	r3, [pc, #196]	; (8001584 <__aeabi_ddiv+0x390>)
 80014be:	4458      	add	r0, fp
 80014c0:	469b      	mov	fp, r3
 80014c2:	4483      	add	fp, r0
 80014c4:	2000      	movs	r0, #0
 80014c6:	e6d5      	b.n	8001274 <__aeabi_ddiv+0x80>
 80014c8:	464b      	mov	r3, r9
 80014ca:	4323      	orrs	r3, r4
 80014cc:	4698      	mov	r8, r3
 80014ce:	d044      	beq.n	800155a <__aeabi_ddiv+0x366>
 80014d0:	2c00      	cmp	r4, #0
 80014d2:	d100      	bne.n	80014d6 <__aeabi_ddiv+0x2e2>
 80014d4:	e0ce      	b.n	8001674 <__aeabi_ddiv+0x480>
 80014d6:	0020      	movs	r0, r4
 80014d8:	f001 fa06 	bl	80028e8 <__clzsi2>
 80014dc:	0001      	movs	r1, r0
 80014de:	0002      	movs	r2, r0
 80014e0:	390b      	subs	r1, #11
 80014e2:	231d      	movs	r3, #29
 80014e4:	1a5b      	subs	r3, r3, r1
 80014e6:	4649      	mov	r1, r9
 80014e8:	0010      	movs	r0, r2
 80014ea:	40d9      	lsrs	r1, r3
 80014ec:	3808      	subs	r0, #8
 80014ee:	4084      	lsls	r4, r0
 80014f0:	000b      	movs	r3, r1
 80014f2:	464d      	mov	r5, r9
 80014f4:	4323      	orrs	r3, r4
 80014f6:	4698      	mov	r8, r3
 80014f8:	4085      	lsls	r5, r0
 80014fa:	4823      	ldr	r0, [pc, #140]	; (8001588 <__aeabi_ddiv+0x394>)
 80014fc:	1a83      	subs	r3, r0, r2
 80014fe:	469b      	mov	fp, r3
 8001500:	2300      	movs	r3, #0
 8001502:	4699      	mov	r9, r3
 8001504:	9300      	str	r3, [sp, #0]
 8001506:	e69a      	b.n	800123e <__aeabi_ddiv+0x4a>
 8001508:	464b      	mov	r3, r9
 800150a:	4323      	orrs	r3, r4
 800150c:	4698      	mov	r8, r3
 800150e:	d11d      	bne.n	800154c <__aeabi_ddiv+0x358>
 8001510:	2308      	movs	r3, #8
 8001512:	4699      	mov	r9, r3
 8001514:	3b06      	subs	r3, #6
 8001516:	2500      	movs	r5, #0
 8001518:	4683      	mov	fp, r0
 800151a:	9300      	str	r3, [sp, #0]
 800151c:	e68f      	b.n	800123e <__aeabi_ddiv+0x4a>
 800151e:	4652      	mov	r2, sl
 8001520:	4322      	orrs	r2, r4
 8001522:	d109      	bne.n	8001538 <__aeabi_ddiv+0x344>
 8001524:	2302      	movs	r3, #2
 8001526:	4649      	mov	r1, r9
 8001528:	4319      	orrs	r1, r3
 800152a:	4b18      	ldr	r3, [pc, #96]	; (800158c <__aeabi_ddiv+0x398>)
 800152c:	4689      	mov	r9, r1
 800152e:	469c      	mov	ip, r3
 8001530:	2400      	movs	r4, #0
 8001532:	2002      	movs	r0, #2
 8001534:	44e3      	add	fp, ip
 8001536:	e69d      	b.n	8001274 <__aeabi_ddiv+0x80>
 8001538:	2303      	movs	r3, #3
 800153a:	464a      	mov	r2, r9
 800153c:	431a      	orrs	r2, r3
 800153e:	4b13      	ldr	r3, [pc, #76]	; (800158c <__aeabi_ddiv+0x398>)
 8001540:	4691      	mov	r9, r2
 8001542:	469c      	mov	ip, r3
 8001544:	4652      	mov	r2, sl
 8001546:	2003      	movs	r0, #3
 8001548:	44e3      	add	fp, ip
 800154a:	e693      	b.n	8001274 <__aeabi_ddiv+0x80>
 800154c:	230c      	movs	r3, #12
 800154e:	4699      	mov	r9, r3
 8001550:	3b09      	subs	r3, #9
 8001552:	46a0      	mov	r8, r4
 8001554:	4683      	mov	fp, r0
 8001556:	9300      	str	r3, [sp, #0]
 8001558:	e671      	b.n	800123e <__aeabi_ddiv+0x4a>
 800155a:	2304      	movs	r3, #4
 800155c:	4699      	mov	r9, r3
 800155e:	2300      	movs	r3, #0
 8001560:	469b      	mov	fp, r3
 8001562:	3301      	adds	r3, #1
 8001564:	2500      	movs	r5, #0
 8001566:	9300      	str	r3, [sp, #0]
 8001568:	e669      	b.n	800123e <__aeabi_ddiv+0x4a>
 800156a:	46c0      	nop			; (mov r8, r8)
 800156c:	000007ff 	.word	0x000007ff
 8001570:	fffffc01 	.word	0xfffffc01
 8001574:	0800a038 	.word	0x0800a038
 8001578:	000003ff 	.word	0x000003ff
 800157c:	feffffff 	.word	0xfeffffff
 8001580:	000007fe 	.word	0x000007fe
 8001584:	000003f3 	.word	0x000003f3
 8001588:	fffffc0d 	.word	0xfffffc0d
 800158c:	fffff801 	.word	0xfffff801
 8001590:	4649      	mov	r1, r9
 8001592:	2301      	movs	r3, #1
 8001594:	4319      	orrs	r1, r3
 8001596:	4689      	mov	r9, r1
 8001598:	2400      	movs	r4, #0
 800159a:	2001      	movs	r0, #1
 800159c:	e66a      	b.n	8001274 <__aeabi_ddiv+0x80>
 800159e:	2300      	movs	r3, #0
 80015a0:	2480      	movs	r4, #128	; 0x80
 80015a2:	469a      	mov	sl, r3
 80015a4:	2500      	movs	r5, #0
 80015a6:	4b8a      	ldr	r3, [pc, #552]	; (80017d0 <__aeabi_ddiv+0x5dc>)
 80015a8:	0324      	lsls	r4, r4, #12
 80015aa:	e67a      	b.n	80012a2 <__aeabi_ddiv+0xae>
 80015ac:	2501      	movs	r5, #1
 80015ae:	426d      	negs	r5, r5
 80015b0:	2301      	movs	r3, #1
 80015b2:	1a9b      	subs	r3, r3, r2
 80015b4:	2b38      	cmp	r3, #56	; 0x38
 80015b6:	dd00      	ble.n	80015ba <__aeabi_ddiv+0x3c6>
 80015b8:	e670      	b.n	800129c <__aeabi_ddiv+0xa8>
 80015ba:	2b1f      	cmp	r3, #31
 80015bc:	dc00      	bgt.n	80015c0 <__aeabi_ddiv+0x3cc>
 80015be:	e0bf      	b.n	8001740 <__aeabi_ddiv+0x54c>
 80015c0:	211f      	movs	r1, #31
 80015c2:	4249      	negs	r1, r1
 80015c4:	1a8a      	subs	r2, r1, r2
 80015c6:	4641      	mov	r1, r8
 80015c8:	40d1      	lsrs	r1, r2
 80015ca:	000a      	movs	r2, r1
 80015cc:	2b20      	cmp	r3, #32
 80015ce:	d004      	beq.n	80015da <__aeabi_ddiv+0x3e6>
 80015d0:	4641      	mov	r1, r8
 80015d2:	4b80      	ldr	r3, [pc, #512]	; (80017d4 <__aeabi_ddiv+0x5e0>)
 80015d4:	445b      	add	r3, fp
 80015d6:	4099      	lsls	r1, r3
 80015d8:	430d      	orrs	r5, r1
 80015da:	1e6b      	subs	r3, r5, #1
 80015dc:	419d      	sbcs	r5, r3
 80015de:	2307      	movs	r3, #7
 80015e0:	432a      	orrs	r2, r5
 80015e2:	001d      	movs	r5, r3
 80015e4:	2400      	movs	r4, #0
 80015e6:	4015      	ands	r5, r2
 80015e8:	4213      	tst	r3, r2
 80015ea:	d100      	bne.n	80015ee <__aeabi_ddiv+0x3fa>
 80015ec:	e0d4      	b.n	8001798 <__aeabi_ddiv+0x5a4>
 80015ee:	210f      	movs	r1, #15
 80015f0:	2300      	movs	r3, #0
 80015f2:	4011      	ands	r1, r2
 80015f4:	2904      	cmp	r1, #4
 80015f6:	d100      	bne.n	80015fa <__aeabi_ddiv+0x406>
 80015f8:	e0cb      	b.n	8001792 <__aeabi_ddiv+0x59e>
 80015fa:	1d11      	adds	r1, r2, #4
 80015fc:	4291      	cmp	r1, r2
 80015fe:	4192      	sbcs	r2, r2
 8001600:	4252      	negs	r2, r2
 8001602:	189b      	adds	r3, r3, r2
 8001604:	000a      	movs	r2, r1
 8001606:	0219      	lsls	r1, r3, #8
 8001608:	d400      	bmi.n	800160c <__aeabi_ddiv+0x418>
 800160a:	e0c2      	b.n	8001792 <__aeabi_ddiv+0x59e>
 800160c:	2301      	movs	r3, #1
 800160e:	2400      	movs	r4, #0
 8001610:	2500      	movs	r5, #0
 8001612:	e646      	b.n	80012a2 <__aeabi_ddiv+0xae>
 8001614:	2380      	movs	r3, #128	; 0x80
 8001616:	4641      	mov	r1, r8
 8001618:	031b      	lsls	r3, r3, #12
 800161a:	4219      	tst	r1, r3
 800161c:	d008      	beq.n	8001630 <__aeabi_ddiv+0x43c>
 800161e:	421c      	tst	r4, r3
 8001620:	d106      	bne.n	8001630 <__aeabi_ddiv+0x43c>
 8001622:	431c      	orrs	r4, r3
 8001624:	0324      	lsls	r4, r4, #12
 8001626:	46ba      	mov	sl, r7
 8001628:	0015      	movs	r5, r2
 800162a:	4b69      	ldr	r3, [pc, #420]	; (80017d0 <__aeabi_ddiv+0x5dc>)
 800162c:	0b24      	lsrs	r4, r4, #12
 800162e:	e638      	b.n	80012a2 <__aeabi_ddiv+0xae>
 8001630:	2480      	movs	r4, #128	; 0x80
 8001632:	4643      	mov	r3, r8
 8001634:	0324      	lsls	r4, r4, #12
 8001636:	431c      	orrs	r4, r3
 8001638:	0324      	lsls	r4, r4, #12
 800163a:	46b2      	mov	sl, r6
 800163c:	4b64      	ldr	r3, [pc, #400]	; (80017d0 <__aeabi_ddiv+0x5dc>)
 800163e:	0b24      	lsrs	r4, r4, #12
 8001640:	e62f      	b.n	80012a2 <__aeabi_ddiv+0xae>
 8001642:	2b00      	cmp	r3, #0
 8001644:	d100      	bne.n	8001648 <__aeabi_ddiv+0x454>
 8001646:	e703      	b.n	8001450 <__aeabi_ddiv+0x25c>
 8001648:	19a6      	adds	r6, r4, r6
 800164a:	1e68      	subs	r0, r5, #1
 800164c:	42a6      	cmp	r6, r4
 800164e:	d200      	bcs.n	8001652 <__aeabi_ddiv+0x45e>
 8001650:	e08d      	b.n	800176e <__aeabi_ddiv+0x57a>
 8001652:	428e      	cmp	r6, r1
 8001654:	d200      	bcs.n	8001658 <__aeabi_ddiv+0x464>
 8001656:	e0a3      	b.n	80017a0 <__aeabi_ddiv+0x5ac>
 8001658:	d100      	bne.n	800165c <__aeabi_ddiv+0x468>
 800165a:	e0b3      	b.n	80017c4 <__aeabi_ddiv+0x5d0>
 800165c:	0005      	movs	r5, r0
 800165e:	e6f5      	b.n	800144c <__aeabi_ddiv+0x258>
 8001660:	42aa      	cmp	r2, r5
 8001662:	d900      	bls.n	8001666 <__aeabi_ddiv+0x472>
 8001664:	e639      	b.n	80012da <__aeabi_ddiv+0xe6>
 8001666:	4643      	mov	r3, r8
 8001668:	07de      	lsls	r6, r3, #31
 800166a:	0858      	lsrs	r0, r3, #1
 800166c:	086b      	lsrs	r3, r5, #1
 800166e:	431e      	orrs	r6, r3
 8001670:	07ed      	lsls	r5, r5, #31
 8001672:	e639      	b.n	80012e8 <__aeabi_ddiv+0xf4>
 8001674:	4648      	mov	r0, r9
 8001676:	f001 f937 	bl	80028e8 <__clzsi2>
 800167a:	0001      	movs	r1, r0
 800167c:	0002      	movs	r2, r0
 800167e:	3115      	adds	r1, #21
 8001680:	3220      	adds	r2, #32
 8001682:	291c      	cmp	r1, #28
 8001684:	dc00      	bgt.n	8001688 <__aeabi_ddiv+0x494>
 8001686:	e72c      	b.n	80014e2 <__aeabi_ddiv+0x2ee>
 8001688:	464b      	mov	r3, r9
 800168a:	3808      	subs	r0, #8
 800168c:	4083      	lsls	r3, r0
 800168e:	2500      	movs	r5, #0
 8001690:	4698      	mov	r8, r3
 8001692:	e732      	b.n	80014fa <__aeabi_ddiv+0x306>
 8001694:	f001 f928 	bl	80028e8 <__clzsi2>
 8001698:	0003      	movs	r3, r0
 800169a:	001a      	movs	r2, r3
 800169c:	3215      	adds	r2, #21
 800169e:	3020      	adds	r0, #32
 80016a0:	2a1c      	cmp	r2, #28
 80016a2:	dc00      	bgt.n	80016a6 <__aeabi_ddiv+0x4b2>
 80016a4:	e700      	b.n	80014a8 <__aeabi_ddiv+0x2b4>
 80016a6:	4654      	mov	r4, sl
 80016a8:	3b08      	subs	r3, #8
 80016aa:	2200      	movs	r2, #0
 80016ac:	409c      	lsls	r4, r3
 80016ae:	e705      	b.n	80014bc <__aeabi_ddiv+0x2c8>
 80016b0:	1936      	adds	r6, r6, r4
 80016b2:	3b01      	subs	r3, #1
 80016b4:	42b4      	cmp	r4, r6
 80016b6:	d900      	bls.n	80016ba <__aeabi_ddiv+0x4c6>
 80016b8:	e6a6      	b.n	8001408 <__aeabi_ddiv+0x214>
 80016ba:	42b2      	cmp	r2, r6
 80016bc:	d800      	bhi.n	80016c0 <__aeabi_ddiv+0x4cc>
 80016be:	e6a3      	b.n	8001408 <__aeabi_ddiv+0x214>
 80016c0:	1e83      	subs	r3, r0, #2
 80016c2:	1936      	adds	r6, r6, r4
 80016c4:	e6a0      	b.n	8001408 <__aeabi_ddiv+0x214>
 80016c6:	1909      	adds	r1, r1, r4
 80016c8:	3d01      	subs	r5, #1
 80016ca:	428c      	cmp	r4, r1
 80016cc:	d900      	bls.n	80016d0 <__aeabi_ddiv+0x4dc>
 80016ce:	e68d      	b.n	80013ec <__aeabi_ddiv+0x1f8>
 80016d0:	428a      	cmp	r2, r1
 80016d2:	d800      	bhi.n	80016d6 <__aeabi_ddiv+0x4e2>
 80016d4:	e68a      	b.n	80013ec <__aeabi_ddiv+0x1f8>
 80016d6:	1e85      	subs	r5, r0, #2
 80016d8:	1909      	adds	r1, r1, r4
 80016da:	e687      	b.n	80013ec <__aeabi_ddiv+0x1f8>
 80016dc:	230f      	movs	r3, #15
 80016de:	402b      	ands	r3, r5
 80016e0:	2b04      	cmp	r3, #4
 80016e2:	d100      	bne.n	80016e6 <__aeabi_ddiv+0x4f2>
 80016e4:	e6bc      	b.n	8001460 <__aeabi_ddiv+0x26c>
 80016e6:	2305      	movs	r3, #5
 80016e8:	425b      	negs	r3, r3
 80016ea:	42ab      	cmp	r3, r5
 80016ec:	419b      	sbcs	r3, r3
 80016ee:	3504      	adds	r5, #4
 80016f0:	425b      	negs	r3, r3
 80016f2:	08ed      	lsrs	r5, r5, #3
 80016f4:	4498      	add	r8, r3
 80016f6:	e6b4      	b.n	8001462 <__aeabi_ddiv+0x26e>
 80016f8:	42af      	cmp	r7, r5
 80016fa:	d900      	bls.n	80016fe <__aeabi_ddiv+0x50a>
 80016fc:	e660      	b.n	80013c0 <__aeabi_ddiv+0x1cc>
 80016fe:	4282      	cmp	r2, r0
 8001700:	d804      	bhi.n	800170c <__aeabi_ddiv+0x518>
 8001702:	d000      	beq.n	8001706 <__aeabi_ddiv+0x512>
 8001704:	e65c      	b.n	80013c0 <__aeabi_ddiv+0x1cc>
 8001706:	42ae      	cmp	r6, r5
 8001708:	d800      	bhi.n	800170c <__aeabi_ddiv+0x518>
 800170a:	e659      	b.n	80013c0 <__aeabi_ddiv+0x1cc>
 800170c:	2302      	movs	r3, #2
 800170e:	425b      	negs	r3, r3
 8001710:	469c      	mov	ip, r3
 8001712:	9b00      	ldr	r3, [sp, #0]
 8001714:	44e0      	add	r8, ip
 8001716:	469c      	mov	ip, r3
 8001718:	4465      	add	r5, ip
 800171a:	429d      	cmp	r5, r3
 800171c:	419b      	sbcs	r3, r3
 800171e:	425b      	negs	r3, r3
 8001720:	191b      	adds	r3, r3, r4
 8001722:	18c0      	adds	r0, r0, r3
 8001724:	e64d      	b.n	80013c2 <__aeabi_ddiv+0x1ce>
 8001726:	428a      	cmp	r2, r1
 8001728:	d800      	bhi.n	800172c <__aeabi_ddiv+0x538>
 800172a:	e60e      	b.n	800134a <__aeabi_ddiv+0x156>
 800172c:	1e83      	subs	r3, r0, #2
 800172e:	1909      	adds	r1, r1, r4
 8001730:	e60b      	b.n	800134a <__aeabi_ddiv+0x156>
 8001732:	428a      	cmp	r2, r1
 8001734:	d800      	bhi.n	8001738 <__aeabi_ddiv+0x544>
 8001736:	e5f4      	b.n	8001322 <__aeabi_ddiv+0x12e>
 8001738:	1e83      	subs	r3, r0, #2
 800173a:	4698      	mov	r8, r3
 800173c:	1909      	adds	r1, r1, r4
 800173e:	e5f0      	b.n	8001322 <__aeabi_ddiv+0x12e>
 8001740:	4925      	ldr	r1, [pc, #148]	; (80017d8 <__aeabi_ddiv+0x5e4>)
 8001742:	0028      	movs	r0, r5
 8001744:	4459      	add	r1, fp
 8001746:	408d      	lsls	r5, r1
 8001748:	4642      	mov	r2, r8
 800174a:	408a      	lsls	r2, r1
 800174c:	1e69      	subs	r1, r5, #1
 800174e:	418d      	sbcs	r5, r1
 8001750:	4641      	mov	r1, r8
 8001752:	40d8      	lsrs	r0, r3
 8001754:	40d9      	lsrs	r1, r3
 8001756:	4302      	orrs	r2, r0
 8001758:	432a      	orrs	r2, r5
 800175a:	000b      	movs	r3, r1
 800175c:	0751      	lsls	r1, r2, #29
 800175e:	d100      	bne.n	8001762 <__aeabi_ddiv+0x56e>
 8001760:	e751      	b.n	8001606 <__aeabi_ddiv+0x412>
 8001762:	210f      	movs	r1, #15
 8001764:	4011      	ands	r1, r2
 8001766:	2904      	cmp	r1, #4
 8001768:	d000      	beq.n	800176c <__aeabi_ddiv+0x578>
 800176a:	e746      	b.n	80015fa <__aeabi_ddiv+0x406>
 800176c:	e74b      	b.n	8001606 <__aeabi_ddiv+0x412>
 800176e:	0005      	movs	r5, r0
 8001770:	428e      	cmp	r6, r1
 8001772:	d000      	beq.n	8001776 <__aeabi_ddiv+0x582>
 8001774:	e66a      	b.n	800144c <__aeabi_ddiv+0x258>
 8001776:	9a00      	ldr	r2, [sp, #0]
 8001778:	4293      	cmp	r3, r2
 800177a:	d000      	beq.n	800177e <__aeabi_ddiv+0x58a>
 800177c:	e666      	b.n	800144c <__aeabi_ddiv+0x258>
 800177e:	e667      	b.n	8001450 <__aeabi_ddiv+0x25c>
 8001780:	4a16      	ldr	r2, [pc, #88]	; (80017dc <__aeabi_ddiv+0x5e8>)
 8001782:	445a      	add	r2, fp
 8001784:	2a00      	cmp	r2, #0
 8001786:	dc00      	bgt.n	800178a <__aeabi_ddiv+0x596>
 8001788:	e710      	b.n	80015ac <__aeabi_ddiv+0x3b8>
 800178a:	2301      	movs	r3, #1
 800178c:	2500      	movs	r5, #0
 800178e:	4498      	add	r8, r3
 8001790:	e667      	b.n	8001462 <__aeabi_ddiv+0x26e>
 8001792:	075d      	lsls	r5, r3, #29
 8001794:	025b      	lsls	r3, r3, #9
 8001796:	0b1c      	lsrs	r4, r3, #12
 8001798:	08d2      	lsrs	r2, r2, #3
 800179a:	2300      	movs	r3, #0
 800179c:	4315      	orrs	r5, r2
 800179e:	e580      	b.n	80012a2 <__aeabi_ddiv+0xae>
 80017a0:	9800      	ldr	r0, [sp, #0]
 80017a2:	3d02      	subs	r5, #2
 80017a4:	0042      	lsls	r2, r0, #1
 80017a6:	4282      	cmp	r2, r0
 80017a8:	41bf      	sbcs	r7, r7
 80017aa:	427f      	negs	r7, r7
 80017ac:	193c      	adds	r4, r7, r4
 80017ae:	1936      	adds	r6, r6, r4
 80017b0:	9200      	str	r2, [sp, #0]
 80017b2:	e7dd      	b.n	8001770 <__aeabi_ddiv+0x57c>
 80017b4:	2480      	movs	r4, #128	; 0x80
 80017b6:	4643      	mov	r3, r8
 80017b8:	0324      	lsls	r4, r4, #12
 80017ba:	431c      	orrs	r4, r3
 80017bc:	0324      	lsls	r4, r4, #12
 80017be:	4b04      	ldr	r3, [pc, #16]	; (80017d0 <__aeabi_ddiv+0x5dc>)
 80017c0:	0b24      	lsrs	r4, r4, #12
 80017c2:	e56e      	b.n	80012a2 <__aeabi_ddiv+0xae>
 80017c4:	9a00      	ldr	r2, [sp, #0]
 80017c6:	429a      	cmp	r2, r3
 80017c8:	d3ea      	bcc.n	80017a0 <__aeabi_ddiv+0x5ac>
 80017ca:	0005      	movs	r5, r0
 80017cc:	e7d3      	b.n	8001776 <__aeabi_ddiv+0x582>
 80017ce:	46c0      	nop			; (mov r8, r8)
 80017d0:	000007ff 	.word	0x000007ff
 80017d4:	0000043e 	.word	0x0000043e
 80017d8:	0000041e 	.word	0x0000041e
 80017dc:	000003ff 	.word	0x000003ff

080017e0 <__eqdf2>:
 80017e0:	b5f0      	push	{r4, r5, r6, r7, lr}
 80017e2:	464e      	mov	r6, r9
 80017e4:	4645      	mov	r5, r8
 80017e6:	46de      	mov	lr, fp
 80017e8:	4657      	mov	r7, sl
 80017ea:	4690      	mov	r8, r2
 80017ec:	b5e0      	push	{r5, r6, r7, lr}
 80017ee:	0017      	movs	r7, r2
 80017f0:	031a      	lsls	r2, r3, #12
 80017f2:	0b12      	lsrs	r2, r2, #12
 80017f4:	0005      	movs	r5, r0
 80017f6:	4684      	mov	ip, r0
 80017f8:	4819      	ldr	r0, [pc, #100]	; (8001860 <__eqdf2+0x80>)
 80017fa:	030e      	lsls	r6, r1, #12
 80017fc:	004c      	lsls	r4, r1, #1
 80017fe:	4691      	mov	r9, r2
 8001800:	005a      	lsls	r2, r3, #1
 8001802:	0fdb      	lsrs	r3, r3, #31
 8001804:	469b      	mov	fp, r3
 8001806:	0b36      	lsrs	r6, r6, #12
 8001808:	0d64      	lsrs	r4, r4, #21
 800180a:	0fc9      	lsrs	r1, r1, #31
 800180c:	0d52      	lsrs	r2, r2, #21
 800180e:	4284      	cmp	r4, r0
 8001810:	d019      	beq.n	8001846 <__eqdf2+0x66>
 8001812:	4282      	cmp	r2, r0
 8001814:	d010      	beq.n	8001838 <__eqdf2+0x58>
 8001816:	2001      	movs	r0, #1
 8001818:	4294      	cmp	r4, r2
 800181a:	d10e      	bne.n	800183a <__eqdf2+0x5a>
 800181c:	454e      	cmp	r6, r9
 800181e:	d10c      	bne.n	800183a <__eqdf2+0x5a>
 8001820:	2001      	movs	r0, #1
 8001822:	45c4      	cmp	ip, r8
 8001824:	d109      	bne.n	800183a <__eqdf2+0x5a>
 8001826:	4559      	cmp	r1, fp
 8001828:	d017      	beq.n	800185a <__eqdf2+0x7a>
 800182a:	2c00      	cmp	r4, #0
 800182c:	d105      	bne.n	800183a <__eqdf2+0x5a>
 800182e:	0030      	movs	r0, r6
 8001830:	4328      	orrs	r0, r5
 8001832:	1e43      	subs	r3, r0, #1
 8001834:	4198      	sbcs	r0, r3
 8001836:	e000      	b.n	800183a <__eqdf2+0x5a>
 8001838:	2001      	movs	r0, #1
 800183a:	bcf0      	pop	{r4, r5, r6, r7}
 800183c:	46bb      	mov	fp, r7
 800183e:	46b2      	mov	sl, r6
 8001840:	46a9      	mov	r9, r5
 8001842:	46a0      	mov	r8, r4
 8001844:	bdf0      	pop	{r4, r5, r6, r7, pc}
 8001846:	0033      	movs	r3, r6
 8001848:	2001      	movs	r0, #1
 800184a:	432b      	orrs	r3, r5
 800184c:	d1f5      	bne.n	800183a <__eqdf2+0x5a>
 800184e:	42a2      	cmp	r2, r4
 8001850:	d1f3      	bne.n	800183a <__eqdf2+0x5a>
 8001852:	464b      	mov	r3, r9
 8001854:	433b      	orrs	r3, r7
 8001856:	d1f0      	bne.n	800183a <__eqdf2+0x5a>
 8001858:	e7e2      	b.n	8001820 <__eqdf2+0x40>
 800185a:	2000      	movs	r0, #0
 800185c:	e7ed      	b.n	800183a <__eqdf2+0x5a>
 800185e:	46c0      	nop			; (mov r8, r8)
 8001860:	000007ff 	.word	0x000007ff

08001864 <__gedf2>:
 8001864:	b5f0      	push	{r4, r5, r6, r7, lr}
 8001866:	4647      	mov	r7, r8
 8001868:	46ce      	mov	lr, r9
 800186a:	0004      	movs	r4, r0
 800186c:	0018      	movs	r0, r3
 800186e:	0016      	movs	r6, r2
 8001870:	031b      	lsls	r3, r3, #12
 8001872:	0b1b      	lsrs	r3, r3, #12
 8001874:	4d2d      	ldr	r5, [pc, #180]	; (800192c <__gedf2+0xc8>)
 8001876:	004a      	lsls	r2, r1, #1
 8001878:	4699      	mov	r9, r3
 800187a:	b580      	push	{r7, lr}
 800187c:	0043      	lsls	r3, r0, #1
 800187e:	030f      	lsls	r7, r1, #12
 8001880:	46a4      	mov	ip, r4
 8001882:	46b0      	mov	r8, r6
 8001884:	0b3f      	lsrs	r7, r7, #12
 8001886:	0d52      	lsrs	r2, r2, #21
 8001888:	0fc9      	lsrs	r1, r1, #31
 800188a:	0d5b      	lsrs	r3, r3, #21
 800188c:	0fc0      	lsrs	r0, r0, #31
 800188e:	42aa      	cmp	r2, r5
 8001890:	d021      	beq.n	80018d6 <__gedf2+0x72>
 8001892:	42ab      	cmp	r3, r5
 8001894:	d013      	beq.n	80018be <__gedf2+0x5a>
 8001896:	2a00      	cmp	r2, #0
 8001898:	d122      	bne.n	80018e0 <__gedf2+0x7c>
 800189a:	433c      	orrs	r4, r7
 800189c:	2b00      	cmp	r3, #0
 800189e:	d102      	bne.n	80018a6 <__gedf2+0x42>
 80018a0:	464d      	mov	r5, r9
 80018a2:	432e      	orrs	r6, r5
 80018a4:	d022      	beq.n	80018ec <__gedf2+0x88>
 80018a6:	2c00      	cmp	r4, #0
 80018a8:	d010      	beq.n	80018cc <__gedf2+0x68>
 80018aa:	4281      	cmp	r1, r0
 80018ac:	d022      	beq.n	80018f4 <__gedf2+0x90>
 80018ae:	2002      	movs	r0, #2
 80018b0:	3901      	subs	r1, #1
 80018b2:	4008      	ands	r0, r1
 80018b4:	3801      	subs	r0, #1
 80018b6:	bcc0      	pop	{r6, r7}
 80018b8:	46b9      	mov	r9, r7
 80018ba:	46b0      	mov	r8, r6
 80018bc:	bdf0      	pop	{r4, r5, r6, r7, pc}
 80018be:	464d      	mov	r5, r9
 80018c0:	432e      	orrs	r6, r5
 80018c2:	d129      	bne.n	8001918 <__gedf2+0xb4>
 80018c4:	2a00      	cmp	r2, #0
 80018c6:	d1f0      	bne.n	80018aa <__gedf2+0x46>
 80018c8:	433c      	orrs	r4, r7
 80018ca:	d1ee      	bne.n	80018aa <__gedf2+0x46>
 80018cc:	2800      	cmp	r0, #0
 80018ce:	d1f2      	bne.n	80018b6 <__gedf2+0x52>
 80018d0:	2001      	movs	r0, #1
 80018d2:	4240      	negs	r0, r0
 80018d4:	e7ef      	b.n	80018b6 <__gedf2+0x52>
 80018d6:	003d      	movs	r5, r7
 80018d8:	4325      	orrs	r5, r4
 80018da:	d11d      	bne.n	8001918 <__gedf2+0xb4>
 80018dc:	4293      	cmp	r3, r2
 80018de:	d0ee      	beq.n	80018be <__gedf2+0x5a>
 80018e0:	2b00      	cmp	r3, #0
 80018e2:	d1e2      	bne.n	80018aa <__gedf2+0x46>
 80018e4:	464c      	mov	r4, r9
 80018e6:	4326      	orrs	r6, r4
 80018e8:	d1df      	bne.n	80018aa <__gedf2+0x46>
 80018ea:	e7e0      	b.n	80018ae <__gedf2+0x4a>
 80018ec:	2000      	movs	r0, #0
 80018ee:	2c00      	cmp	r4, #0
 80018f0:	d0e1      	beq.n	80018b6 <__gedf2+0x52>
 80018f2:	e7dc      	b.n	80018ae <__gedf2+0x4a>
 80018f4:	429a      	cmp	r2, r3
 80018f6:	dc0a      	bgt.n	800190e <__gedf2+0xaa>
 80018f8:	dbe8      	blt.n	80018cc <__gedf2+0x68>
 80018fa:	454f      	cmp	r7, r9
 80018fc:	d8d7      	bhi.n	80018ae <__gedf2+0x4a>
 80018fe:	d00e      	beq.n	800191e <__gedf2+0xba>
 8001900:	2000      	movs	r0, #0
 8001902:	454f      	cmp	r7, r9
 8001904:	d2d7      	bcs.n	80018b6 <__gedf2+0x52>
 8001906:	2900      	cmp	r1, #0
 8001908:	d0e2      	beq.n	80018d0 <__gedf2+0x6c>
 800190a:	0008      	movs	r0, r1
 800190c:	e7d3      	b.n	80018b6 <__gedf2+0x52>
 800190e:	4243      	negs	r3, r0
 8001910:	4158      	adcs	r0, r3
 8001912:	0040      	lsls	r0, r0, #1
 8001914:	3801      	subs	r0, #1
 8001916:	e7ce      	b.n	80018b6 <__gedf2+0x52>
 8001918:	2002      	movs	r0, #2
 800191a:	4240      	negs	r0, r0
 800191c:	e7cb      	b.n	80018b6 <__gedf2+0x52>
 800191e:	45c4      	cmp	ip, r8
 8001920:	d8c5      	bhi.n	80018ae <__gedf2+0x4a>
 8001922:	2000      	movs	r0, #0
 8001924:	45c4      	cmp	ip, r8
 8001926:	d2c6      	bcs.n	80018b6 <__gedf2+0x52>
 8001928:	e7ed      	b.n	8001906 <__gedf2+0xa2>
 800192a:	46c0      	nop			; (mov r8, r8)
 800192c:	000007ff 	.word	0x000007ff

08001930 <__ledf2>:
 8001930:	b5f0      	push	{r4, r5, r6, r7, lr}
 8001932:	4647      	mov	r7, r8
 8001934:	46ce      	mov	lr, r9
 8001936:	0004      	movs	r4, r0
 8001938:	0018      	movs	r0, r3
 800193a:	0016      	movs	r6, r2
 800193c:	031b      	lsls	r3, r3, #12
 800193e:	0b1b      	lsrs	r3, r3, #12
 8001940:	4d2c      	ldr	r5, [pc, #176]	; (80019f4 <__ledf2+0xc4>)
 8001942:	004a      	lsls	r2, r1, #1
 8001944:	4699      	mov	r9, r3
 8001946:	b580      	push	{r7, lr}
 8001948:	0043      	lsls	r3, r0, #1
 800194a:	030f      	lsls	r7, r1, #12
 800194c:	46a4      	mov	ip, r4
 800194e:	46b0      	mov	r8, r6
 8001950:	0b3f      	lsrs	r7, r7, #12
 8001952:	0d52      	lsrs	r2, r2, #21
 8001954:	0fc9      	lsrs	r1, r1, #31
 8001956:	0d5b      	lsrs	r3, r3, #21
 8001958:	0fc0      	lsrs	r0, r0, #31
 800195a:	42aa      	cmp	r2, r5
 800195c:	d00d      	beq.n	800197a <__ledf2+0x4a>
 800195e:	42ab      	cmp	r3, r5
 8001960:	d010      	beq.n	8001984 <__ledf2+0x54>
 8001962:	2a00      	cmp	r2, #0
 8001964:	d127      	bne.n	80019b6 <__ledf2+0x86>
 8001966:	433c      	orrs	r4, r7
 8001968:	2b00      	cmp	r3, #0
 800196a:	d111      	bne.n	8001990 <__ledf2+0x60>
 800196c:	464d      	mov	r5, r9
 800196e:	432e      	orrs	r6, r5
 8001970:	d10e      	bne.n	8001990 <__ledf2+0x60>
 8001972:	2000      	movs	r0, #0
 8001974:	2c00      	cmp	r4, #0
 8001976:	d015      	beq.n	80019a4 <__ledf2+0x74>
 8001978:	e00e      	b.n	8001998 <__ledf2+0x68>
 800197a:	003d      	movs	r5, r7
 800197c:	4325      	orrs	r5, r4
 800197e:	d110      	bne.n	80019a2 <__ledf2+0x72>
 8001980:	4293      	cmp	r3, r2
 8001982:	d118      	bne.n	80019b6 <__ledf2+0x86>
 8001984:	464d      	mov	r5, r9
 8001986:	432e      	orrs	r6, r5
 8001988:	d10b      	bne.n	80019a2 <__ledf2+0x72>
 800198a:	2a00      	cmp	r2, #0
 800198c:	d102      	bne.n	8001994 <__ledf2+0x64>
 800198e:	433c      	orrs	r4, r7
 8001990:	2c00      	cmp	r4, #0
 8001992:	d00b      	beq.n	80019ac <__ledf2+0x7c>
 8001994:	4281      	cmp	r1, r0
 8001996:	d014      	beq.n	80019c2 <__ledf2+0x92>
 8001998:	2002      	movs	r0, #2
 800199a:	3901      	subs	r1, #1
 800199c:	4008      	ands	r0, r1
 800199e:	3801      	subs	r0, #1
 80019a0:	e000      	b.n	80019a4 <__ledf2+0x74>
 80019a2:	2002      	movs	r0, #2
 80019a4:	bcc0      	pop	{r6, r7}
 80019a6:	46b9      	mov	r9, r7
 80019a8:	46b0      	mov	r8, r6
 80019aa:	bdf0      	pop	{r4, r5, r6, r7, pc}
 80019ac:	2800      	cmp	r0, #0
 80019ae:	d1f9      	bne.n	80019a4 <__ledf2+0x74>
 80019b0:	2001      	movs	r0, #1
 80019b2:	4240      	negs	r0, r0
 80019b4:	e7f6      	b.n	80019a4 <__ledf2+0x74>
 80019b6:	2b00      	cmp	r3, #0
 80019b8:	d1ec      	bne.n	8001994 <__ledf2+0x64>
 80019ba:	464c      	mov	r4, r9
 80019bc:	4326      	orrs	r6, r4
 80019be:	d1e9      	bne.n	8001994 <__ledf2+0x64>
 80019c0:	e7ea      	b.n	8001998 <__ledf2+0x68>
 80019c2:	429a      	cmp	r2, r3
 80019c4:	dd04      	ble.n	80019d0 <__ledf2+0xa0>
 80019c6:	4243      	negs	r3, r0
 80019c8:	4158      	adcs	r0, r3
 80019ca:	0040      	lsls	r0, r0, #1
 80019cc:	3801      	subs	r0, #1
 80019ce:	e7e9      	b.n	80019a4 <__ledf2+0x74>
 80019d0:	429a      	cmp	r2, r3
 80019d2:	dbeb      	blt.n	80019ac <__ledf2+0x7c>
 80019d4:	454f      	cmp	r7, r9
 80019d6:	d8df      	bhi.n	8001998 <__ledf2+0x68>
 80019d8:	d006      	beq.n	80019e8 <__ledf2+0xb8>
 80019da:	2000      	movs	r0, #0
 80019dc:	454f      	cmp	r7, r9
 80019de:	d2e1      	bcs.n	80019a4 <__ledf2+0x74>
 80019e0:	2900      	cmp	r1, #0
 80019e2:	d0e5      	beq.n	80019b0 <__ledf2+0x80>
 80019e4:	0008      	movs	r0, r1
 80019e6:	e7dd      	b.n	80019a4 <__ledf2+0x74>
 80019e8:	45c4      	cmp	ip, r8
 80019ea:	d8d5      	bhi.n	8001998 <__ledf2+0x68>
 80019ec:	2000      	movs	r0, #0
 80019ee:	45c4      	cmp	ip, r8
 80019f0:	d2d8      	bcs.n	80019a4 <__ledf2+0x74>
 80019f2:	e7f5      	b.n	80019e0 <__ledf2+0xb0>
 80019f4:	000007ff 	.word	0x000007ff

080019f8 <__aeabi_dmul>:
 80019f8:	b5f0      	push	{r4, r5, r6, r7, lr}
 80019fa:	4657      	mov	r7, sl
 80019fc:	464e      	mov	r6, r9
 80019fe:	4645      	mov	r5, r8
 8001a00:	46de      	mov	lr, fp
 8001a02:	b5e0      	push	{r5, r6, r7, lr}
 8001a04:	4698      	mov	r8, r3
 8001a06:	030c      	lsls	r4, r1, #12
 8001a08:	004b      	lsls	r3, r1, #1
 8001a0a:	0006      	movs	r6, r0
 8001a0c:	4692      	mov	sl, r2
 8001a0e:	b087      	sub	sp, #28
 8001a10:	0b24      	lsrs	r4, r4, #12
 8001a12:	0d5b      	lsrs	r3, r3, #21
 8001a14:	0fcf      	lsrs	r7, r1, #31
 8001a16:	2b00      	cmp	r3, #0
 8001a18:	d100      	bne.n	8001a1c <__aeabi_dmul+0x24>
 8001a1a:	e15c      	b.n	8001cd6 <__aeabi_dmul+0x2de>
 8001a1c:	4ad9      	ldr	r2, [pc, #868]	; (8001d84 <__aeabi_dmul+0x38c>)
 8001a1e:	4293      	cmp	r3, r2
 8001a20:	d100      	bne.n	8001a24 <__aeabi_dmul+0x2c>
 8001a22:	e175      	b.n	8001d10 <__aeabi_dmul+0x318>
 8001a24:	0f42      	lsrs	r2, r0, #29
 8001a26:	00e4      	lsls	r4, r4, #3
 8001a28:	4314      	orrs	r4, r2
 8001a2a:	2280      	movs	r2, #128	; 0x80
 8001a2c:	0412      	lsls	r2, r2, #16
 8001a2e:	4314      	orrs	r4, r2
 8001a30:	4ad5      	ldr	r2, [pc, #852]	; (8001d88 <__aeabi_dmul+0x390>)
 8001a32:	00c5      	lsls	r5, r0, #3
 8001a34:	4694      	mov	ip, r2
 8001a36:	4463      	add	r3, ip
 8001a38:	9300      	str	r3, [sp, #0]
 8001a3a:	2300      	movs	r3, #0
 8001a3c:	4699      	mov	r9, r3
 8001a3e:	469b      	mov	fp, r3
 8001a40:	4643      	mov	r3, r8
 8001a42:	4642      	mov	r2, r8
 8001a44:	031e      	lsls	r6, r3, #12
 8001a46:	0fd2      	lsrs	r2, r2, #31
 8001a48:	005b      	lsls	r3, r3, #1
 8001a4a:	4650      	mov	r0, sl
 8001a4c:	4690      	mov	r8, r2
 8001a4e:	0b36      	lsrs	r6, r6, #12
 8001a50:	0d5b      	lsrs	r3, r3, #21
 8001a52:	d100      	bne.n	8001a56 <__aeabi_dmul+0x5e>
 8001a54:	e120      	b.n	8001c98 <__aeabi_dmul+0x2a0>
 8001a56:	4acb      	ldr	r2, [pc, #812]	; (8001d84 <__aeabi_dmul+0x38c>)
 8001a58:	4293      	cmp	r3, r2
 8001a5a:	d100      	bne.n	8001a5e <__aeabi_dmul+0x66>
 8001a5c:	e162      	b.n	8001d24 <__aeabi_dmul+0x32c>
 8001a5e:	49ca      	ldr	r1, [pc, #808]	; (8001d88 <__aeabi_dmul+0x390>)
 8001a60:	0f42      	lsrs	r2, r0, #29
 8001a62:	468c      	mov	ip, r1
 8001a64:	9900      	ldr	r1, [sp, #0]
 8001a66:	4463      	add	r3, ip
 8001a68:	00f6      	lsls	r6, r6, #3
 8001a6a:	468c      	mov	ip, r1
 8001a6c:	4316      	orrs	r6, r2
 8001a6e:	2280      	movs	r2, #128	; 0x80
 8001a70:	449c      	add	ip, r3
 8001a72:	0412      	lsls	r2, r2, #16
 8001a74:	4663      	mov	r3, ip
 8001a76:	4316      	orrs	r6, r2
 8001a78:	00c2      	lsls	r2, r0, #3
 8001a7a:	2000      	movs	r0, #0
 8001a7c:	9300      	str	r3, [sp, #0]
 8001a7e:	9900      	ldr	r1, [sp, #0]
 8001a80:	4643      	mov	r3, r8
 8001a82:	3101      	adds	r1, #1
 8001a84:	468c      	mov	ip, r1
 8001a86:	4649      	mov	r1, r9
 8001a88:	407b      	eors	r3, r7
 8001a8a:	9301      	str	r3, [sp, #4]
 8001a8c:	290f      	cmp	r1, #15
 8001a8e:	d826      	bhi.n	8001ade <__aeabi_dmul+0xe6>
 8001a90:	4bbe      	ldr	r3, [pc, #760]	; (8001d8c <__aeabi_dmul+0x394>)
 8001a92:	0089      	lsls	r1, r1, #2
 8001a94:	5859      	ldr	r1, [r3, r1]
 8001a96:	468f      	mov	pc, r1
 8001a98:	4643      	mov	r3, r8
 8001a9a:	9301      	str	r3, [sp, #4]
 8001a9c:	0034      	movs	r4, r6
 8001a9e:	0015      	movs	r5, r2
 8001aa0:	4683      	mov	fp, r0
 8001aa2:	465b      	mov	r3, fp
 8001aa4:	2b02      	cmp	r3, #2
 8001aa6:	d016      	beq.n	8001ad6 <__aeabi_dmul+0xde>
 8001aa8:	2b03      	cmp	r3, #3
 8001aaa:	d100      	bne.n	8001aae <__aeabi_dmul+0xb6>
 8001aac:	e203      	b.n	8001eb6 <__aeabi_dmul+0x4be>
 8001aae:	2b01      	cmp	r3, #1
 8001ab0:	d000      	beq.n	8001ab4 <__aeabi_dmul+0xbc>
 8001ab2:	e0cd      	b.n	8001c50 <__aeabi_dmul+0x258>
 8001ab4:	2200      	movs	r2, #0
 8001ab6:	2400      	movs	r4, #0
 8001ab8:	2500      	movs	r5, #0
 8001aba:	9b01      	ldr	r3, [sp, #4]
 8001abc:	0512      	lsls	r2, r2, #20
 8001abe:	4322      	orrs	r2, r4
 8001ac0:	07db      	lsls	r3, r3, #31
 8001ac2:	431a      	orrs	r2, r3
 8001ac4:	0028      	movs	r0, r5
 8001ac6:	0011      	movs	r1, r2
 8001ac8:	b007      	add	sp, #28
 8001aca:	bcf0      	pop	{r4, r5, r6, r7}
 8001acc:	46bb      	mov	fp, r7
 8001ace:	46b2      	mov	sl, r6
 8001ad0:	46a9      	mov	r9, r5
 8001ad2:	46a0      	mov	r8, r4
 8001ad4:	bdf0      	pop	{r4, r5, r6, r7, pc}
 8001ad6:	2400      	movs	r4, #0
 8001ad8:	2500      	movs	r5, #0
 8001ada:	4aaa      	ldr	r2, [pc, #680]	; (8001d84 <__aeabi_dmul+0x38c>)
 8001adc:	e7ed      	b.n	8001aba <__aeabi_dmul+0xc2>
 8001ade:	0c28      	lsrs	r0, r5, #16
 8001ae0:	042d      	lsls	r5, r5, #16
 8001ae2:	0c2d      	lsrs	r5, r5, #16
 8001ae4:	002b      	movs	r3, r5
 8001ae6:	0c11      	lsrs	r1, r2, #16
 8001ae8:	0412      	lsls	r2, r2, #16
 8001aea:	0c12      	lsrs	r2, r2, #16
 8001aec:	4353      	muls	r3, r2
 8001aee:	4698      	mov	r8, r3
 8001af0:	0013      	movs	r3, r2
 8001af2:	002f      	movs	r7, r5
 8001af4:	4343      	muls	r3, r0
 8001af6:	4699      	mov	r9, r3
 8001af8:	434f      	muls	r7, r1
 8001afa:	444f      	add	r7, r9
 8001afc:	46bb      	mov	fp, r7
 8001afe:	4647      	mov	r7, r8
 8001b00:	000b      	movs	r3, r1
 8001b02:	0c3f      	lsrs	r7, r7, #16
 8001b04:	46ba      	mov	sl, r7
 8001b06:	4343      	muls	r3, r0
 8001b08:	44da      	add	sl, fp
 8001b0a:	9302      	str	r3, [sp, #8]
 8001b0c:	45d1      	cmp	r9, sl
 8001b0e:	d904      	bls.n	8001b1a <__aeabi_dmul+0x122>
 8001b10:	2780      	movs	r7, #128	; 0x80
 8001b12:	027f      	lsls	r7, r7, #9
 8001b14:	46b9      	mov	r9, r7
 8001b16:	444b      	add	r3, r9
 8001b18:	9302      	str	r3, [sp, #8]
 8001b1a:	4653      	mov	r3, sl
 8001b1c:	0c1b      	lsrs	r3, r3, #16
 8001b1e:	469b      	mov	fp, r3
 8001b20:	4653      	mov	r3, sl
 8001b22:	041f      	lsls	r7, r3, #16
 8001b24:	4643      	mov	r3, r8
 8001b26:	041b      	lsls	r3, r3, #16
 8001b28:	0c1b      	lsrs	r3, r3, #16
 8001b2a:	4698      	mov	r8, r3
 8001b2c:	003b      	movs	r3, r7
 8001b2e:	4443      	add	r3, r8
 8001b30:	9304      	str	r3, [sp, #16]
 8001b32:	0c33      	lsrs	r3, r6, #16
 8001b34:	0436      	lsls	r6, r6, #16
 8001b36:	0c36      	lsrs	r6, r6, #16
 8001b38:	4698      	mov	r8, r3
 8001b3a:	0033      	movs	r3, r6
 8001b3c:	4343      	muls	r3, r0
 8001b3e:	4699      	mov	r9, r3
 8001b40:	4643      	mov	r3, r8
 8001b42:	4343      	muls	r3, r0
 8001b44:	002f      	movs	r7, r5
 8001b46:	469a      	mov	sl, r3
 8001b48:	4643      	mov	r3, r8
 8001b4a:	4377      	muls	r7, r6
 8001b4c:	435d      	muls	r5, r3
 8001b4e:	0c38      	lsrs	r0, r7, #16
 8001b50:	444d      	add	r5, r9
 8001b52:	1945      	adds	r5, r0, r5
 8001b54:	45a9      	cmp	r9, r5
 8001b56:	d903      	bls.n	8001b60 <__aeabi_dmul+0x168>
 8001b58:	2380      	movs	r3, #128	; 0x80
 8001b5a:	025b      	lsls	r3, r3, #9
 8001b5c:	4699      	mov	r9, r3
 8001b5e:	44ca      	add	sl, r9
 8001b60:	043f      	lsls	r7, r7, #16
 8001b62:	0c28      	lsrs	r0, r5, #16
 8001b64:	0c3f      	lsrs	r7, r7, #16
 8001b66:	042d      	lsls	r5, r5, #16
 8001b68:	19ed      	adds	r5, r5, r7
 8001b6a:	0c27      	lsrs	r7, r4, #16
 8001b6c:	0424      	lsls	r4, r4, #16
 8001b6e:	0c24      	lsrs	r4, r4, #16
 8001b70:	0003      	movs	r3, r0
 8001b72:	0020      	movs	r0, r4
 8001b74:	4350      	muls	r0, r2
 8001b76:	437a      	muls	r2, r7
 8001b78:	4691      	mov	r9, r2
 8001b7a:	003a      	movs	r2, r7
 8001b7c:	4453      	add	r3, sl
 8001b7e:	9305      	str	r3, [sp, #20]
 8001b80:	0c03      	lsrs	r3, r0, #16
 8001b82:	469a      	mov	sl, r3
 8001b84:	434a      	muls	r2, r1
 8001b86:	4361      	muls	r1, r4
 8001b88:	4449      	add	r1, r9
 8001b8a:	4451      	add	r1, sl
 8001b8c:	44ab      	add	fp, r5
 8001b8e:	4589      	cmp	r9, r1
 8001b90:	d903      	bls.n	8001b9a <__aeabi_dmul+0x1a2>
 8001b92:	2380      	movs	r3, #128	; 0x80
 8001b94:	025b      	lsls	r3, r3, #9
 8001b96:	4699      	mov	r9, r3
 8001b98:	444a      	add	r2, r9
 8001b9a:	0400      	lsls	r0, r0, #16
 8001b9c:	0c0b      	lsrs	r3, r1, #16
 8001b9e:	0c00      	lsrs	r0, r0, #16
 8001ba0:	0409      	lsls	r1, r1, #16
 8001ba2:	1809      	adds	r1, r1, r0
 8001ba4:	0020      	movs	r0, r4
 8001ba6:	4699      	mov	r9, r3
 8001ba8:	4643      	mov	r3, r8
 8001baa:	4370      	muls	r0, r6
 8001bac:	435c      	muls	r4, r3
 8001bae:	437e      	muls	r6, r7
 8001bb0:	435f      	muls	r7, r3
 8001bb2:	0c03      	lsrs	r3, r0, #16
 8001bb4:	4698      	mov	r8, r3
 8001bb6:	19a4      	adds	r4, r4, r6
 8001bb8:	4444      	add	r4, r8
 8001bba:	444a      	add	r2, r9
 8001bbc:	9703      	str	r7, [sp, #12]
 8001bbe:	42a6      	cmp	r6, r4
 8001bc0:	d904      	bls.n	8001bcc <__aeabi_dmul+0x1d4>
 8001bc2:	2380      	movs	r3, #128	; 0x80
 8001bc4:	025b      	lsls	r3, r3, #9
 8001bc6:	4698      	mov	r8, r3
 8001bc8:	4447      	add	r7, r8
 8001bca:	9703      	str	r7, [sp, #12]
 8001bcc:	0423      	lsls	r3, r4, #16
 8001bce:	9e02      	ldr	r6, [sp, #8]
 8001bd0:	469a      	mov	sl, r3
 8001bd2:	9b05      	ldr	r3, [sp, #20]
 8001bd4:	445e      	add	r6, fp
 8001bd6:	4698      	mov	r8, r3
 8001bd8:	42ae      	cmp	r6, r5
 8001bda:	41ad      	sbcs	r5, r5
 8001bdc:	1876      	adds	r6, r6, r1
 8001bde:	428e      	cmp	r6, r1
 8001be0:	4189      	sbcs	r1, r1
 8001be2:	0400      	lsls	r0, r0, #16
 8001be4:	0c00      	lsrs	r0, r0, #16
 8001be6:	4450      	add	r0, sl
 8001be8:	4440      	add	r0, r8
 8001bea:	426d      	negs	r5, r5
 8001bec:	1947      	adds	r7, r0, r5
 8001bee:	46b8      	mov	r8, r7
 8001bf0:	4693      	mov	fp, r2
 8001bf2:	4249      	negs	r1, r1
 8001bf4:	4689      	mov	r9, r1
 8001bf6:	44c3      	add	fp, r8
 8001bf8:	44d9      	add	r9, fp
 8001bfa:	4298      	cmp	r0, r3
 8001bfc:	4180      	sbcs	r0, r0
 8001bfe:	45a8      	cmp	r8, r5
 8001c00:	41ad      	sbcs	r5, r5
 8001c02:	4593      	cmp	fp, r2
 8001c04:	4192      	sbcs	r2, r2
 8001c06:	4589      	cmp	r9, r1
 8001c08:	4189      	sbcs	r1, r1
 8001c0a:	426d      	negs	r5, r5
 8001c0c:	4240      	negs	r0, r0
 8001c0e:	4328      	orrs	r0, r5
 8001c10:	0c24      	lsrs	r4, r4, #16
 8001c12:	4252      	negs	r2, r2
 8001c14:	4249      	negs	r1, r1
 8001c16:	430a      	orrs	r2, r1
 8001c18:	9b03      	ldr	r3, [sp, #12]
 8001c1a:	1900      	adds	r0, r0, r4
 8001c1c:	1880      	adds	r0, r0, r2
 8001c1e:	18c7      	adds	r7, r0, r3
 8001c20:	464b      	mov	r3, r9
 8001c22:	0ddc      	lsrs	r4, r3, #23
 8001c24:	9b04      	ldr	r3, [sp, #16]
 8001c26:	0275      	lsls	r5, r6, #9
 8001c28:	431d      	orrs	r5, r3
 8001c2a:	1e6a      	subs	r2, r5, #1
 8001c2c:	4195      	sbcs	r5, r2
 8001c2e:	464b      	mov	r3, r9
 8001c30:	0df6      	lsrs	r6, r6, #23
 8001c32:	027f      	lsls	r7, r7, #9
 8001c34:	4335      	orrs	r5, r6
 8001c36:	025a      	lsls	r2, r3, #9
 8001c38:	433c      	orrs	r4, r7
 8001c3a:	4315      	orrs	r5, r2
 8001c3c:	01fb      	lsls	r3, r7, #7
 8001c3e:	d400      	bmi.n	8001c42 <__aeabi_dmul+0x24a>
 8001c40:	e11c      	b.n	8001e7c <__aeabi_dmul+0x484>
 8001c42:	2101      	movs	r1, #1
 8001c44:	086a      	lsrs	r2, r5, #1
 8001c46:	400d      	ands	r5, r1
 8001c48:	4315      	orrs	r5, r2
 8001c4a:	07e2      	lsls	r2, r4, #31
 8001c4c:	4315      	orrs	r5, r2
 8001c4e:	0864      	lsrs	r4, r4, #1
 8001c50:	494f      	ldr	r1, [pc, #316]	; (8001d90 <__aeabi_dmul+0x398>)
 8001c52:	4461      	add	r1, ip
 8001c54:	2900      	cmp	r1, #0
 8001c56:	dc00      	bgt.n	8001c5a <__aeabi_dmul+0x262>
 8001c58:	e0b0      	b.n	8001dbc <__aeabi_dmul+0x3c4>
 8001c5a:	076b      	lsls	r3, r5, #29
 8001c5c:	d009      	beq.n	8001c72 <__aeabi_dmul+0x27a>
 8001c5e:	220f      	movs	r2, #15
 8001c60:	402a      	ands	r2, r5
 8001c62:	2a04      	cmp	r2, #4
 8001c64:	d005      	beq.n	8001c72 <__aeabi_dmul+0x27a>
 8001c66:	1d2a      	adds	r2, r5, #4
 8001c68:	42aa      	cmp	r2, r5
 8001c6a:	41ad      	sbcs	r5, r5
 8001c6c:	426d      	negs	r5, r5
 8001c6e:	1964      	adds	r4, r4, r5
 8001c70:	0015      	movs	r5, r2
 8001c72:	01e3      	lsls	r3, r4, #7
 8001c74:	d504      	bpl.n	8001c80 <__aeabi_dmul+0x288>
 8001c76:	2180      	movs	r1, #128	; 0x80
 8001c78:	4a46      	ldr	r2, [pc, #280]	; (8001d94 <__aeabi_dmul+0x39c>)
 8001c7a:	00c9      	lsls	r1, r1, #3
 8001c7c:	4014      	ands	r4, r2
 8001c7e:	4461      	add	r1, ip
 8001c80:	4a45      	ldr	r2, [pc, #276]	; (8001d98 <__aeabi_dmul+0x3a0>)
 8001c82:	4291      	cmp	r1, r2
 8001c84:	dd00      	ble.n	8001c88 <__aeabi_dmul+0x290>
 8001c86:	e726      	b.n	8001ad6 <__aeabi_dmul+0xde>
 8001c88:	0762      	lsls	r2, r4, #29
 8001c8a:	08ed      	lsrs	r5, r5, #3
 8001c8c:	0264      	lsls	r4, r4, #9
 8001c8e:	0549      	lsls	r1, r1, #21
 8001c90:	4315      	orrs	r5, r2
 8001c92:	0b24      	lsrs	r4, r4, #12
 8001c94:	0d4a      	lsrs	r2, r1, #21
 8001c96:	e710      	b.n	8001aba <__aeabi_dmul+0xc2>
 8001c98:	4652      	mov	r2, sl
 8001c9a:	4332      	orrs	r2, r6
 8001c9c:	d100      	bne.n	8001ca0 <__aeabi_dmul+0x2a8>
 8001c9e:	e07f      	b.n	8001da0 <__aeabi_dmul+0x3a8>
 8001ca0:	2e00      	cmp	r6, #0
 8001ca2:	d100      	bne.n	8001ca6 <__aeabi_dmul+0x2ae>
 8001ca4:	e0dc      	b.n	8001e60 <__aeabi_dmul+0x468>
 8001ca6:	0030      	movs	r0, r6
 8001ca8:	f000 fe1e 	bl	80028e8 <__clzsi2>
 8001cac:	0002      	movs	r2, r0
 8001cae:	3a0b      	subs	r2, #11
 8001cb0:	231d      	movs	r3, #29
 8001cb2:	0001      	movs	r1, r0
 8001cb4:	1a9b      	subs	r3, r3, r2
 8001cb6:	4652      	mov	r2, sl
 8001cb8:	3908      	subs	r1, #8
 8001cba:	40da      	lsrs	r2, r3
 8001cbc:	408e      	lsls	r6, r1
 8001cbe:	4316      	orrs	r6, r2
 8001cc0:	4652      	mov	r2, sl
 8001cc2:	408a      	lsls	r2, r1
 8001cc4:	9b00      	ldr	r3, [sp, #0]
 8001cc6:	4935      	ldr	r1, [pc, #212]	; (8001d9c <__aeabi_dmul+0x3a4>)
 8001cc8:	1a18      	subs	r0, r3, r0
 8001cca:	0003      	movs	r3, r0
 8001ccc:	468c      	mov	ip, r1
 8001cce:	4463      	add	r3, ip
 8001cd0:	2000      	movs	r0, #0
 8001cd2:	9300      	str	r3, [sp, #0]
 8001cd4:	e6d3      	b.n	8001a7e <__aeabi_dmul+0x86>
 8001cd6:	0025      	movs	r5, r4
 8001cd8:	4305      	orrs	r5, r0
 8001cda:	d04a      	beq.n	8001d72 <__aeabi_dmul+0x37a>
 8001cdc:	2c00      	cmp	r4, #0
 8001cde:	d100      	bne.n	8001ce2 <__aeabi_dmul+0x2ea>
 8001ce0:	e0b0      	b.n	8001e44 <__aeabi_dmul+0x44c>
 8001ce2:	0020      	movs	r0, r4
 8001ce4:	f000 fe00 	bl	80028e8 <__clzsi2>
 8001ce8:	0001      	movs	r1, r0
 8001cea:	0002      	movs	r2, r0
 8001cec:	390b      	subs	r1, #11
 8001cee:	231d      	movs	r3, #29
 8001cf0:	0010      	movs	r0, r2
 8001cf2:	1a5b      	subs	r3, r3, r1
 8001cf4:	0031      	movs	r1, r6
 8001cf6:	0035      	movs	r5, r6
 8001cf8:	3808      	subs	r0, #8
 8001cfa:	4084      	lsls	r4, r0
 8001cfc:	40d9      	lsrs	r1, r3
 8001cfe:	4085      	lsls	r5, r0
 8001d00:	430c      	orrs	r4, r1
 8001d02:	4826      	ldr	r0, [pc, #152]	; (8001d9c <__aeabi_dmul+0x3a4>)
 8001d04:	1a83      	subs	r3, r0, r2
 8001d06:	9300      	str	r3, [sp, #0]
 8001d08:	2300      	movs	r3, #0
 8001d0a:	4699      	mov	r9, r3
 8001d0c:	469b      	mov	fp, r3
 8001d0e:	e697      	b.n	8001a40 <__aeabi_dmul+0x48>
 8001d10:	0005      	movs	r5, r0
 8001d12:	4325      	orrs	r5, r4
 8001d14:	d126      	bne.n	8001d64 <__aeabi_dmul+0x36c>
 8001d16:	2208      	movs	r2, #8
 8001d18:	9300      	str	r3, [sp, #0]
 8001d1a:	2302      	movs	r3, #2
 8001d1c:	2400      	movs	r4, #0
 8001d1e:	4691      	mov	r9, r2
 8001d20:	469b      	mov	fp, r3
 8001d22:	e68d      	b.n	8001a40 <__aeabi_dmul+0x48>
 8001d24:	4652      	mov	r2, sl
 8001d26:	9b00      	ldr	r3, [sp, #0]
 8001d28:	4332      	orrs	r2, r6
 8001d2a:	d110      	bne.n	8001d4e <__aeabi_dmul+0x356>
 8001d2c:	4915      	ldr	r1, [pc, #84]	; (8001d84 <__aeabi_dmul+0x38c>)
 8001d2e:	2600      	movs	r6, #0
 8001d30:	468c      	mov	ip, r1
 8001d32:	4463      	add	r3, ip
 8001d34:	4649      	mov	r1, r9
 8001d36:	9300      	str	r3, [sp, #0]
 8001d38:	2302      	movs	r3, #2
 8001d3a:	4319      	orrs	r1, r3
 8001d3c:	4689      	mov	r9, r1
 8001d3e:	2002      	movs	r0, #2
 8001d40:	e69d      	b.n	8001a7e <__aeabi_dmul+0x86>
 8001d42:	465b      	mov	r3, fp
 8001d44:	9701      	str	r7, [sp, #4]
 8001d46:	2b02      	cmp	r3, #2
 8001d48:	d000      	beq.n	8001d4c <__aeabi_dmul+0x354>
 8001d4a:	e6ad      	b.n	8001aa8 <__aeabi_dmul+0xb0>
 8001d4c:	e6c3      	b.n	8001ad6 <__aeabi_dmul+0xde>
 8001d4e:	4a0d      	ldr	r2, [pc, #52]	; (8001d84 <__aeabi_dmul+0x38c>)
 8001d50:	2003      	movs	r0, #3
 8001d52:	4694      	mov	ip, r2
 8001d54:	4463      	add	r3, ip
 8001d56:	464a      	mov	r2, r9
 8001d58:	9300      	str	r3, [sp, #0]
 8001d5a:	2303      	movs	r3, #3
 8001d5c:	431a      	orrs	r2, r3
 8001d5e:	4691      	mov	r9, r2
 8001d60:	4652      	mov	r2, sl
 8001d62:	e68c      	b.n	8001a7e <__aeabi_dmul+0x86>
 8001d64:	220c      	movs	r2, #12
 8001d66:	9300      	str	r3, [sp, #0]
 8001d68:	2303      	movs	r3, #3
 8001d6a:	0005      	movs	r5, r0
 8001d6c:	4691      	mov	r9, r2
 8001d6e:	469b      	mov	fp, r3
 8001d70:	e666      	b.n	8001a40 <__aeabi_dmul+0x48>
 8001d72:	2304      	movs	r3, #4
 8001d74:	4699      	mov	r9, r3
 8001d76:	2300      	movs	r3, #0
 8001d78:	9300      	str	r3, [sp, #0]
 8001d7a:	3301      	adds	r3, #1
 8001d7c:	2400      	movs	r4, #0
 8001d7e:	469b      	mov	fp, r3
 8001d80:	e65e      	b.n	8001a40 <__aeabi_dmul+0x48>
 8001d82:	46c0      	nop			; (mov r8, r8)
 8001d84:	000007ff 	.word	0x000007ff
 8001d88:	fffffc01 	.word	0xfffffc01
 8001d8c:	0800a078 	.word	0x0800a078
 8001d90:	000003ff 	.word	0x000003ff
 8001d94:	feffffff 	.word	0xfeffffff
 8001d98:	000007fe 	.word	0x000007fe
 8001d9c:	fffffc0d 	.word	0xfffffc0d
 8001da0:	4649      	mov	r1, r9
 8001da2:	2301      	movs	r3, #1
 8001da4:	4319      	orrs	r1, r3
 8001da6:	4689      	mov	r9, r1
 8001da8:	2600      	movs	r6, #0
 8001daa:	2001      	movs	r0, #1
 8001dac:	e667      	b.n	8001a7e <__aeabi_dmul+0x86>
 8001dae:	2300      	movs	r3, #0
 8001db0:	2480      	movs	r4, #128	; 0x80
 8001db2:	2500      	movs	r5, #0
 8001db4:	4a43      	ldr	r2, [pc, #268]	; (8001ec4 <__aeabi_dmul+0x4cc>)
 8001db6:	9301      	str	r3, [sp, #4]
 8001db8:	0324      	lsls	r4, r4, #12
 8001dba:	e67e      	b.n	8001aba <__aeabi_dmul+0xc2>
 8001dbc:	2001      	movs	r0, #1
 8001dbe:	1a40      	subs	r0, r0, r1
 8001dc0:	2838      	cmp	r0, #56	; 0x38
 8001dc2:	dd00      	ble.n	8001dc6 <__aeabi_dmul+0x3ce>
 8001dc4:	e676      	b.n	8001ab4 <__aeabi_dmul+0xbc>
 8001dc6:	281f      	cmp	r0, #31
 8001dc8:	dd5b      	ble.n	8001e82 <__aeabi_dmul+0x48a>
 8001dca:	221f      	movs	r2, #31
 8001dcc:	0023      	movs	r3, r4
 8001dce:	4252      	negs	r2, r2
 8001dd0:	1a51      	subs	r1, r2, r1
 8001dd2:	40cb      	lsrs	r3, r1
 8001dd4:	0019      	movs	r1, r3
 8001dd6:	2820      	cmp	r0, #32
 8001dd8:	d003      	beq.n	8001de2 <__aeabi_dmul+0x3ea>
 8001dda:	4a3b      	ldr	r2, [pc, #236]	; (8001ec8 <__aeabi_dmul+0x4d0>)
 8001ddc:	4462      	add	r2, ip
 8001dde:	4094      	lsls	r4, r2
 8001de0:	4325      	orrs	r5, r4
 8001de2:	1e6a      	subs	r2, r5, #1
 8001de4:	4195      	sbcs	r5, r2
 8001de6:	002a      	movs	r2, r5
 8001de8:	430a      	orrs	r2, r1
 8001dea:	2107      	movs	r1, #7
 8001dec:	000d      	movs	r5, r1
 8001dee:	2400      	movs	r4, #0
 8001df0:	4015      	ands	r5, r2
 8001df2:	4211      	tst	r1, r2
 8001df4:	d05b      	beq.n	8001eae <__aeabi_dmul+0x4b6>
 8001df6:	210f      	movs	r1, #15
 8001df8:	2400      	movs	r4, #0
 8001dfa:	4011      	ands	r1, r2
 8001dfc:	2904      	cmp	r1, #4
 8001dfe:	d053      	beq.n	8001ea8 <__aeabi_dmul+0x4b0>
 8001e00:	1d11      	adds	r1, r2, #4
 8001e02:	4291      	cmp	r1, r2
 8001e04:	4192      	sbcs	r2, r2
 8001e06:	4252      	negs	r2, r2
 8001e08:	18a4      	adds	r4, r4, r2
 8001e0a:	000a      	movs	r2, r1
 8001e0c:	0223      	lsls	r3, r4, #8
 8001e0e:	d54b      	bpl.n	8001ea8 <__aeabi_dmul+0x4b0>
 8001e10:	2201      	movs	r2, #1
 8001e12:	2400      	movs	r4, #0
 8001e14:	2500      	movs	r5, #0
 8001e16:	e650      	b.n	8001aba <__aeabi_dmul+0xc2>
 8001e18:	2380      	movs	r3, #128	; 0x80
 8001e1a:	031b      	lsls	r3, r3, #12
 8001e1c:	421c      	tst	r4, r3
 8001e1e:	d009      	beq.n	8001e34 <__aeabi_dmul+0x43c>
 8001e20:	421e      	tst	r6, r3
 8001e22:	d107      	bne.n	8001e34 <__aeabi_dmul+0x43c>
 8001e24:	4333      	orrs	r3, r6
 8001e26:	031c      	lsls	r4, r3, #12
 8001e28:	4643      	mov	r3, r8
 8001e2a:	0015      	movs	r5, r2
 8001e2c:	0b24      	lsrs	r4, r4, #12
 8001e2e:	4a25      	ldr	r2, [pc, #148]	; (8001ec4 <__aeabi_dmul+0x4cc>)
 8001e30:	9301      	str	r3, [sp, #4]
 8001e32:	e642      	b.n	8001aba <__aeabi_dmul+0xc2>
 8001e34:	2280      	movs	r2, #128	; 0x80
 8001e36:	0312      	lsls	r2, r2, #12
 8001e38:	4314      	orrs	r4, r2
 8001e3a:	0324      	lsls	r4, r4, #12
 8001e3c:	4a21      	ldr	r2, [pc, #132]	; (8001ec4 <__aeabi_dmul+0x4cc>)
 8001e3e:	0b24      	lsrs	r4, r4, #12
 8001e40:	9701      	str	r7, [sp, #4]
 8001e42:	e63a      	b.n	8001aba <__aeabi_dmul+0xc2>
 8001e44:	f000 fd50 	bl	80028e8 <__clzsi2>
 8001e48:	0001      	movs	r1, r0
 8001e4a:	0002      	movs	r2, r0
 8001e4c:	3115      	adds	r1, #21
 8001e4e:	3220      	adds	r2, #32
 8001e50:	291c      	cmp	r1, #28
 8001e52:	dc00      	bgt.n	8001e56 <__aeabi_dmul+0x45e>
 8001e54:	e74b      	b.n	8001cee <__aeabi_dmul+0x2f6>
 8001e56:	0034      	movs	r4, r6
 8001e58:	3808      	subs	r0, #8
 8001e5a:	2500      	movs	r5, #0
 8001e5c:	4084      	lsls	r4, r0
 8001e5e:	e750      	b.n	8001d02 <__aeabi_dmul+0x30a>
 8001e60:	f000 fd42 	bl	80028e8 <__clzsi2>
 8001e64:	0003      	movs	r3, r0
 8001e66:	001a      	movs	r2, r3
 8001e68:	3215      	adds	r2, #21
 8001e6a:	3020      	adds	r0, #32
 8001e6c:	2a1c      	cmp	r2, #28
 8001e6e:	dc00      	bgt.n	8001e72 <__aeabi_dmul+0x47a>
 8001e70:	e71e      	b.n	8001cb0 <__aeabi_dmul+0x2b8>
 8001e72:	4656      	mov	r6, sl
 8001e74:	3b08      	subs	r3, #8
 8001e76:	2200      	movs	r2, #0
 8001e78:	409e      	lsls	r6, r3
 8001e7a:	e723      	b.n	8001cc4 <__aeabi_dmul+0x2cc>
 8001e7c:	9b00      	ldr	r3, [sp, #0]
 8001e7e:	469c      	mov	ip, r3
 8001e80:	e6e6      	b.n	8001c50 <__aeabi_dmul+0x258>
 8001e82:	4912      	ldr	r1, [pc, #72]	; (8001ecc <__aeabi_dmul+0x4d4>)
 8001e84:	0022      	movs	r2, r4
 8001e86:	4461      	add	r1, ip
 8001e88:	002e      	movs	r6, r5
 8001e8a:	408d      	lsls	r5, r1
 8001e8c:	408a      	lsls	r2, r1
 8001e8e:	40c6      	lsrs	r6, r0
 8001e90:	1e69      	subs	r1, r5, #1
 8001e92:	418d      	sbcs	r5, r1
 8001e94:	4332      	orrs	r2, r6
 8001e96:	432a      	orrs	r2, r5
 8001e98:	40c4      	lsrs	r4, r0
 8001e9a:	0753      	lsls	r3, r2, #29
 8001e9c:	d0b6      	beq.n	8001e0c <__aeabi_dmul+0x414>
 8001e9e:	210f      	movs	r1, #15
 8001ea0:	4011      	ands	r1, r2
 8001ea2:	2904      	cmp	r1, #4
 8001ea4:	d1ac      	bne.n	8001e00 <__aeabi_dmul+0x408>
 8001ea6:	e7b1      	b.n	8001e0c <__aeabi_dmul+0x414>
 8001ea8:	0765      	lsls	r5, r4, #29
 8001eaa:	0264      	lsls	r4, r4, #9
 8001eac:	0b24      	lsrs	r4, r4, #12
 8001eae:	08d2      	lsrs	r2, r2, #3
 8001eb0:	4315      	orrs	r5, r2
 8001eb2:	2200      	movs	r2, #0
 8001eb4:	e601      	b.n	8001aba <__aeabi_dmul+0xc2>
 8001eb6:	2280      	movs	r2, #128	; 0x80
 8001eb8:	0312      	lsls	r2, r2, #12
 8001eba:	4314      	orrs	r4, r2
 8001ebc:	0324      	lsls	r4, r4, #12
 8001ebe:	4a01      	ldr	r2, [pc, #4]	; (8001ec4 <__aeabi_dmul+0x4cc>)
 8001ec0:	0b24      	lsrs	r4, r4, #12
 8001ec2:	e5fa      	b.n	8001aba <__aeabi_dmul+0xc2>
 8001ec4:	000007ff 	.word	0x000007ff
 8001ec8:	0000043e 	.word	0x0000043e
 8001ecc:	0000041e 	.word	0x0000041e

08001ed0 <__aeabi_dsub>:
 8001ed0:	b5f8      	push	{r3, r4, r5, r6, r7, lr}
 8001ed2:	4657      	mov	r7, sl
 8001ed4:	464e      	mov	r6, r9
 8001ed6:	4645      	mov	r5, r8
 8001ed8:	46de      	mov	lr, fp
 8001eda:	b5e0      	push	{r5, r6, r7, lr}
 8001edc:	001e      	movs	r6, r3
 8001ede:	0017      	movs	r7, r2
 8001ee0:	004a      	lsls	r2, r1, #1
 8001ee2:	030b      	lsls	r3, r1, #12
 8001ee4:	0d52      	lsrs	r2, r2, #21
 8001ee6:	0a5b      	lsrs	r3, r3, #9
 8001ee8:	4690      	mov	r8, r2
 8001eea:	0f42      	lsrs	r2, r0, #29
 8001eec:	431a      	orrs	r2, r3
 8001eee:	0fcd      	lsrs	r5, r1, #31
 8001ef0:	4ccd      	ldr	r4, [pc, #820]	; (8002228 <__aeabi_dsub+0x358>)
 8001ef2:	0331      	lsls	r1, r6, #12
 8001ef4:	00c3      	lsls	r3, r0, #3
 8001ef6:	4694      	mov	ip, r2
 8001ef8:	0070      	lsls	r0, r6, #1
 8001efa:	0f7a      	lsrs	r2, r7, #29
 8001efc:	0a49      	lsrs	r1, r1, #9
 8001efe:	00ff      	lsls	r7, r7, #3
 8001f00:	469a      	mov	sl, r3
 8001f02:	46b9      	mov	r9, r7
 8001f04:	0d40      	lsrs	r0, r0, #21
 8001f06:	0ff6      	lsrs	r6, r6, #31
 8001f08:	4311      	orrs	r1, r2
 8001f0a:	42a0      	cmp	r0, r4
 8001f0c:	d100      	bne.n	8001f10 <__aeabi_dsub+0x40>
 8001f0e:	e0b1      	b.n	8002074 <__aeabi_dsub+0x1a4>
 8001f10:	2201      	movs	r2, #1
 8001f12:	4056      	eors	r6, r2
 8001f14:	46b3      	mov	fp, r6
 8001f16:	42b5      	cmp	r5, r6
 8001f18:	d100      	bne.n	8001f1c <__aeabi_dsub+0x4c>
 8001f1a:	e088      	b.n	800202e <__aeabi_dsub+0x15e>
 8001f1c:	4642      	mov	r2, r8
 8001f1e:	1a12      	subs	r2, r2, r0
 8001f20:	2a00      	cmp	r2, #0
 8001f22:	dc00      	bgt.n	8001f26 <__aeabi_dsub+0x56>
 8001f24:	e0ae      	b.n	8002084 <__aeabi_dsub+0x1b4>
 8001f26:	2800      	cmp	r0, #0
 8001f28:	d100      	bne.n	8001f2c <__aeabi_dsub+0x5c>
 8001f2a:	e0c1      	b.n	80020b0 <__aeabi_dsub+0x1e0>
 8001f2c:	48be      	ldr	r0, [pc, #760]	; (8002228 <__aeabi_dsub+0x358>)
 8001f2e:	4580      	cmp	r8, r0
 8001f30:	d100      	bne.n	8001f34 <__aeabi_dsub+0x64>
 8001f32:	e151      	b.n	80021d8 <__aeabi_dsub+0x308>
 8001f34:	2080      	movs	r0, #128	; 0x80
 8001f36:	0400      	lsls	r0, r0, #16
 8001f38:	4301      	orrs	r1, r0
 8001f3a:	2a38      	cmp	r2, #56	; 0x38
 8001f3c:	dd00      	ble.n	8001f40 <__aeabi_dsub+0x70>
 8001f3e:	e17b      	b.n	8002238 <__aeabi_dsub+0x368>
 8001f40:	2a1f      	cmp	r2, #31
 8001f42:	dd00      	ble.n	8001f46 <__aeabi_dsub+0x76>
 8001f44:	e1ee      	b.n	8002324 <__aeabi_dsub+0x454>
 8001f46:	2020      	movs	r0, #32
 8001f48:	003e      	movs	r6, r7
 8001f4a:	1a80      	subs	r0, r0, r2
 8001f4c:	000c      	movs	r4, r1
 8001f4e:	40d6      	lsrs	r6, r2
 8001f50:	40d1      	lsrs	r1, r2
 8001f52:	4087      	lsls	r7, r0
 8001f54:	4662      	mov	r2, ip
 8001f56:	4084      	lsls	r4, r0
 8001f58:	1a52      	subs	r2, r2, r1
 8001f5a:	1e78      	subs	r0, r7, #1
 8001f5c:	4187      	sbcs	r7, r0
 8001f5e:	4694      	mov	ip, r2
 8001f60:	4334      	orrs	r4, r6
 8001f62:	4327      	orrs	r7, r4
 8001f64:	1bdc      	subs	r4, r3, r7
 8001f66:	42a3      	cmp	r3, r4
 8001f68:	419b      	sbcs	r3, r3
 8001f6a:	4662      	mov	r2, ip
 8001f6c:	425b      	negs	r3, r3
 8001f6e:	1ad3      	subs	r3, r2, r3
 8001f70:	4699      	mov	r9, r3
 8001f72:	464b      	mov	r3, r9
 8001f74:	021b      	lsls	r3, r3, #8
 8001f76:	d400      	bmi.n	8001f7a <__aeabi_dsub+0xaa>
 8001f78:	e118      	b.n	80021ac <__aeabi_dsub+0x2dc>
 8001f7a:	464b      	mov	r3, r9
 8001f7c:	0258      	lsls	r0, r3, #9
 8001f7e:	0a43      	lsrs	r3, r0, #9
 8001f80:	4699      	mov	r9, r3
 8001f82:	464b      	mov	r3, r9
 8001f84:	2b00      	cmp	r3, #0
 8001f86:	d100      	bne.n	8001f8a <__aeabi_dsub+0xba>
 8001f88:	e137      	b.n	80021fa <__aeabi_dsub+0x32a>
 8001f8a:	4648      	mov	r0, r9
 8001f8c:	f000 fcac 	bl	80028e8 <__clzsi2>
 8001f90:	0001      	movs	r1, r0
 8001f92:	3908      	subs	r1, #8
 8001f94:	2320      	movs	r3, #32
 8001f96:	0022      	movs	r2, r4
 8001f98:	4648      	mov	r0, r9
 8001f9a:	1a5b      	subs	r3, r3, r1
 8001f9c:	40da      	lsrs	r2, r3
 8001f9e:	4088      	lsls	r0, r1
 8001fa0:	408c      	lsls	r4, r1
 8001fa2:	4643      	mov	r3, r8
 8001fa4:	4310      	orrs	r0, r2
 8001fa6:	4588      	cmp	r8, r1
 8001fa8:	dd00      	ble.n	8001fac <__aeabi_dsub+0xdc>
 8001faa:	e136      	b.n	800221a <__aeabi_dsub+0x34a>
 8001fac:	1ac9      	subs	r1, r1, r3
 8001fae:	1c4b      	adds	r3, r1, #1
 8001fb0:	2b1f      	cmp	r3, #31
 8001fb2:	dd00      	ble.n	8001fb6 <__aeabi_dsub+0xe6>
 8001fb4:	e0ea      	b.n	800218c <__aeabi_dsub+0x2bc>
 8001fb6:	2220      	movs	r2, #32
 8001fb8:	0026      	movs	r6, r4
 8001fba:	1ad2      	subs	r2, r2, r3
 8001fbc:	0001      	movs	r1, r0
 8001fbe:	4094      	lsls	r4, r2
 8001fc0:	40de      	lsrs	r6, r3
 8001fc2:	40d8      	lsrs	r0, r3
 8001fc4:	2300      	movs	r3, #0
 8001fc6:	4091      	lsls	r1, r2
 8001fc8:	1e62      	subs	r2, r4, #1
 8001fca:	4194      	sbcs	r4, r2
 8001fcc:	4681      	mov	r9, r0
 8001fce:	4698      	mov	r8, r3
 8001fd0:	4331      	orrs	r1, r6
 8001fd2:	430c      	orrs	r4, r1
 8001fd4:	0763      	lsls	r3, r4, #29
 8001fd6:	d009      	beq.n	8001fec <__aeabi_dsub+0x11c>
 8001fd8:	230f      	movs	r3, #15
 8001fda:	4023      	ands	r3, r4
 8001fdc:	2b04      	cmp	r3, #4
 8001fde:	d005      	beq.n	8001fec <__aeabi_dsub+0x11c>
 8001fe0:	1d23      	adds	r3, r4, #4
 8001fe2:	42a3      	cmp	r3, r4
 8001fe4:	41a4      	sbcs	r4, r4
 8001fe6:	4264      	negs	r4, r4
 8001fe8:	44a1      	add	r9, r4
 8001fea:	001c      	movs	r4, r3
 8001fec:	464b      	mov	r3, r9
 8001fee:	021b      	lsls	r3, r3, #8
 8001ff0:	d400      	bmi.n	8001ff4 <__aeabi_dsub+0x124>
 8001ff2:	e0de      	b.n	80021b2 <__aeabi_dsub+0x2e2>
 8001ff4:	4641      	mov	r1, r8
 8001ff6:	4b8c      	ldr	r3, [pc, #560]	; (8002228 <__aeabi_dsub+0x358>)
 8001ff8:	3101      	adds	r1, #1
 8001ffa:	4299      	cmp	r1, r3
 8001ffc:	d100      	bne.n	8002000 <__aeabi_dsub+0x130>
 8001ffe:	e0e7      	b.n	80021d0 <__aeabi_dsub+0x300>
 8002000:	464b      	mov	r3, r9
 8002002:	488a      	ldr	r0, [pc, #552]	; (800222c <__aeabi_dsub+0x35c>)
 8002004:	08e4      	lsrs	r4, r4, #3
 8002006:	4003      	ands	r3, r0
 8002008:	0018      	movs	r0, r3
 800200a:	0549      	lsls	r1, r1, #21
 800200c:	075b      	lsls	r3, r3, #29
 800200e:	0240      	lsls	r0, r0, #9
 8002010:	4323      	orrs	r3, r4
 8002012:	0d4a      	lsrs	r2, r1, #21
 8002014:	0b04      	lsrs	r4, r0, #12
 8002016:	0512      	lsls	r2, r2, #20
 8002018:	07ed      	lsls	r5, r5, #31
 800201a:	4322      	orrs	r2, r4
 800201c:	432a      	orrs	r2, r5
 800201e:	0018      	movs	r0, r3
 8002020:	0011      	movs	r1, r2
 8002022:	bcf0      	pop	{r4, r5, r6, r7}
 8002024:	46bb      	mov	fp, r7
 8002026:	46b2      	mov	sl, r6
 8002028:	46a9      	mov	r9, r5
 800202a:	46a0      	mov	r8, r4
 800202c:	bdf8      	pop	{r3, r4, r5, r6, r7, pc}
 800202e:	4642      	mov	r2, r8
 8002030:	1a12      	subs	r2, r2, r0
 8002032:	2a00      	cmp	r2, #0
 8002034:	dd52      	ble.n	80020dc <__aeabi_dsub+0x20c>
 8002036:	2800      	cmp	r0, #0
 8002038:	d100      	bne.n	800203c <__aeabi_dsub+0x16c>
 800203a:	e09c      	b.n	8002176 <__aeabi_dsub+0x2a6>
 800203c:	45a0      	cmp	r8, r4
 800203e:	d100      	bne.n	8002042 <__aeabi_dsub+0x172>
 8002040:	e0ca      	b.n	80021d8 <__aeabi_dsub+0x308>
 8002042:	2080      	movs	r0, #128	; 0x80
 8002044:	0400      	lsls	r0, r0, #16
 8002046:	4301      	orrs	r1, r0
 8002048:	2a38      	cmp	r2, #56	; 0x38
 800204a:	dd00      	ble.n	800204e <__aeabi_dsub+0x17e>
 800204c:	e149      	b.n	80022e2 <__aeabi_dsub+0x412>
 800204e:	2a1f      	cmp	r2, #31
 8002050:	dc00      	bgt.n	8002054 <__aeabi_dsub+0x184>
 8002052:	e197      	b.n	8002384 <__aeabi_dsub+0x4b4>
 8002054:	0010      	movs	r0, r2
 8002056:	000e      	movs	r6, r1
 8002058:	3820      	subs	r0, #32
 800205a:	40c6      	lsrs	r6, r0
 800205c:	2a20      	cmp	r2, #32
 800205e:	d004      	beq.n	800206a <__aeabi_dsub+0x19a>
 8002060:	2040      	movs	r0, #64	; 0x40
 8002062:	1a82      	subs	r2, r0, r2
 8002064:	4091      	lsls	r1, r2
 8002066:	430f      	orrs	r7, r1
 8002068:	46b9      	mov	r9, r7
 800206a:	464c      	mov	r4, r9
 800206c:	1e62      	subs	r2, r4, #1
 800206e:	4194      	sbcs	r4, r2
 8002070:	4334      	orrs	r4, r6
 8002072:	e13a      	b.n	80022ea <__aeabi_dsub+0x41a>
 8002074:	000a      	movs	r2, r1
 8002076:	433a      	orrs	r2, r7
 8002078:	d028      	beq.n	80020cc <__aeabi_dsub+0x1fc>
 800207a:	46b3      	mov	fp, r6
 800207c:	42b5      	cmp	r5, r6
 800207e:	d02b      	beq.n	80020d8 <__aeabi_dsub+0x208>
 8002080:	4a6b      	ldr	r2, [pc, #428]	; (8002230 <__aeabi_dsub+0x360>)
 8002082:	4442      	add	r2, r8
 8002084:	2a00      	cmp	r2, #0
 8002086:	d05d      	beq.n	8002144 <__aeabi_dsub+0x274>
 8002088:	4642      	mov	r2, r8
 800208a:	4644      	mov	r4, r8
 800208c:	1a82      	subs	r2, r0, r2
 800208e:	2c00      	cmp	r4, #0
 8002090:	d000      	beq.n	8002094 <__aeabi_dsub+0x1c4>
 8002092:	e0f5      	b.n	8002280 <__aeabi_dsub+0x3b0>
 8002094:	4665      	mov	r5, ip
 8002096:	431d      	orrs	r5, r3
 8002098:	d100      	bne.n	800209c <__aeabi_dsub+0x1cc>
 800209a:	e19c      	b.n	80023d6 <__aeabi_dsub+0x506>
 800209c:	1e55      	subs	r5, r2, #1
 800209e:	2a01      	cmp	r2, #1
 80020a0:	d100      	bne.n	80020a4 <__aeabi_dsub+0x1d4>
 80020a2:	e1fb      	b.n	800249c <__aeabi_dsub+0x5cc>
 80020a4:	4c60      	ldr	r4, [pc, #384]	; (8002228 <__aeabi_dsub+0x358>)
 80020a6:	42a2      	cmp	r2, r4
 80020a8:	d100      	bne.n	80020ac <__aeabi_dsub+0x1dc>
 80020aa:	e1bd      	b.n	8002428 <__aeabi_dsub+0x558>
 80020ac:	002a      	movs	r2, r5
 80020ae:	e0f0      	b.n	8002292 <__aeabi_dsub+0x3c2>
 80020b0:	0008      	movs	r0, r1
 80020b2:	4338      	orrs	r0, r7
 80020b4:	d100      	bne.n	80020b8 <__aeabi_dsub+0x1e8>
 80020b6:	e0c3      	b.n	8002240 <__aeabi_dsub+0x370>
 80020b8:	1e50      	subs	r0, r2, #1
 80020ba:	2a01      	cmp	r2, #1
 80020bc:	d100      	bne.n	80020c0 <__aeabi_dsub+0x1f0>
 80020be:	e1a8      	b.n	8002412 <__aeabi_dsub+0x542>
 80020c0:	4c59      	ldr	r4, [pc, #356]	; (8002228 <__aeabi_dsub+0x358>)
 80020c2:	42a2      	cmp	r2, r4
 80020c4:	d100      	bne.n	80020c8 <__aeabi_dsub+0x1f8>
 80020c6:	e087      	b.n	80021d8 <__aeabi_dsub+0x308>
 80020c8:	0002      	movs	r2, r0
 80020ca:	e736      	b.n	8001f3a <__aeabi_dsub+0x6a>
 80020cc:	2201      	movs	r2, #1
 80020ce:	4056      	eors	r6, r2
 80020d0:	46b3      	mov	fp, r6
 80020d2:	42b5      	cmp	r5, r6
 80020d4:	d000      	beq.n	80020d8 <__aeabi_dsub+0x208>
 80020d6:	e721      	b.n	8001f1c <__aeabi_dsub+0x4c>
 80020d8:	4a55      	ldr	r2, [pc, #340]	; (8002230 <__aeabi_dsub+0x360>)
 80020da:	4442      	add	r2, r8
 80020dc:	2a00      	cmp	r2, #0
 80020de:	d100      	bne.n	80020e2 <__aeabi_dsub+0x212>
 80020e0:	e0b5      	b.n	800224e <__aeabi_dsub+0x37e>
 80020e2:	4642      	mov	r2, r8
 80020e4:	4644      	mov	r4, r8
 80020e6:	1a82      	subs	r2, r0, r2
 80020e8:	2c00      	cmp	r4, #0
 80020ea:	d100      	bne.n	80020ee <__aeabi_dsub+0x21e>
 80020ec:	e138      	b.n	8002360 <__aeabi_dsub+0x490>
 80020ee:	4e4e      	ldr	r6, [pc, #312]	; (8002228 <__aeabi_dsub+0x358>)
 80020f0:	42b0      	cmp	r0, r6
 80020f2:	d100      	bne.n	80020f6 <__aeabi_dsub+0x226>
 80020f4:	e1de      	b.n	80024b4 <__aeabi_dsub+0x5e4>
 80020f6:	2680      	movs	r6, #128	; 0x80
 80020f8:	4664      	mov	r4, ip
 80020fa:	0436      	lsls	r6, r6, #16
 80020fc:	4334      	orrs	r4, r6
 80020fe:	46a4      	mov	ip, r4
 8002100:	2a38      	cmp	r2, #56	; 0x38
 8002102:	dd00      	ble.n	8002106 <__aeabi_dsub+0x236>
 8002104:	e196      	b.n	8002434 <__aeabi_dsub+0x564>
 8002106:	2a1f      	cmp	r2, #31
 8002108:	dd00      	ble.n	800210c <__aeabi_dsub+0x23c>
 800210a:	e224      	b.n	8002556 <__aeabi_dsub+0x686>
 800210c:	2620      	movs	r6, #32
 800210e:	1ab4      	subs	r4, r6, r2
 8002110:	46a2      	mov	sl, r4
 8002112:	4664      	mov	r4, ip
 8002114:	4656      	mov	r6, sl
 8002116:	40b4      	lsls	r4, r6
 8002118:	46a1      	mov	r9, r4
 800211a:	001c      	movs	r4, r3
 800211c:	464e      	mov	r6, r9
 800211e:	40d4      	lsrs	r4, r2
 8002120:	4326      	orrs	r6, r4
 8002122:	0034      	movs	r4, r6
 8002124:	4656      	mov	r6, sl
 8002126:	40b3      	lsls	r3, r6
 8002128:	1e5e      	subs	r6, r3, #1
 800212a:	41b3      	sbcs	r3, r6
 800212c:	431c      	orrs	r4, r3
 800212e:	4663      	mov	r3, ip
 8002130:	40d3      	lsrs	r3, r2
 8002132:	18c9      	adds	r1, r1, r3
 8002134:	19e4      	adds	r4, r4, r7
 8002136:	42bc      	cmp	r4, r7
 8002138:	41bf      	sbcs	r7, r7
 800213a:	427f      	negs	r7, r7
 800213c:	46b9      	mov	r9, r7
 800213e:	4680      	mov	r8, r0
 8002140:	4489      	add	r9, r1
 8002142:	e0d8      	b.n	80022f6 <__aeabi_dsub+0x426>
 8002144:	4640      	mov	r0, r8
 8002146:	4c3b      	ldr	r4, [pc, #236]	; (8002234 <__aeabi_dsub+0x364>)
 8002148:	3001      	adds	r0, #1
 800214a:	4220      	tst	r0, r4
 800214c:	d000      	beq.n	8002150 <__aeabi_dsub+0x280>
 800214e:	e0b4      	b.n	80022ba <__aeabi_dsub+0x3ea>
 8002150:	4640      	mov	r0, r8
 8002152:	2800      	cmp	r0, #0
 8002154:	d000      	beq.n	8002158 <__aeabi_dsub+0x288>
 8002156:	e144      	b.n	80023e2 <__aeabi_dsub+0x512>
 8002158:	4660      	mov	r0, ip
 800215a:	4318      	orrs	r0, r3
 800215c:	d100      	bne.n	8002160 <__aeabi_dsub+0x290>
 800215e:	e190      	b.n	8002482 <__aeabi_dsub+0x5b2>
 8002160:	0008      	movs	r0, r1
 8002162:	4338      	orrs	r0, r7
 8002164:	d000      	beq.n	8002168 <__aeabi_dsub+0x298>
 8002166:	e1aa      	b.n	80024be <__aeabi_dsub+0x5ee>
 8002168:	4661      	mov	r1, ip
 800216a:	08db      	lsrs	r3, r3, #3
 800216c:	0749      	lsls	r1, r1, #29
 800216e:	430b      	orrs	r3, r1
 8002170:	4661      	mov	r1, ip
 8002172:	08cc      	lsrs	r4, r1, #3
 8002174:	e027      	b.n	80021c6 <__aeabi_dsub+0x2f6>
 8002176:	0008      	movs	r0, r1
 8002178:	4338      	orrs	r0, r7
 800217a:	d061      	beq.n	8002240 <__aeabi_dsub+0x370>
 800217c:	1e50      	subs	r0, r2, #1
 800217e:	2a01      	cmp	r2, #1
 8002180:	d100      	bne.n	8002184 <__aeabi_dsub+0x2b4>
 8002182:	e139      	b.n	80023f8 <__aeabi_dsub+0x528>
 8002184:	42a2      	cmp	r2, r4
 8002186:	d027      	beq.n	80021d8 <__aeabi_dsub+0x308>
 8002188:	0002      	movs	r2, r0
 800218a:	e75d      	b.n	8002048 <__aeabi_dsub+0x178>
 800218c:	0002      	movs	r2, r0
 800218e:	391f      	subs	r1, #31
 8002190:	40ca      	lsrs	r2, r1
 8002192:	0011      	movs	r1, r2
 8002194:	2b20      	cmp	r3, #32
 8002196:	d003      	beq.n	80021a0 <__aeabi_dsub+0x2d0>
 8002198:	2240      	movs	r2, #64	; 0x40
 800219a:	1ad3      	subs	r3, r2, r3
 800219c:	4098      	lsls	r0, r3
 800219e:	4304      	orrs	r4, r0
 80021a0:	1e63      	subs	r3, r4, #1
 80021a2:	419c      	sbcs	r4, r3
 80021a4:	2300      	movs	r3, #0
 80021a6:	4699      	mov	r9, r3
 80021a8:	4698      	mov	r8, r3
 80021aa:	430c      	orrs	r4, r1
 80021ac:	0763      	lsls	r3, r4, #29
 80021ae:	d000      	beq.n	80021b2 <__aeabi_dsub+0x2e2>
 80021b0:	e712      	b.n	8001fd8 <__aeabi_dsub+0x108>
 80021b2:	464b      	mov	r3, r9
 80021b4:	464a      	mov	r2, r9
 80021b6:	08e4      	lsrs	r4, r4, #3
 80021b8:	075b      	lsls	r3, r3, #29
 80021ba:	4323      	orrs	r3, r4
 80021bc:	08d4      	lsrs	r4, r2, #3
 80021be:	4642      	mov	r2, r8
 80021c0:	4919      	ldr	r1, [pc, #100]	; (8002228 <__aeabi_dsub+0x358>)
 80021c2:	428a      	cmp	r2, r1
 80021c4:	d00e      	beq.n	80021e4 <__aeabi_dsub+0x314>
 80021c6:	0324      	lsls	r4, r4, #12
 80021c8:	0552      	lsls	r2, r2, #21
 80021ca:	0b24      	lsrs	r4, r4, #12
 80021cc:	0d52      	lsrs	r2, r2, #21
 80021ce:	e722      	b.n	8002016 <__aeabi_dsub+0x146>
 80021d0:	000a      	movs	r2, r1
 80021d2:	2400      	movs	r4, #0
 80021d4:	2300      	movs	r3, #0
 80021d6:	e71e      	b.n	8002016 <__aeabi_dsub+0x146>
 80021d8:	08db      	lsrs	r3, r3, #3
 80021da:	4662      	mov	r2, ip
 80021dc:	0752      	lsls	r2, r2, #29
 80021de:	4313      	orrs	r3, r2
 80021e0:	4662      	mov	r2, ip
 80021e2:	08d4      	lsrs	r4, r2, #3
 80021e4:	001a      	movs	r2, r3
 80021e6:	4322      	orrs	r2, r4
 80021e8:	d100      	bne.n	80021ec <__aeabi_dsub+0x31c>
 80021ea:	e1fc      	b.n	80025e6 <__aeabi_dsub+0x716>
 80021ec:	2280      	movs	r2, #128	; 0x80
 80021ee:	0312      	lsls	r2, r2, #12
 80021f0:	4314      	orrs	r4, r2
 80021f2:	0324      	lsls	r4, r4, #12
 80021f4:	4a0c      	ldr	r2, [pc, #48]	; (8002228 <__aeabi_dsub+0x358>)
 80021f6:	0b24      	lsrs	r4, r4, #12
 80021f8:	e70d      	b.n	8002016 <__aeabi_dsub+0x146>
 80021fa:	0020      	movs	r0, r4
 80021fc:	f000 fb74 	bl	80028e8 <__clzsi2>
 8002200:	0001      	movs	r1, r0
 8002202:	3118      	adds	r1, #24
 8002204:	291f      	cmp	r1, #31
 8002206:	dc00      	bgt.n	800220a <__aeabi_dsub+0x33a>
 8002208:	e6c4      	b.n	8001f94 <__aeabi_dsub+0xc4>
 800220a:	3808      	subs	r0, #8
 800220c:	4084      	lsls	r4, r0
 800220e:	4643      	mov	r3, r8
 8002210:	0020      	movs	r0, r4
 8002212:	2400      	movs	r4, #0
 8002214:	4588      	cmp	r8, r1
 8002216:	dc00      	bgt.n	800221a <__aeabi_dsub+0x34a>
 8002218:	e6c8      	b.n	8001fac <__aeabi_dsub+0xdc>
 800221a:	4a04      	ldr	r2, [pc, #16]	; (800222c <__aeabi_dsub+0x35c>)
 800221c:	1a5b      	subs	r3, r3, r1
 800221e:	4010      	ands	r0, r2
 8002220:	4698      	mov	r8, r3
 8002222:	4681      	mov	r9, r0
 8002224:	e6d6      	b.n	8001fd4 <__aeabi_dsub+0x104>
 8002226:	46c0      	nop			; (mov r8, r8)
 8002228:	000007ff 	.word	0x000007ff
 800222c:	ff7fffff 	.word	0xff7fffff
 8002230:	fffff801 	.word	0xfffff801
 8002234:	000007fe 	.word	0x000007fe
 8002238:	430f      	orrs	r7, r1
 800223a:	1e7a      	subs	r2, r7, #1
 800223c:	4197      	sbcs	r7, r2
 800223e:	e691      	b.n	8001f64 <__aeabi_dsub+0x94>
 8002240:	4661      	mov	r1, ip
 8002242:	08db      	lsrs	r3, r3, #3
 8002244:	0749      	lsls	r1, r1, #29
 8002246:	430b      	orrs	r3, r1
 8002248:	4661      	mov	r1, ip
 800224a:	08cc      	lsrs	r4, r1, #3
 800224c:	e7b8      	b.n	80021c0 <__aeabi_dsub+0x2f0>
 800224e:	4640      	mov	r0, r8
 8002250:	4cd3      	ldr	r4, [pc, #844]	; (80025a0 <__aeabi_dsub+0x6d0>)
 8002252:	3001      	adds	r0, #1
 8002254:	4220      	tst	r0, r4
 8002256:	d000      	beq.n	800225a <__aeabi_dsub+0x38a>
 8002258:	e0a2      	b.n	80023a0 <__aeabi_dsub+0x4d0>
 800225a:	4640      	mov	r0, r8
 800225c:	2800      	cmp	r0, #0
 800225e:	d000      	beq.n	8002262 <__aeabi_dsub+0x392>
 8002260:	e101      	b.n	8002466 <__aeabi_dsub+0x596>
 8002262:	4660      	mov	r0, ip
 8002264:	4318      	orrs	r0, r3
 8002266:	d100      	bne.n	800226a <__aeabi_dsub+0x39a>
 8002268:	e15e      	b.n	8002528 <__aeabi_dsub+0x658>
 800226a:	0008      	movs	r0, r1
 800226c:	4338      	orrs	r0, r7
 800226e:	d000      	beq.n	8002272 <__aeabi_dsub+0x3a2>
 8002270:	e15f      	b.n	8002532 <__aeabi_dsub+0x662>
 8002272:	4661      	mov	r1, ip
 8002274:	08db      	lsrs	r3, r3, #3
 8002276:	0749      	lsls	r1, r1, #29
 8002278:	430b      	orrs	r3, r1
 800227a:	4661      	mov	r1, ip
 800227c:	08cc      	lsrs	r4, r1, #3
 800227e:	e7a2      	b.n	80021c6 <__aeabi_dsub+0x2f6>
 8002280:	4dc8      	ldr	r5, [pc, #800]	; (80025a4 <__aeabi_dsub+0x6d4>)
 8002282:	42a8      	cmp	r0, r5
 8002284:	d100      	bne.n	8002288 <__aeabi_dsub+0x3b8>
 8002286:	e0cf      	b.n	8002428 <__aeabi_dsub+0x558>
 8002288:	2580      	movs	r5, #128	; 0x80
 800228a:	4664      	mov	r4, ip
 800228c:	042d      	lsls	r5, r5, #16
 800228e:	432c      	orrs	r4, r5
 8002290:	46a4      	mov	ip, r4
 8002292:	2a38      	cmp	r2, #56	; 0x38
 8002294:	dc56      	bgt.n	8002344 <__aeabi_dsub+0x474>
 8002296:	2a1f      	cmp	r2, #31
 8002298:	dd00      	ble.n	800229c <__aeabi_dsub+0x3cc>
 800229a:	e0d1      	b.n	8002440 <__aeabi_dsub+0x570>
 800229c:	2520      	movs	r5, #32
 800229e:	001e      	movs	r6, r3
 80022a0:	1aad      	subs	r5, r5, r2
 80022a2:	4664      	mov	r4, ip
 80022a4:	40ab      	lsls	r3, r5
 80022a6:	40ac      	lsls	r4, r5
 80022a8:	40d6      	lsrs	r6, r2
 80022aa:	1e5d      	subs	r5, r3, #1
 80022ac:	41ab      	sbcs	r3, r5
 80022ae:	4334      	orrs	r4, r6
 80022b0:	4323      	orrs	r3, r4
 80022b2:	4664      	mov	r4, ip
 80022b4:	40d4      	lsrs	r4, r2
 80022b6:	1b09      	subs	r1, r1, r4
 80022b8:	e049      	b.n	800234e <__aeabi_dsub+0x47e>
 80022ba:	4660      	mov	r0, ip
 80022bc:	1bdc      	subs	r4, r3, r7
 80022be:	1a46      	subs	r6, r0, r1
 80022c0:	42a3      	cmp	r3, r4
 80022c2:	4180      	sbcs	r0, r0
 80022c4:	4240      	negs	r0, r0
 80022c6:	4681      	mov	r9, r0
 80022c8:	0030      	movs	r0, r6
 80022ca:	464e      	mov	r6, r9
 80022cc:	1b80      	subs	r0, r0, r6
 80022ce:	4681      	mov	r9, r0
 80022d0:	0200      	lsls	r0, r0, #8
 80022d2:	d476      	bmi.n	80023c2 <__aeabi_dsub+0x4f2>
 80022d4:	464b      	mov	r3, r9
 80022d6:	4323      	orrs	r3, r4
 80022d8:	d000      	beq.n	80022dc <__aeabi_dsub+0x40c>
 80022da:	e652      	b.n	8001f82 <__aeabi_dsub+0xb2>
 80022dc:	2400      	movs	r4, #0
 80022de:	2500      	movs	r5, #0
 80022e0:	e771      	b.n	80021c6 <__aeabi_dsub+0x2f6>
 80022e2:	4339      	orrs	r1, r7
 80022e4:	000c      	movs	r4, r1
 80022e6:	1e62      	subs	r2, r4, #1
 80022e8:	4194      	sbcs	r4, r2
 80022ea:	18e4      	adds	r4, r4, r3
 80022ec:	429c      	cmp	r4, r3
 80022ee:	419b      	sbcs	r3, r3
 80022f0:	425b      	negs	r3, r3
 80022f2:	4463      	add	r3, ip
 80022f4:	4699      	mov	r9, r3
 80022f6:	464b      	mov	r3, r9
 80022f8:	021b      	lsls	r3, r3, #8
 80022fa:	d400      	bmi.n	80022fe <__aeabi_dsub+0x42e>
 80022fc:	e756      	b.n	80021ac <__aeabi_dsub+0x2dc>
 80022fe:	2301      	movs	r3, #1
 8002300:	469c      	mov	ip, r3
 8002302:	4ba8      	ldr	r3, [pc, #672]	; (80025a4 <__aeabi_dsub+0x6d4>)
 8002304:	44e0      	add	r8, ip
 8002306:	4598      	cmp	r8, r3
 8002308:	d038      	beq.n	800237c <__aeabi_dsub+0x4ac>
 800230a:	464b      	mov	r3, r9
 800230c:	48a6      	ldr	r0, [pc, #664]	; (80025a8 <__aeabi_dsub+0x6d8>)
 800230e:	2201      	movs	r2, #1
 8002310:	4003      	ands	r3, r0
 8002312:	0018      	movs	r0, r3
 8002314:	0863      	lsrs	r3, r4, #1
 8002316:	4014      	ands	r4, r2
 8002318:	431c      	orrs	r4, r3
 800231a:	07c3      	lsls	r3, r0, #31
 800231c:	431c      	orrs	r4, r3
 800231e:	0843      	lsrs	r3, r0, #1
 8002320:	4699      	mov	r9, r3
 8002322:	e657      	b.n	8001fd4 <__aeabi_dsub+0x104>
 8002324:	0010      	movs	r0, r2
 8002326:	000e      	movs	r6, r1
 8002328:	3820      	subs	r0, #32
 800232a:	40c6      	lsrs	r6, r0
 800232c:	2a20      	cmp	r2, #32
 800232e:	d004      	beq.n	800233a <__aeabi_dsub+0x46a>
 8002330:	2040      	movs	r0, #64	; 0x40
 8002332:	1a82      	subs	r2, r0, r2
 8002334:	4091      	lsls	r1, r2
 8002336:	430f      	orrs	r7, r1
 8002338:	46b9      	mov	r9, r7
 800233a:	464f      	mov	r7, r9
 800233c:	1e7a      	subs	r2, r7, #1
 800233e:	4197      	sbcs	r7, r2
 8002340:	4337      	orrs	r7, r6
 8002342:	e60f      	b.n	8001f64 <__aeabi_dsub+0x94>
 8002344:	4662      	mov	r2, ip
 8002346:	431a      	orrs	r2, r3
 8002348:	0013      	movs	r3, r2
 800234a:	1e5a      	subs	r2, r3, #1
 800234c:	4193      	sbcs	r3, r2
 800234e:	1afc      	subs	r4, r7, r3
 8002350:	42a7      	cmp	r7, r4
 8002352:	41bf      	sbcs	r7, r7
 8002354:	427f      	negs	r7, r7
 8002356:	1bcb      	subs	r3, r1, r7
 8002358:	4699      	mov	r9, r3
 800235a:	465d      	mov	r5, fp
 800235c:	4680      	mov	r8, r0
 800235e:	e608      	b.n	8001f72 <__aeabi_dsub+0xa2>
 8002360:	4666      	mov	r6, ip
 8002362:	431e      	orrs	r6, r3
 8002364:	d100      	bne.n	8002368 <__aeabi_dsub+0x498>
 8002366:	e0be      	b.n	80024e6 <__aeabi_dsub+0x616>
 8002368:	1e56      	subs	r6, r2, #1
 800236a:	2a01      	cmp	r2, #1
 800236c:	d100      	bne.n	8002370 <__aeabi_dsub+0x4a0>
 800236e:	e109      	b.n	8002584 <__aeabi_dsub+0x6b4>
 8002370:	4c8c      	ldr	r4, [pc, #560]	; (80025a4 <__aeabi_dsub+0x6d4>)
 8002372:	42a2      	cmp	r2, r4
 8002374:	d100      	bne.n	8002378 <__aeabi_dsub+0x4a8>
 8002376:	e119      	b.n	80025ac <__aeabi_dsub+0x6dc>
 8002378:	0032      	movs	r2, r6
 800237a:	e6c1      	b.n	8002100 <__aeabi_dsub+0x230>
 800237c:	4642      	mov	r2, r8
 800237e:	2400      	movs	r4, #0
 8002380:	2300      	movs	r3, #0
 8002382:	e648      	b.n	8002016 <__aeabi_dsub+0x146>
 8002384:	2020      	movs	r0, #32
 8002386:	000c      	movs	r4, r1
 8002388:	1a80      	subs	r0, r0, r2
 800238a:	003e      	movs	r6, r7
 800238c:	4087      	lsls	r7, r0
 800238e:	4084      	lsls	r4, r0
 8002390:	40d6      	lsrs	r6, r2
 8002392:	1e78      	subs	r0, r7, #1
 8002394:	4187      	sbcs	r7, r0
 8002396:	40d1      	lsrs	r1, r2
 8002398:	4334      	orrs	r4, r6
 800239a:	433c      	orrs	r4, r7
 800239c:	448c      	add	ip, r1
 800239e:	e7a4      	b.n	80022ea <__aeabi_dsub+0x41a>
 80023a0:	4a80      	ldr	r2, [pc, #512]	; (80025a4 <__aeabi_dsub+0x6d4>)
 80023a2:	4290      	cmp	r0, r2
 80023a4:	d100      	bne.n	80023a8 <__aeabi_dsub+0x4d8>
 80023a6:	e0e9      	b.n	800257c <__aeabi_dsub+0x6ac>
 80023a8:	19df      	adds	r7, r3, r7
 80023aa:	429f      	cmp	r7, r3
 80023ac:	419b      	sbcs	r3, r3
 80023ae:	4461      	add	r1, ip
 80023b0:	425b      	negs	r3, r3
 80023b2:	18c9      	adds	r1, r1, r3
 80023b4:	07cc      	lsls	r4, r1, #31
 80023b6:	087f      	lsrs	r7, r7, #1
 80023b8:	084b      	lsrs	r3, r1, #1
 80023ba:	4699      	mov	r9, r3
 80023bc:	4680      	mov	r8, r0
 80023be:	433c      	orrs	r4, r7
 80023c0:	e6f4      	b.n	80021ac <__aeabi_dsub+0x2dc>
 80023c2:	1afc      	subs	r4, r7, r3
 80023c4:	42a7      	cmp	r7, r4
 80023c6:	41bf      	sbcs	r7, r7
 80023c8:	4663      	mov	r3, ip
 80023ca:	427f      	negs	r7, r7
 80023cc:	1ac9      	subs	r1, r1, r3
 80023ce:	1bcb      	subs	r3, r1, r7
 80023d0:	4699      	mov	r9, r3
 80023d2:	465d      	mov	r5, fp
 80023d4:	e5d5      	b.n	8001f82 <__aeabi_dsub+0xb2>
 80023d6:	08ff      	lsrs	r7, r7, #3
 80023d8:	074b      	lsls	r3, r1, #29
 80023da:	465d      	mov	r5, fp
 80023dc:	433b      	orrs	r3, r7
 80023de:	08cc      	lsrs	r4, r1, #3
 80023e0:	e6ee      	b.n	80021c0 <__aeabi_dsub+0x2f0>
 80023e2:	4662      	mov	r2, ip
 80023e4:	431a      	orrs	r2, r3
 80023e6:	d000      	beq.n	80023ea <__aeabi_dsub+0x51a>
 80023e8:	e082      	b.n	80024f0 <__aeabi_dsub+0x620>
 80023ea:	000b      	movs	r3, r1
 80023ec:	433b      	orrs	r3, r7
 80023ee:	d11b      	bne.n	8002428 <__aeabi_dsub+0x558>
 80023f0:	2480      	movs	r4, #128	; 0x80
 80023f2:	2500      	movs	r5, #0
 80023f4:	0324      	lsls	r4, r4, #12
 80023f6:	e6f9      	b.n	80021ec <__aeabi_dsub+0x31c>
 80023f8:	19dc      	adds	r4, r3, r7
 80023fa:	429c      	cmp	r4, r3
 80023fc:	419b      	sbcs	r3, r3
 80023fe:	4461      	add	r1, ip
 8002400:	4689      	mov	r9, r1
 8002402:	425b      	negs	r3, r3
 8002404:	4499      	add	r9, r3
 8002406:	464b      	mov	r3, r9
 8002408:	021b      	lsls	r3, r3, #8
 800240a:	d444      	bmi.n	8002496 <__aeabi_dsub+0x5c6>
 800240c:	2301      	movs	r3, #1
 800240e:	4698      	mov	r8, r3
 8002410:	e6cc      	b.n	80021ac <__aeabi_dsub+0x2dc>
 8002412:	1bdc      	subs	r4, r3, r7
 8002414:	4662      	mov	r2, ip
 8002416:	42a3      	cmp	r3, r4
 8002418:	419b      	sbcs	r3, r3
 800241a:	1a51      	subs	r1, r2, r1
 800241c:	425b      	negs	r3, r3
 800241e:	1acb      	subs	r3, r1, r3
 8002420:	4699      	mov	r9, r3
 8002422:	2301      	movs	r3, #1
 8002424:	4698      	mov	r8, r3
 8002426:	e5a4      	b.n	8001f72 <__aeabi_dsub+0xa2>
 8002428:	08ff      	lsrs	r7, r7, #3
 800242a:	074b      	lsls	r3, r1, #29
 800242c:	465d      	mov	r5, fp
 800242e:	433b      	orrs	r3, r7
 8002430:	08cc      	lsrs	r4, r1, #3
 8002432:	e6d7      	b.n	80021e4 <__aeabi_dsub+0x314>
 8002434:	4662      	mov	r2, ip
 8002436:	431a      	orrs	r2, r3
 8002438:	0014      	movs	r4, r2
 800243a:	1e63      	subs	r3, r4, #1
 800243c:	419c      	sbcs	r4, r3
 800243e:	e679      	b.n	8002134 <__aeabi_dsub+0x264>
 8002440:	0015      	movs	r5, r2
 8002442:	4664      	mov	r4, ip
 8002444:	3d20      	subs	r5, #32
 8002446:	40ec      	lsrs	r4, r5
 8002448:	46a0      	mov	r8, r4
 800244a:	2a20      	cmp	r2, #32
 800244c:	d005      	beq.n	800245a <__aeabi_dsub+0x58a>
 800244e:	2540      	movs	r5, #64	; 0x40
 8002450:	4664      	mov	r4, ip
 8002452:	1aaa      	subs	r2, r5, r2
 8002454:	4094      	lsls	r4, r2
 8002456:	4323      	orrs	r3, r4
 8002458:	469a      	mov	sl, r3
 800245a:	4654      	mov	r4, sl
 800245c:	1e63      	subs	r3, r4, #1
 800245e:	419c      	sbcs	r4, r3
 8002460:	4643      	mov	r3, r8
 8002462:	4323      	orrs	r3, r4
 8002464:	e773      	b.n	800234e <__aeabi_dsub+0x47e>
 8002466:	4662      	mov	r2, ip
 8002468:	431a      	orrs	r2, r3
 800246a:	d023      	beq.n	80024b4 <__aeabi_dsub+0x5e4>
 800246c:	000a      	movs	r2, r1
 800246e:	433a      	orrs	r2, r7
 8002470:	d000      	beq.n	8002474 <__aeabi_dsub+0x5a4>
 8002472:	e0a0      	b.n	80025b6 <__aeabi_dsub+0x6e6>
 8002474:	4662      	mov	r2, ip
 8002476:	08db      	lsrs	r3, r3, #3
 8002478:	0752      	lsls	r2, r2, #29
 800247a:	4313      	orrs	r3, r2
 800247c:	4662      	mov	r2, ip
 800247e:	08d4      	lsrs	r4, r2, #3
 8002480:	e6b0      	b.n	80021e4 <__aeabi_dsub+0x314>
 8002482:	000b      	movs	r3, r1
 8002484:	433b      	orrs	r3, r7
 8002486:	d100      	bne.n	800248a <__aeabi_dsub+0x5ba>
 8002488:	e728      	b.n	80022dc <__aeabi_dsub+0x40c>
 800248a:	08ff      	lsrs	r7, r7, #3
 800248c:	074b      	lsls	r3, r1, #29
 800248e:	465d      	mov	r5, fp
 8002490:	433b      	orrs	r3, r7
 8002492:	08cc      	lsrs	r4, r1, #3
 8002494:	e697      	b.n	80021c6 <__aeabi_dsub+0x2f6>
 8002496:	2302      	movs	r3, #2
 8002498:	4698      	mov	r8, r3
 800249a:	e736      	b.n	800230a <__aeabi_dsub+0x43a>
 800249c:	1afc      	subs	r4, r7, r3
 800249e:	42a7      	cmp	r7, r4
 80024a0:	41bf      	sbcs	r7, r7
 80024a2:	4663      	mov	r3, ip
 80024a4:	427f      	negs	r7, r7
 80024a6:	1ac9      	subs	r1, r1, r3
 80024a8:	1bcb      	subs	r3, r1, r7
 80024aa:	4699      	mov	r9, r3
 80024ac:	2301      	movs	r3, #1
 80024ae:	465d      	mov	r5, fp
 80024b0:	4698      	mov	r8, r3
 80024b2:	e55e      	b.n	8001f72 <__aeabi_dsub+0xa2>
 80024b4:	074b      	lsls	r3, r1, #29
 80024b6:	08ff      	lsrs	r7, r7, #3
 80024b8:	433b      	orrs	r3, r7
 80024ba:	08cc      	lsrs	r4, r1, #3
 80024bc:	e692      	b.n	80021e4 <__aeabi_dsub+0x314>
 80024be:	1bdc      	subs	r4, r3, r7
 80024c0:	4660      	mov	r0, ip
 80024c2:	42a3      	cmp	r3, r4
 80024c4:	41b6      	sbcs	r6, r6
 80024c6:	1a40      	subs	r0, r0, r1
 80024c8:	4276      	negs	r6, r6
 80024ca:	1b80      	subs	r0, r0, r6
 80024cc:	4681      	mov	r9, r0
 80024ce:	0200      	lsls	r0, r0, #8
 80024d0:	d560      	bpl.n	8002594 <__aeabi_dsub+0x6c4>
 80024d2:	1afc      	subs	r4, r7, r3
 80024d4:	42a7      	cmp	r7, r4
 80024d6:	41bf      	sbcs	r7, r7
 80024d8:	4663      	mov	r3, ip
 80024da:	427f      	negs	r7, r7
 80024dc:	1ac9      	subs	r1, r1, r3
 80024de:	1bcb      	subs	r3, r1, r7
 80024e0:	4699      	mov	r9, r3
 80024e2:	465d      	mov	r5, fp
 80024e4:	e576      	b.n	8001fd4 <__aeabi_dsub+0x104>
 80024e6:	08ff      	lsrs	r7, r7, #3
 80024e8:	074b      	lsls	r3, r1, #29
 80024ea:	433b      	orrs	r3, r7
 80024ec:	08cc      	lsrs	r4, r1, #3
 80024ee:	e667      	b.n	80021c0 <__aeabi_dsub+0x2f0>
 80024f0:	000a      	movs	r2, r1
 80024f2:	08db      	lsrs	r3, r3, #3
 80024f4:	433a      	orrs	r2, r7
 80024f6:	d100      	bne.n	80024fa <__aeabi_dsub+0x62a>
 80024f8:	e66f      	b.n	80021da <__aeabi_dsub+0x30a>
 80024fa:	4662      	mov	r2, ip
 80024fc:	0752      	lsls	r2, r2, #29
 80024fe:	4313      	orrs	r3, r2
 8002500:	4662      	mov	r2, ip
 8002502:	08d4      	lsrs	r4, r2, #3
 8002504:	2280      	movs	r2, #128	; 0x80
 8002506:	0312      	lsls	r2, r2, #12
 8002508:	4214      	tst	r4, r2
 800250a:	d007      	beq.n	800251c <__aeabi_dsub+0x64c>
 800250c:	08c8      	lsrs	r0, r1, #3
 800250e:	4210      	tst	r0, r2
 8002510:	d104      	bne.n	800251c <__aeabi_dsub+0x64c>
 8002512:	465d      	mov	r5, fp
 8002514:	0004      	movs	r4, r0
 8002516:	08fb      	lsrs	r3, r7, #3
 8002518:	0749      	lsls	r1, r1, #29
 800251a:	430b      	orrs	r3, r1
 800251c:	0f5a      	lsrs	r2, r3, #29
 800251e:	00db      	lsls	r3, r3, #3
 8002520:	08db      	lsrs	r3, r3, #3
 8002522:	0752      	lsls	r2, r2, #29
 8002524:	4313      	orrs	r3, r2
 8002526:	e65d      	b.n	80021e4 <__aeabi_dsub+0x314>
 8002528:	074b      	lsls	r3, r1, #29
 800252a:	08ff      	lsrs	r7, r7, #3
 800252c:	433b      	orrs	r3, r7
 800252e:	08cc      	lsrs	r4, r1, #3
 8002530:	e649      	b.n	80021c6 <__aeabi_dsub+0x2f6>
 8002532:	19dc      	adds	r4, r3, r7
 8002534:	429c      	cmp	r4, r3
 8002536:	419b      	sbcs	r3, r3
 8002538:	4461      	add	r1, ip
 800253a:	4689      	mov	r9, r1
 800253c:	425b      	negs	r3, r3
 800253e:	4499      	add	r9, r3
 8002540:	464b      	mov	r3, r9
 8002542:	021b      	lsls	r3, r3, #8
 8002544:	d400      	bmi.n	8002548 <__aeabi_dsub+0x678>
 8002546:	e631      	b.n	80021ac <__aeabi_dsub+0x2dc>
 8002548:	464a      	mov	r2, r9
 800254a:	4b17      	ldr	r3, [pc, #92]	; (80025a8 <__aeabi_dsub+0x6d8>)
 800254c:	401a      	ands	r2, r3
 800254e:	2301      	movs	r3, #1
 8002550:	4691      	mov	r9, r2
 8002552:	4698      	mov	r8, r3
 8002554:	e62a      	b.n	80021ac <__aeabi_dsub+0x2dc>
 8002556:	0016      	movs	r6, r2
 8002558:	4664      	mov	r4, ip
 800255a:	3e20      	subs	r6, #32
 800255c:	40f4      	lsrs	r4, r6
 800255e:	46a0      	mov	r8, r4
 8002560:	2a20      	cmp	r2, #32
 8002562:	d005      	beq.n	8002570 <__aeabi_dsub+0x6a0>
 8002564:	2640      	movs	r6, #64	; 0x40
 8002566:	4664      	mov	r4, ip
 8002568:	1ab2      	subs	r2, r6, r2
 800256a:	4094      	lsls	r4, r2
 800256c:	4323      	orrs	r3, r4
 800256e:	469a      	mov	sl, r3
 8002570:	4654      	mov	r4, sl
 8002572:	1e63      	subs	r3, r4, #1
 8002574:	419c      	sbcs	r4, r3
 8002576:	4643      	mov	r3, r8
 8002578:	431c      	orrs	r4, r3
 800257a:	e5db      	b.n	8002134 <__aeabi_dsub+0x264>
 800257c:	0002      	movs	r2, r0
 800257e:	2400      	movs	r4, #0
 8002580:	2300      	movs	r3, #0
 8002582:	e548      	b.n	8002016 <__aeabi_dsub+0x146>
 8002584:	19dc      	adds	r4, r3, r7
 8002586:	42bc      	cmp	r4, r7
 8002588:	41bf      	sbcs	r7, r7
 800258a:	4461      	add	r1, ip
 800258c:	4689      	mov	r9, r1
 800258e:	427f      	negs	r7, r7
 8002590:	44b9      	add	r9, r7
 8002592:	e738      	b.n	8002406 <__aeabi_dsub+0x536>
 8002594:	464b      	mov	r3, r9
 8002596:	4323      	orrs	r3, r4
 8002598:	d100      	bne.n	800259c <__aeabi_dsub+0x6cc>
 800259a:	e69f      	b.n	80022dc <__aeabi_dsub+0x40c>
 800259c:	e606      	b.n	80021ac <__aeabi_dsub+0x2dc>
 800259e:	46c0      	nop			; (mov r8, r8)
 80025a0:	000007fe 	.word	0x000007fe
 80025a4:	000007ff 	.word	0x000007ff
 80025a8:	ff7fffff 	.word	0xff7fffff
 80025ac:	08ff      	lsrs	r7, r7, #3
 80025ae:	074b      	lsls	r3, r1, #29
 80025b0:	433b      	orrs	r3, r7
 80025b2:	08cc      	lsrs	r4, r1, #3
 80025b4:	e616      	b.n	80021e4 <__aeabi_dsub+0x314>
 80025b6:	4662      	mov	r2, ip
 80025b8:	08db      	lsrs	r3, r3, #3
 80025ba:	0752      	lsls	r2, r2, #29
 80025bc:	4313      	orrs	r3, r2
 80025be:	4662      	mov	r2, ip
 80025c0:	08d4      	lsrs	r4, r2, #3
 80025c2:	2280      	movs	r2, #128	; 0x80
 80025c4:	0312      	lsls	r2, r2, #12
 80025c6:	4214      	tst	r4, r2
 80025c8:	d007      	beq.n	80025da <__aeabi_dsub+0x70a>
 80025ca:	08c8      	lsrs	r0, r1, #3
 80025cc:	4210      	tst	r0, r2
 80025ce:	d104      	bne.n	80025da <__aeabi_dsub+0x70a>
 80025d0:	465d      	mov	r5, fp
 80025d2:	0004      	movs	r4, r0
 80025d4:	08fb      	lsrs	r3, r7, #3
 80025d6:	0749      	lsls	r1, r1, #29
 80025d8:	430b      	orrs	r3, r1
 80025da:	0f5a      	lsrs	r2, r3, #29
 80025dc:	00db      	lsls	r3, r3, #3
 80025de:	0752      	lsls	r2, r2, #29
 80025e0:	08db      	lsrs	r3, r3, #3
 80025e2:	4313      	orrs	r3, r2
 80025e4:	e5fe      	b.n	80021e4 <__aeabi_dsub+0x314>
 80025e6:	2300      	movs	r3, #0
 80025e8:	4a01      	ldr	r2, [pc, #4]	; (80025f0 <__aeabi_dsub+0x720>)
 80025ea:	001c      	movs	r4, r3
 80025ec:	e513      	b.n	8002016 <__aeabi_dsub+0x146>
 80025ee:	46c0      	nop			; (mov r8, r8)
 80025f0:	000007ff 	.word	0x000007ff

080025f4 <__aeabi_dcmpun>:
 80025f4:	b570      	push	{r4, r5, r6, lr}
 80025f6:	0005      	movs	r5, r0
 80025f8:	480c      	ldr	r0, [pc, #48]	; (800262c <__aeabi_dcmpun+0x38>)
 80025fa:	031c      	lsls	r4, r3, #12
 80025fc:	0016      	movs	r6, r2
 80025fe:	005b      	lsls	r3, r3, #1
 8002600:	030a      	lsls	r2, r1, #12
 8002602:	0049      	lsls	r1, r1, #1
 8002604:	0b12      	lsrs	r2, r2, #12
 8002606:	0d49      	lsrs	r1, r1, #21
 8002608:	0b24      	lsrs	r4, r4, #12
 800260a:	0d5b      	lsrs	r3, r3, #21
 800260c:	4281      	cmp	r1, r0
 800260e:	d008      	beq.n	8002622 <__aeabi_dcmpun+0x2e>
 8002610:	4a06      	ldr	r2, [pc, #24]	; (800262c <__aeabi_dcmpun+0x38>)
 8002612:	2000      	movs	r0, #0
 8002614:	4293      	cmp	r3, r2
 8002616:	d103      	bne.n	8002620 <__aeabi_dcmpun+0x2c>
 8002618:	0020      	movs	r0, r4
 800261a:	4330      	orrs	r0, r6
 800261c:	1e43      	subs	r3, r0, #1
 800261e:	4198      	sbcs	r0, r3
 8002620:	bd70      	pop	{r4, r5, r6, pc}
 8002622:	2001      	movs	r0, #1
 8002624:	432a      	orrs	r2, r5
 8002626:	d1fb      	bne.n	8002620 <__aeabi_dcmpun+0x2c>
 8002628:	e7f2      	b.n	8002610 <__aeabi_dcmpun+0x1c>
 800262a:	46c0      	nop			; (mov r8, r8)
 800262c:	000007ff 	.word	0x000007ff

08002630 <__aeabi_d2iz>:
 8002630:	000a      	movs	r2, r1
 8002632:	b530      	push	{r4, r5, lr}
 8002634:	4c13      	ldr	r4, [pc, #76]	; (8002684 <__aeabi_d2iz+0x54>)
 8002636:	0053      	lsls	r3, r2, #1
 8002638:	0309      	lsls	r1, r1, #12
 800263a:	0005      	movs	r5, r0
 800263c:	0b09      	lsrs	r1, r1, #12
 800263e:	2000      	movs	r0, #0
 8002640:	0d5b      	lsrs	r3, r3, #21
 8002642:	0fd2      	lsrs	r2, r2, #31
 8002644:	42a3      	cmp	r3, r4
 8002646:	dd04      	ble.n	8002652 <__aeabi_d2iz+0x22>
 8002648:	480f      	ldr	r0, [pc, #60]	; (8002688 <__aeabi_d2iz+0x58>)
 800264a:	4283      	cmp	r3, r0
 800264c:	dd02      	ble.n	8002654 <__aeabi_d2iz+0x24>
 800264e:	4b0f      	ldr	r3, [pc, #60]	; (800268c <__aeabi_d2iz+0x5c>)
 8002650:	18d0      	adds	r0, r2, r3
 8002652:	bd30      	pop	{r4, r5, pc}
 8002654:	2080      	movs	r0, #128	; 0x80
 8002656:	0340      	lsls	r0, r0, #13
 8002658:	4301      	orrs	r1, r0
 800265a:	480d      	ldr	r0, [pc, #52]	; (8002690 <__aeabi_d2iz+0x60>)
 800265c:	1ac0      	subs	r0, r0, r3
 800265e:	281f      	cmp	r0, #31
 8002660:	dd08      	ble.n	8002674 <__aeabi_d2iz+0x44>
 8002662:	480c      	ldr	r0, [pc, #48]	; (8002694 <__aeabi_d2iz+0x64>)
 8002664:	1ac3      	subs	r3, r0, r3
 8002666:	40d9      	lsrs	r1, r3
 8002668:	000b      	movs	r3, r1
 800266a:	4258      	negs	r0, r3
 800266c:	2a00      	cmp	r2, #0
 800266e:	d1f0      	bne.n	8002652 <__aeabi_d2iz+0x22>
 8002670:	0018      	movs	r0, r3
 8002672:	e7ee      	b.n	8002652 <__aeabi_d2iz+0x22>
 8002674:	4c08      	ldr	r4, [pc, #32]	; (8002698 <__aeabi_d2iz+0x68>)
 8002676:	40c5      	lsrs	r5, r0
 8002678:	46a4      	mov	ip, r4
 800267a:	4463      	add	r3, ip
 800267c:	4099      	lsls	r1, r3
 800267e:	000b      	movs	r3, r1
 8002680:	432b      	orrs	r3, r5
 8002682:	e7f2      	b.n	800266a <__aeabi_d2iz+0x3a>
 8002684:	000003fe 	.word	0x000003fe
 8002688:	0000041d 	.word	0x0000041d
 800268c:	7fffffff 	.word	0x7fffffff
 8002690:	00000433 	.word	0x00000433
 8002694:	00000413 	.word	0x00000413
 8002698:	fffffbed 	.word	0xfffffbed

0800269c <__aeabi_i2d>:
 800269c:	b570      	push	{r4, r5, r6, lr}
 800269e:	2800      	cmp	r0, #0
 80026a0:	d016      	beq.n	80026d0 <__aeabi_i2d+0x34>
 80026a2:	17c3      	asrs	r3, r0, #31
 80026a4:	18c5      	adds	r5, r0, r3
 80026a6:	405d      	eors	r5, r3
 80026a8:	0fc4      	lsrs	r4, r0, #31
 80026aa:	0028      	movs	r0, r5
 80026ac:	f000 f91c 	bl	80028e8 <__clzsi2>
 80026b0:	4a11      	ldr	r2, [pc, #68]	; (80026f8 <__aeabi_i2d+0x5c>)
 80026b2:	1a12      	subs	r2, r2, r0
 80026b4:	280a      	cmp	r0, #10
 80026b6:	dc16      	bgt.n	80026e6 <__aeabi_i2d+0x4a>
 80026b8:	0003      	movs	r3, r0
 80026ba:	002e      	movs	r6, r5
 80026bc:	3315      	adds	r3, #21
 80026be:	409e      	lsls	r6, r3
 80026c0:	230b      	movs	r3, #11
 80026c2:	1a18      	subs	r0, r3, r0
 80026c4:	40c5      	lsrs	r5, r0
 80026c6:	0552      	lsls	r2, r2, #21
 80026c8:	032d      	lsls	r5, r5, #12
 80026ca:	0b2d      	lsrs	r5, r5, #12
 80026cc:	0d53      	lsrs	r3, r2, #21
 80026ce:	e003      	b.n	80026d8 <__aeabi_i2d+0x3c>
 80026d0:	2400      	movs	r4, #0
 80026d2:	2300      	movs	r3, #0
 80026d4:	2500      	movs	r5, #0
 80026d6:	2600      	movs	r6, #0
 80026d8:	051b      	lsls	r3, r3, #20
 80026da:	432b      	orrs	r3, r5
 80026dc:	07e4      	lsls	r4, r4, #31
 80026de:	4323      	orrs	r3, r4
 80026e0:	0030      	movs	r0, r6
 80026e2:	0019      	movs	r1, r3
 80026e4:	bd70      	pop	{r4, r5, r6, pc}
 80026e6:	380b      	subs	r0, #11
 80026e8:	4085      	lsls	r5, r0
 80026ea:	0552      	lsls	r2, r2, #21
 80026ec:	032d      	lsls	r5, r5, #12
 80026ee:	2600      	movs	r6, #0
 80026f0:	0b2d      	lsrs	r5, r5, #12
 80026f2:	0d53      	lsrs	r3, r2, #21
 80026f4:	e7f0      	b.n	80026d8 <__aeabi_i2d+0x3c>
 80026f6:	46c0      	nop			; (mov r8, r8)
 80026f8:	0000041e 	.word	0x0000041e

080026fc <__aeabi_ui2d>:
 80026fc:	b510      	push	{r4, lr}
 80026fe:	1e04      	subs	r4, r0, #0
 8002700:	d010      	beq.n	8002724 <__aeabi_ui2d+0x28>
 8002702:	f000 f8f1 	bl	80028e8 <__clzsi2>
 8002706:	4b0f      	ldr	r3, [pc, #60]	; (8002744 <__aeabi_ui2d+0x48>)
 8002708:	1a1b      	subs	r3, r3, r0
 800270a:	280a      	cmp	r0, #10
 800270c:	dc11      	bgt.n	8002732 <__aeabi_ui2d+0x36>
 800270e:	220b      	movs	r2, #11
 8002710:	0021      	movs	r1, r4
 8002712:	1a12      	subs	r2, r2, r0
 8002714:	40d1      	lsrs	r1, r2
 8002716:	3015      	adds	r0, #21
 8002718:	030a      	lsls	r2, r1, #12
 800271a:	055b      	lsls	r3, r3, #21
 800271c:	4084      	lsls	r4, r0
 800271e:	0b12      	lsrs	r2, r2, #12
 8002720:	0d5b      	lsrs	r3, r3, #21
 8002722:	e001      	b.n	8002728 <__aeabi_ui2d+0x2c>
 8002724:	2300      	movs	r3, #0
 8002726:	2200      	movs	r2, #0
 8002728:	051b      	lsls	r3, r3, #20
 800272a:	4313      	orrs	r3, r2
 800272c:	0020      	movs	r0, r4
 800272e:	0019      	movs	r1, r3
 8002730:	bd10      	pop	{r4, pc}
 8002732:	0022      	movs	r2, r4
 8002734:	380b      	subs	r0, #11
 8002736:	4082      	lsls	r2, r0
 8002738:	055b      	lsls	r3, r3, #21
 800273a:	0312      	lsls	r2, r2, #12
 800273c:	2400      	movs	r4, #0
 800273e:	0b12      	lsrs	r2, r2, #12
 8002740:	0d5b      	lsrs	r3, r3, #21
 8002742:	e7f1      	b.n	8002728 <__aeabi_ui2d+0x2c>
 8002744:	0000041e 	.word	0x0000041e

08002748 <__aeabi_f2d>:
 8002748:	b570      	push	{r4, r5, r6, lr}
 800274a:	0043      	lsls	r3, r0, #1
 800274c:	0246      	lsls	r6, r0, #9
 800274e:	0fc4      	lsrs	r4, r0, #31
 8002750:	20fe      	movs	r0, #254	; 0xfe
 8002752:	0e1b      	lsrs	r3, r3, #24
 8002754:	1c59      	adds	r1, r3, #1
 8002756:	0a75      	lsrs	r5, r6, #9
 8002758:	4208      	tst	r0, r1
 800275a:	d00c      	beq.n	8002776 <__aeabi_f2d+0x2e>
 800275c:	22e0      	movs	r2, #224	; 0xe0
 800275e:	0092      	lsls	r2, r2, #2
 8002760:	4694      	mov	ip, r2
 8002762:	076d      	lsls	r5, r5, #29
 8002764:	0b36      	lsrs	r6, r6, #12
 8002766:	4463      	add	r3, ip
 8002768:	051b      	lsls	r3, r3, #20
 800276a:	4333      	orrs	r3, r6
 800276c:	07e4      	lsls	r4, r4, #31
 800276e:	4323      	orrs	r3, r4
 8002770:	0028      	movs	r0, r5
 8002772:	0019      	movs	r1, r3
 8002774:	bd70      	pop	{r4, r5, r6, pc}
 8002776:	2b00      	cmp	r3, #0
 8002778:	d114      	bne.n	80027a4 <__aeabi_f2d+0x5c>
 800277a:	2d00      	cmp	r5, #0
 800277c:	d01b      	beq.n	80027b6 <__aeabi_f2d+0x6e>
 800277e:	0028      	movs	r0, r5
 8002780:	f000 f8b2 	bl	80028e8 <__clzsi2>
 8002784:	280a      	cmp	r0, #10
 8002786:	dc1c      	bgt.n	80027c2 <__aeabi_f2d+0x7a>
 8002788:	230b      	movs	r3, #11
 800278a:	002e      	movs	r6, r5
 800278c:	1a1b      	subs	r3, r3, r0
 800278e:	40de      	lsrs	r6, r3
 8002790:	0003      	movs	r3, r0
 8002792:	3315      	adds	r3, #21
 8002794:	409d      	lsls	r5, r3
 8002796:	4a0e      	ldr	r2, [pc, #56]	; (80027d0 <__aeabi_f2d+0x88>)
 8002798:	0336      	lsls	r6, r6, #12
 800279a:	1a12      	subs	r2, r2, r0
 800279c:	0552      	lsls	r2, r2, #21
 800279e:	0b36      	lsrs	r6, r6, #12
 80027a0:	0d53      	lsrs	r3, r2, #21
 80027a2:	e7e1      	b.n	8002768 <__aeabi_f2d+0x20>
 80027a4:	2d00      	cmp	r5, #0
 80027a6:	d009      	beq.n	80027bc <__aeabi_f2d+0x74>
 80027a8:	2280      	movs	r2, #128	; 0x80
 80027aa:	0b36      	lsrs	r6, r6, #12
 80027ac:	0312      	lsls	r2, r2, #12
 80027ae:	4b09      	ldr	r3, [pc, #36]	; (80027d4 <__aeabi_f2d+0x8c>)
 80027b0:	076d      	lsls	r5, r5, #29
 80027b2:	4316      	orrs	r6, r2
 80027b4:	e7d8      	b.n	8002768 <__aeabi_f2d+0x20>
 80027b6:	2300      	movs	r3, #0
 80027b8:	2600      	movs	r6, #0
 80027ba:	e7d5      	b.n	8002768 <__aeabi_f2d+0x20>
 80027bc:	2600      	movs	r6, #0
 80027be:	4b05      	ldr	r3, [pc, #20]	; (80027d4 <__aeabi_f2d+0x8c>)
 80027c0:	e7d2      	b.n	8002768 <__aeabi_f2d+0x20>
 80027c2:	0003      	movs	r3, r0
 80027c4:	3b0b      	subs	r3, #11
 80027c6:	409d      	lsls	r5, r3
 80027c8:	002e      	movs	r6, r5
 80027ca:	2500      	movs	r5, #0
 80027cc:	e7e3      	b.n	8002796 <__aeabi_f2d+0x4e>
 80027ce:	46c0      	nop			; (mov r8, r8)
 80027d0:	00000389 	.word	0x00000389
 80027d4:	000007ff 	.word	0x000007ff

080027d8 <__aeabi_d2f>:
 80027d8:	0002      	movs	r2, r0
 80027da:	004b      	lsls	r3, r1, #1
 80027dc:	b5f0      	push	{r4, r5, r6, r7, lr}
 80027de:	0d5b      	lsrs	r3, r3, #21
 80027e0:	030c      	lsls	r4, r1, #12
 80027e2:	4e3d      	ldr	r6, [pc, #244]	; (80028d8 <__aeabi_d2f+0x100>)
 80027e4:	0a64      	lsrs	r4, r4, #9
 80027e6:	0f40      	lsrs	r0, r0, #29
 80027e8:	1c5f      	adds	r7, r3, #1
 80027ea:	0fc9      	lsrs	r1, r1, #31
 80027ec:	4304      	orrs	r4, r0
 80027ee:	00d5      	lsls	r5, r2, #3
 80027f0:	4237      	tst	r7, r6
 80027f2:	d00a      	beq.n	800280a <__aeabi_d2f+0x32>
 80027f4:	4839      	ldr	r0, [pc, #228]	; (80028dc <__aeabi_d2f+0x104>)
 80027f6:	181e      	adds	r6, r3, r0
 80027f8:	2efe      	cmp	r6, #254	; 0xfe
 80027fa:	dd16      	ble.n	800282a <__aeabi_d2f+0x52>
 80027fc:	20ff      	movs	r0, #255	; 0xff
 80027fe:	2400      	movs	r4, #0
 8002800:	05c0      	lsls	r0, r0, #23
 8002802:	4320      	orrs	r0, r4
 8002804:	07c9      	lsls	r1, r1, #31
 8002806:	4308      	orrs	r0, r1
 8002808:	bdf0      	pop	{r4, r5, r6, r7, pc}
 800280a:	2b00      	cmp	r3, #0
 800280c:	d106      	bne.n	800281c <__aeabi_d2f+0x44>
 800280e:	432c      	orrs	r4, r5
 8002810:	d026      	beq.n	8002860 <__aeabi_d2f+0x88>
 8002812:	2205      	movs	r2, #5
 8002814:	0192      	lsls	r2, r2, #6
 8002816:	0a54      	lsrs	r4, r2, #9
 8002818:	b2d8      	uxtb	r0, r3
 800281a:	e7f1      	b.n	8002800 <__aeabi_d2f+0x28>
 800281c:	4325      	orrs	r5, r4
 800281e:	d0ed      	beq.n	80027fc <__aeabi_d2f+0x24>
 8002820:	2080      	movs	r0, #128	; 0x80
 8002822:	03c0      	lsls	r0, r0, #15
 8002824:	4304      	orrs	r4, r0
 8002826:	20ff      	movs	r0, #255	; 0xff
 8002828:	e7ea      	b.n	8002800 <__aeabi_d2f+0x28>
 800282a:	2e00      	cmp	r6, #0
 800282c:	dd1b      	ble.n	8002866 <__aeabi_d2f+0x8e>
 800282e:	0192      	lsls	r2, r2, #6
 8002830:	1e53      	subs	r3, r2, #1
 8002832:	419a      	sbcs	r2, r3
 8002834:	00e4      	lsls	r4, r4, #3
 8002836:	0f6d      	lsrs	r5, r5, #29
 8002838:	4322      	orrs	r2, r4
 800283a:	432a      	orrs	r2, r5
 800283c:	0753      	lsls	r3, r2, #29
 800283e:	d048      	beq.n	80028d2 <__aeabi_d2f+0xfa>
 8002840:	230f      	movs	r3, #15
 8002842:	4013      	ands	r3, r2
 8002844:	2b04      	cmp	r3, #4
 8002846:	d000      	beq.n	800284a <__aeabi_d2f+0x72>
 8002848:	3204      	adds	r2, #4
 800284a:	2380      	movs	r3, #128	; 0x80
 800284c:	04db      	lsls	r3, r3, #19
 800284e:	4013      	ands	r3, r2
 8002850:	d03f      	beq.n	80028d2 <__aeabi_d2f+0xfa>
 8002852:	1c70      	adds	r0, r6, #1
 8002854:	2efe      	cmp	r6, #254	; 0xfe
 8002856:	d0d1      	beq.n	80027fc <__aeabi_d2f+0x24>
 8002858:	0192      	lsls	r2, r2, #6
 800285a:	0a54      	lsrs	r4, r2, #9
 800285c:	b2c0      	uxtb	r0, r0
 800285e:	e7cf      	b.n	8002800 <__aeabi_d2f+0x28>
 8002860:	2000      	movs	r0, #0
 8002862:	2400      	movs	r4, #0
 8002864:	e7cc      	b.n	8002800 <__aeabi_d2f+0x28>
 8002866:	0032      	movs	r2, r6
 8002868:	3217      	adds	r2, #23
 800286a:	db22      	blt.n	80028b2 <__aeabi_d2f+0xda>
 800286c:	2080      	movs	r0, #128	; 0x80
 800286e:	0400      	lsls	r0, r0, #16
 8002870:	4320      	orrs	r0, r4
 8002872:	241e      	movs	r4, #30
 8002874:	1ba4      	subs	r4, r4, r6
 8002876:	2c1f      	cmp	r4, #31
 8002878:	dd1d      	ble.n	80028b6 <__aeabi_d2f+0xde>
 800287a:	2202      	movs	r2, #2
 800287c:	4252      	negs	r2, r2
 800287e:	1b96      	subs	r6, r2, r6
 8002880:	0002      	movs	r2, r0
 8002882:	40f2      	lsrs	r2, r6
 8002884:	0016      	movs	r6, r2
 8002886:	2c20      	cmp	r4, #32
 8002888:	d004      	beq.n	8002894 <__aeabi_d2f+0xbc>
 800288a:	4a15      	ldr	r2, [pc, #84]	; (80028e0 <__aeabi_d2f+0x108>)
 800288c:	4694      	mov	ip, r2
 800288e:	4463      	add	r3, ip
 8002890:	4098      	lsls	r0, r3
 8002892:	4305      	orrs	r5, r0
 8002894:	002a      	movs	r2, r5
 8002896:	1e53      	subs	r3, r2, #1
 8002898:	419a      	sbcs	r2, r3
 800289a:	4332      	orrs	r2, r6
 800289c:	2600      	movs	r6, #0
 800289e:	0753      	lsls	r3, r2, #29
 80028a0:	d1ce      	bne.n	8002840 <__aeabi_d2f+0x68>
 80028a2:	2480      	movs	r4, #128	; 0x80
 80028a4:	0013      	movs	r3, r2
 80028a6:	04e4      	lsls	r4, r4, #19
 80028a8:	2001      	movs	r0, #1
 80028aa:	4023      	ands	r3, r4
 80028ac:	4222      	tst	r2, r4
